:020000040800F2
:1080000020CA00204DB50008DD8F0008E78F00086A
:10801000F98F0008039000080D9000080000000090
:10802000000000000000000000000000598200086D
:1080300021900008000000008D8200086BF300080A
:1080400067B5000867B5000867B5000867B50008A0
:1080500067B5000867B5000881E60008ABE60008D0
:10806000D1E60008F7E6000867B5000867B5000824
:1080700067B5000867B5000867B5000867B5000870
:1080800067B5000867B5000867B5000867B5000860
:1080900067B5000867B5000867B500081DE7000868
:1080A00067B5000867B5000867B5000867B5000840
:1080B00067B50008E1D6000867B5000867B5000895
:1080C00067B5000867B5000867B5000867B5000820
:1080D00067B500082529010867B5000867B50008DD
:1080E0008BE7000867B5000867B5000867B50008AA
:1080F00067B5000867B5000867B5000867B50008F0
:1081000067B5000867B5000867B5000867B50008DF
:1081100067B5000867B500084FD7000867B50008C5
:1081200067B5000867B5000867B5000867B50008BF
:1081300000F002F800F080F80AA090E8000C8244F9
:108140008344AAF10107DA4501D100F075F8AFF2D6
:10815000090EBAE80F0013F0010F18BFFB1A43F025
:10816000010318478CAF0100ACAF01000A444FF087
:10817000000C10F8013B13F0070408BF10F8014B86
:108180001D1108BF10F8015B641E05D010F8016BCB
:10819000641E01F8016BF9D113F0080F1EBF10F82F
:1081A000014BAD1C0C1B09D16D1E58BF01F801CB52
:1081B000FAD505E014F8016B01F8016B6D1EF9D5D5
:1081C0009142D6D3704700000023002400250026EA
:1081D000103A28BF78C1FBD8520728BF30C148BF2A
:1081E0000B607047642917F07F84752917F07C8431
:1081F0000020704710B510BD70477047704770473A
:1082000054656D636F5049443533202000000048A9
:10821000003530001FB517F076FE18F0A1F9040004
:108220000020002119F08CFD401C6060002000211E
:1082300019F09CFDE0601FBD18F0D0FB1146FFF760
:10824000E9FF00F02EFE18F06BFE03B4FFF7D2FF3B
:1082500003BC07F02BF900001A4B19680868B0E856
:10826000F00F80F309884FF0000080F311884EF082
:108270000D0E70470000000003480068006880F39E
:10828000088862B600DF00BF08ED00E0EFF3098068
:108290000C4B1A6820E9F00F106008B54FF0BF00D2
:1082A00080F3118806F09CFD4FF0000080F31188E8
:1082B000BDE8084019680868B0E8F00F80F3098845
:1082C000704700BFB800002001B44FF0BF0080F33A
:1082D000118801BC704701B44FF0000080F3118891
:1082E00001BC70470B49D1F800C04A685CF8043BF8
:1082F0001068184442F8040B8C4528BFA1F1DC0C2F
:108300008A4228BFA1F1DC02C1F800C04A6020F017
:1083100000407047B8B7002010B501210D2001F0D2
:1083200019FE0121FA4801F00AFC10BD10B510F049
:108330003DFAF848006810F040FA0FF001FD4FF0E8
:10834000FF300DF0DAFF2020F3490870F349087080
:108350003420F34908800DF093FE10BD86B0002450
:10836000FFF7E4FF002010F0BBFE002011F06CFDD1
:1083700000BFEC48807C80B9002003464FF41672A1
:10838000E949009001A810F0E4F904462CB100235B
:108390002246E54901A811F01AFD052007F055F91C
:1083A000E7E738B5E148007860B90120DF49087097
:1083B0004FF4FA71DE4807F06BF942F21071DD48B4
:1083C00007F066F909F002F9DB49088008460088E1
:1083D000002835DD0220D9490870800207F0D3F962
:1083E000D7498989884217D1012007F0C6FBD248B6
:1083F000008800286DDD08F0C8FE09F0EFF80220C3
:10840000D0490870D048006800680090CE490968DB
:10841000C88807F0B8F95CE040F6060007F0B3F949
:10842000C7498989884254D108F043FEC248008870
:1084300000284EDD09F0D2F80220C249087048E059
:10844000BB4807F038F9002843D0B94807F028F9AD
:10845000002418E000BF04EB8400BC4901EBC0001D
:10846000BB490860022007F088FB00BFB2480088C3
:10847000002806DD08F089FE09F0B0F80220B149B5
:108480000870601CC4B21E2CE4DB002416E000BFA0
:10849000B04800EB8410AC490860052007F06DFB84
:1084A00000BFA5480088002806DD08F06EFE09F030
:1084B00095F80220A3490870601CC4B20A2CE6DBC0
:1084C0009C4807F0F8F820B19A4807F0E9F808F05E
:1084D00042FD38BD002405E0322007F0B6F89EA02A
:1084E00017F0E2FA08F02CFF0028F5D100BFFFF7E3
:1084F00058FFA0480078012803D09F480078012841
:1085000009D1601CC4B20A2C05D10024002099496D
:1085100008700AF03BFB01F098FB022007F095F889
:10852000E5E710B595480068012805D19448008812
:10853000401C9349088002E000209149088090483F
:108540000088642804DD00208D4908800AF0E2F9E3
:1085500010BD0AF010FB00BFFFF7E3FF8948007869
:1085600050B188480078401E864908700846007857
:10857000012801D10CF070FB83480078002809DD48
:1085800081480078401E804908700846007808B984
:108590000AF0C0F9052007F058F8DDE702F0F6FF11
:1085A00000207A4908707A49088000BF794800782D
:1085B000401C7849087008460078022803DB002038
:1085C000087003F055F874488088401C7249888010
:1085D0000A2007F03AF871480078401C6F4908708B
:1085E000084600786428E1DB0DF01EFD07F05FF916
:1085F00000206A490870D9E700BF002431E06848CC
:1086000030F8140001282AD1464A403212F83410BA
:10861000A20002F1BE0004F03DFD424A403202EBEE
:10862000C4025178A20002F1BF0004F033FD3D4ABC
:10863000403202EBC4029178A20002F1C00004F0C3
:1086400029FD384A403202EBC402D178A20002F17F
:10865000C10004F01FFD0020514921F81400601CE6
:10866000C4B2202CCBDB40F6B83006F0EEFFC4E7F6
:1086700005F0F2FB00BFFFF727FE4A48046805F04B
:108680008DFE48480068051B681D0521B0FBF1F010
:108690004549098808444449088008460088C82894
:1086A00001DB0EF05DFA40480088B0F57A7F04DB0C
:1086B00000203D4908800EF0B7FB052006F0C5FFFD
:1086C00035480089401C34490881FFF7FDFDD2E799
:1086D0007CB504F0AFFC1D2004F0B0FC8DF8000068
:1086E000202004F0ABFC8DF801009DF800109DF8EF
:1086F000010001EB00202D4908800DF0CFFB9428EC
:108700005AD10A202449888229A00CF00DFB7DE073
:108710000004300004000020E9010020EB010020EB
:10872000EA010020506000203C04002024000020CA
:10873000140000201C0000203C0100205B000020F1
:10874000904800205C000020480100209450002048
:1087500044010020805500207461706465765F6973
:108760006E69742829206661696C6564202E2E2E3E
:108770000D0A00008201002000000020A00121421B
:10878000100000208A010020880100200A0000203B
:108790000C0000200E000020E06700200F000020E9
:1087A000941600206400002012000020C001002068
:1087B00054335F33324149000DF070FB40F2CA512F
:1087C000884203D11420FE4988821FE01E20FC4904
:1087D00088821422FB4940F2BA2004F0CFFCF94809
:1087E0000078FF2812D1F7484078FF280ED1F548CD
:1087F0008078FF280AD1F348C078FF2806D1F148D5
:108800000079FF2802D1F0A00CF08EFA002004F0CD
:1088100015FCF0490870012004F010FCED49487087
:10882000022004F00BFCEB498870032004F006FCE6
:10883000E849C87008460078FF2811D108464078FA
:10884000FF280DD108468078FF2809D10846C07856
:10885000FF2805D101200870487002208870C87078
:10886000002407E004F1160004F0E8FB0DF8040012
:10887000601CC4B2042CF5DB9DF800009DF80110CB
:1088800000EB01209DF8021000EB01409DF8031061
:1088900000EB0160D049086008460068401C70B1D8
:1088A0000846008880B24FF6FF71884207D0CA4858
:1088B000006820B1C8480068B0F5800F0FD3C548E4
:1088C0000078C449497800EB0120C249897800EB5F
:1088D0000140C049C97800EB0160BF49086004202D
:1088E00004F0ACFB8DF80000052004F0A7FB8DF828
:1088F00001009DF800109DF8010001EB002085B2F9
:108900004821042004F0C6FB0021052004F0C2FB2E
:108910003F2D02DA04200EF043FB062004F08EFB0C
:10892000AC49087108460079FF2802D00846007952
:1089300038B9FE20A749087108460179062004F0DD
:10894000A9FB3520A3498873122004F077FBA349C3
:10895000087008460078FF2803D0084600780128F0
:1089600007DCFE209D49087008460178122004F0BB
:1089700091FB984800799A4908701B2004F05EFB2F
:108980008DF800001C2004F059FB8DF801009DF8C3
:108990000000FF2801D1012000E000209DF8011017
:1089A000FF2901D1012100E00021084020B14BF650
:1089B000C0208849888707E09DF801009DF80010D5
:1089C00040EA012083498887082004F037FB814969
:1089D000C8730846C07BFF2802D00846C07B10B988
:1089E00003207C49C873102004F028FB79494873A0
:1089F000112004F023FB77490874132004F01EFBB8
:108A000074490873152004F019FB8DF800007148B3
:108A1000007B052802DD01206E4908739DF80000E7
:108A20006C49097B884204D06A48017B152004F018
:108A300031FB6848007B062834D2DFE800F0030BE6
:108A4000131B232B4FF4165062498860062065499A
:108A5000087028E04FF496405E4988600320614921
:108A6000087020E04FF416405A49886002205D49A2
:108A7000087018E04FF46140564988600120594958
:108A8000087010E04FF4E1305249886001205549E8
:108A9000087008E04FF496304E4988600120514933
:108AA000087000E000BF00BF4A49886806F018FD62
:108AB000142004F0C3FA474988740846807C0328D0
:108AC00004D00846807C08B103208874002407E0A5
:108AD00004F1280004F0B2FA0DF80400601CC4B2DE
:108AE000062CF5DB9DF80000FF2825D19DF801003C
:108AF000FF2821D19DF80200FF281DD19DF8030019
:108B0000FF2819D19DF80400FF2815D19DF8050014
:108B1000FF2811D104208DF8000002208DF80100FB
:108B200035208DF80200AF208DF8030000208DF86D
:108B3000040001208DF80500002406E01DF8041053
:108B4000244814300155601CC4B2062CF6DB002406
:108B500007E004F12F0004F071FA0DF80400601C26
:108B6000C4B2042CF5DB9DF80000FF2841D19DF82C
:108B70000100FF283DD19DF80200FF2839D19DF862
:108B80000300FF2835D1C0208DF80000A8208DF803
:108B9000010000208DF8020003208DF803009DF8ED
:108BA00000102F2004F076FA9DF80110302004F018
:108BB00071FA9DF80210312004F06CFA14E0000004
:108BC000E0670020C06200203372642070726F641E
:108BD0007563740050600020040000208F010020A5
:108BE0008E010020890100209DF80310322004F03E
:108BF00051FA002408E01DF80410E1480155015D18
:108C000011300155601CC4B2042CF4DB2E2004F09A
:108C100015FA8DF800009DF80000012807DD0020FE
:108C20008DF800009DF800102E2004F033FA9DF816
:108C30000000D3491A3988770846807F81F82F00D1
:108C4000002407E004F1330004F0F8F90DF8040003
:108C5000601CC4B2042CF5DB9DF80000FF2828D16D
:108C60009DF80100FF2824D19DF80200FF2820D1A3
:108C70009DF80300FF281CD18DF800008DF801003D
:108C80008DF8020000208DF803009DF800103320BD
:108C900004F000FA9DF80110342004F0FBF99DF86F
:108CA0000210352004F0F6F99DF80310362004F088
:108CB000F1F9002409E01DF80410B148401D0155E8
:108CC000015D11300155601CC4B2042CF3DB00249B
:108CD00007E004F1370004F0B1F90DF80400601C5E
:108CE000C4B2042CF5DB9DF80000FF282BD19DF8C1
:108CF0000100FF2827D19DF80200FF2823D19DF80D
:108D00000300FF281FD1C0208DF80000A8208DF897
:108D1000010000208DF8020004208DF803009DF86A
:108D20000010372004F0B6F99DF80110382004F047
:108D3000B1F99DF80210392004F0ACF99DF8031048
:108D40003A2004F0A7F9002409E01DF804108C482B
:108D500009300155015D11300155601CC4B2042C6D
:108D6000F3DB3B2004F06AF98DF800009DF8000069
:108D7000FF2807D100208DF800009DF800103B204F
:108D800004F088F99DF800007D491A3981F8270020
:108D9000084690F8270081F838003C2004F04EF98E
:108DA0008DF800003D2004F049F98DF801009DF890
:108DB0000000FF2812D19DF80100FF280ED14FF4CA
:108DC000FB706F491A3908850846008D000A8DF836
:108DD0000000084690F828008DF801009DF8010079
:108DE0009DF8001040EA012065491A3908850846B7
:108DF000008D4887002081F83E00C8740C2004F0E4
:108E00001DF960490870002448E0A10001F1BE008E
:108E100004F014F95A49263101F83400A10001F197
:108E2000BF0004F00BF95649263101EBC40148702C
:108E3000A10001F1C00004F001F95149263101EB14
:108E4000C4018870A10001F1C10004F0F7F84C4999
:108E5000263101EBC401C8704948263010F83400AF
:108E6000FF2819D14648263000EBC4004078FF287F
:108E700012D14348263000EBC4008078FF280BD184
:108E80003F48263000EBC400C078FF2804D1002101
:108E90003B48263040F83410601CC4B2202CB4DBB0
:108EA0007CBD1FB53849080300F02BFAFFF734FAF0
:108EB0004FF4A06000F0EEF90121202001F04AF803
:108EC000482006F073FBFFF703FC0EF09BF804F05C
:108ED000B7F904F03DFA0EF077FA2CA016F0E4FD95
:108EE00000200323CDE900300290034680222AA10E
:108EF00003902B4805F006FD00200123CDE900304A
:108F000002900346802227A10390AFF6131005F0CC
:108F1000F9FC00200223CDE90030029003468022B4
:108F200023A10390244805F0EDFC00200423CDE9A3
:108F3000003002900346802220A10390214805F0D2
:108F4000E1FC00200123CDE90030029003464FF4FC
:108F500020721DA103901D4805F0D4FC00200423BD
:108F6000CDE90030029003464FF4207218A103901F
:108F7000194805F0C7FC06F04DF8002004B010BDFC
:108F80006A600020090000200080000854335F73ED
:108F900065726965730A0D00494E505554530000BF
:108FA0007186000853544F5245454550000000005B
:108FB0004C454430000000009D850008434F4D4D56
:108FC00000000000538500084E455400D584000879
:108FD0004D535450000000005D83000810B518A0E8
:108FE00016F062FD10BD06E01848838842880188AB
:108FF00017A016F059FDF7E702E01BA016F054FD8C
:10900000FBE702E01BA016F04FFDFBE702E01CA00F
:1090100016F04AFDFBE710B51DA016F045FD10BD8A
:1090200010B51DA016F040FD10BD10B51CA016F027
:109030003BFD10BD10B51CA016F036FD10BD0000A4
:109040004E4D49206661756C74000000E067002099
:1090500048617264204661756C742025642C256417
:109060002C256420000000004D656D204661756C64
:1090700074200000427573204661756C74200000F6
:109080005573616765204661756C742000000000AF
:1090900053564320000000004465627567200000BD
:1090A00050656E20000000005379735469636B2093
:1090B000000000000CB50020019000906C48006892
:1090C00040F480306A49086000BF6948006800F4D5
:1090D000003000900198401C0190009818B9019848
:1090E000B0F5A06FF1D16248006800F4003010B113
:1090F0000120009001E0002000900098012843D159
:109100005C48006840F010005A4908600846006852
:1091100020F0030008600846006840F00200086084
:1091200053484068524948600846406848600846CD
:10913000406840F4806048600846406820F47C1035
:1091400048600846406840F4E810486008460068F7
:1091500040F08070086000BF4548006800F0007073
:109160000028F9D04248406820F003004049486098
:109170000846406840F00200486000BF3C48406834
:1091800000F00C000828F9D10CBD10B5FFF792FFD4
:1091900010BD10B53648006840F001003449086041
:1091A000084640683449084031494860084600682C
:1091B000324908402E4908600846006820F48020A3
:1091C00008600846406820F4FE0048604FF41F0025
:1091D0008860FFF7DAFF4FF000602949086010BD92
:1091E00010B5002100200022214B5B6803F00C0128
:1091F00021B1042906D0082928D107E0214B224CAF
:10920000236027E01F4B204C236023E0184B5B6852
:1092100003F47010164B5B6803F48032022303EBF7
:10922000904022B9194B4343174C23600DE0104B7B
:109230005B6803F4003323B1144B4343124C2360A7
:1092400003E0104B4343104C236003E00D4B0E4CE6
:10925000236000BF00BF064B5B68C3F303130C4CD5
:10926000E15C094B1B68CB40074C236010BD00003C
:1092700000100240002002400000FFF8FFFFF6FE51
:1092800008ED00E000127A002800002000093D00EF
:109290002C00002031490143314A1160704770B5FC
:1092A000002100230F22C47804B32D4C246804F459
:1092B000E064C4F5E064210AC1F10403CA404478C3
:1092C00004FA03F18478144021430901254C0678FF
:1092D000A155047804F01F050124AC4005786D11F8
:1092E000AD0005F1E025C5F8004109E0047804F07F
:1092F0001F050124AC401C4D0678761145F8264028
:1093000070BD1A4A0A400243154B1B1F1A60704772
:1093100039B1134A121D12680243114B1B1D1A600A
:1093200006E00F4A121D126882430D4B1B1D1A6086
:109330007047042808D14FF0E021096941F0040189
:109340004FF0E022116107E04FF0E021096921F0C0
:1093500004014FF0E0221161704700000000FA059F
:109360000CED00E000E400E080E100E080FFFF1F82
:1093700010B50446FA48844208D10121401500F096
:1093800003FE0021601500F0FFFD17E0F548844260
:1093900008D10121001500F0F7FD0021201500F093
:1093A000F3FD0BE0F048844208D10121C80300F02E
:1093B000EBFD00214FF4004000F0E6FD10BD30B59C
:1093C0000246002000235068E84C20400D790C68CC
:1093D00044EA0524204350609068E54C2040D1E9E0
:1093E00002542C434D7944EA450420439060D06AEE
:1093F00020F470000C7C641EE4B2234340EA035066
:10940000D06230BD00210160017141718160C16095
:1094100001210174704721B1826842F0010282602B
:1094200003E0826822F001028260704721B1826805
:1094300042F48072826003E0826822F4807282606B
:10944000704710B50023CBB21AB144681C43446086
:1094500002E044689C43446010BD816841F008010B
:1094600081607047014600208A6802F008020AB154
:10947000012000E000207047816841F00401816014
:109480007047014600208A6802F004020AB10120F8
:1094900000E00020704721B1826842F4A00282609F
:1094A00003E0826822F4A002826070470146002037
:1094B0008A6802F480020AB1012000E000207047AF
:1094C00010B50A4600210023416821F46041531E73
:1094D00041EA4331416010BD21B1426842F400626B
:1094E000426003E0426822F4006242607047F0B5D7
:1094F00004460D4600200021092D11DDE068A5F18C
:109500000A0606EB4607072606FA07F18843A5F187
:109510000A0606EB460603FA06F10843E0600CE093
:10952000206905EB4507072606FA07F1884305EB96
:10953000450603FA06F108432061072A0FDA606B3B
:10954000561E06EB86071F2606FA07F18843561EAD
:1095500006EB860605FA06F10843606322E00D2A51
:109560000FDA206BD61F06EB86071F2606FA07F1D7
:109570008843D61F06EB860605FA06F108432063EA
:1095800010E0E06AA2F10D0606EB86071F2606FA38
:1095900007F18843A2F10D0606EB860605FA06F1EF
:1095A0000843E062F0BD21B1826842F4801282601B
:1095B00003E0826822F48012826070470146C86C22
:1095C00080B2704766484C300068704721B14268ED
:1095D00042F48062426003E0426822F480624260AA
:1095E000704721B1426842F48052426003E0426811
:1095F00022F48052426070470A460021816821F4BB
:10960000E04111438160704721B1826842F4004219
:10961000826003E0826822F400428260704721B1D8
:10962000826842F40212826003E0826822F402122D
:1096300082607047014600208A6802F400120AB175
:10964000012000E000207047F0B5044615460020D8
:1096500000220026092911DDE068A1F10A0707EBC5
:10966000470C072707FA0CF29043A1F10A0707EB12
:10967000470703FA07F21043E0600CE0206901EBB2
:10968000410C072707FA0CF2904301EB410703FA5C
:1096900007F210432061A06BC0F30156EF1C06F1E6
:1096A000010CA7EB0C0707EB870C1F2707FA0CF23E
:1096B0009043EF1C06F1010CA7EB0C0707EB8707A3
:1096C00001FA07F21043A063F0BD10B50A4600216D
:1096D0000023816B21F44011531E41EA0351816341
:1096E00010BD08B5002300930090009B0B4400932D
:1096F000009B1A6008BD08B5024600200090009249
:1097000001F12800009B184400900098006880B286
:1097100008BD0A4600214168164B194011434160BB
:1097200070474162826270470A460021416821F019
:109730001F0111434160704740B109490831096870
:1097400041F40001064A0832116007E0044908317B
:10975000096821F40001024A0832116070470000D4
:109760000024014000280140003C0140FFFEF0FFC2
:10977000FDF7F1FFFFFD3FFF0246002013680B409D
:109780000BB1012000E000207047CA43026070471F
:1097900070B502460020002300240B125568CEB29B
:1097A00005EA060415681D4015B10CB1012000E062
:1097B000002070BD00220A12D343036070470000EE
:1097C000002044490860091D0860091D0860091D42
:1097D000086041483F4914310860704700213D4905
:1097E0008279002A3AD00A46126803689A430B46E7
:1097F0001A600A1D126803689A430B1D1A600279E9
:1098000011440A6803681A430A60324A083212682F
:1098100003689A432F4B08331A601A1D12680368B5
:109820009A432C4B0C331A604279102A0ED11A1F1E
:10983000126803681A43274B08331A601A1D12680E
:1098400003681A43234B0C331A600DE02149427917
:1098500011440A6803681A430A6005E0027911445A
:109860000A6803689A430A60704700210160017129
:109870000C2141710021817170471649103109682E
:109880000143144A10321160704701460020114A0A
:10989000143212680A400AB1012000E0002070472B
:1098A0000C49143108607047014600200022094B22
:1098B0001B6803EA0102074B14331B680B4013B10A
:1098C0000AB1012000E0002070470249143108600D
:1098D0007047000000040140FFFF0F0010B5044670
:1098E000CC48844208D10121042000F04DFB002126
:1098F000042000F049FB46E0C748844208D101211A
:10990000082000F041FB0021082000F03DFB3AE078
:10991000C248844208D10121102000F035FB00210B
:10992000102000F031FB2EE0BD48844208D1012117
:10993000202000F029FB0021202000F025FB22E060
:10994000B848844208D10121402000F01DFB0021CD
:10995000402000F019FB16E0B348844208D10121F1
:10996000802000F011FB0021802000F00DFB0AE0B8
:10997000AE48844207D10121801500F005FB00218B
:10998000A01500F001FB10BD10B50121084600F044
:10999000FBFA0021012000F0F7FA10BD2DE9F0419B
:1099A000024600250026002000230024002791F80D
:1099B00003C00CF00F0591F803C00CF0100CBCF1C3
:1099C000000F03D091F802C04CEA050591F800C0E1
:1099D000BCF1000F31D0146800202BE04FF0010CD7
:1099E0000CFA00F3B1F800C00CEA03069E4220D145
:1099F00083004FF00F0C0CFA03F7BC4305FA03FC8D
:109A00004CEA040491F803C0BCF1280F06D14FF0D2
:109A1000010C0CFA00FCC2F814C00AE091F803C073
:109A2000BCF1480F05D14FF0010C0CFA00FCC2F854
:109A300010C0401C0828D1D31460B1F800C0BCF19C
:109A4000FF0F34DD546800202EE000F1080C4FF0C9
:109A5000010808FA0CF3B1F800C00CEA03069E42B4
:109A600021D183004FF00F0C0CFA03F7BC4305FA29
:109A700003FC4CEA040491F803C0BCF1280F05D1A3
:109A800000F1080C08FA0CF8C2F8148091F803C031
:109A9000BCF1480F07D100F1080C4FF0010808FA9B
:109AA0000CF8C2F81080401C0828CED35460BDE8E2
:109AB000F0814FF6FF710180022181700421C17095
:109AC00070470246002093680B400BB1012000E074
:109AD000002070470146886880B270470246002027
:109AE000D3680B400BB1012000E000207047014615
:109AF000C86880B2704701617047416170470AB120
:109B0000016100E041617047C16070474FF48032ED
:109B10000A4382618161826182698269704702467B
:109B20000020434B18684FF68073184040EA02103B
:109B300008433F4B186070473E49C8617047F0B515
:109B40000A46002300240021002500F00046B6F15B
:109B5000004F02D1364EF16901E0354E7168C0F315
:109B6000034583B200F44016B6F5401F08D121F03A
:109B700070612F4E766826F070662D4F7E6012E081
:109B800000F48016B6F5801F06D1032606FA05F408
:109B9000A14341F0706106E0460D360103FA06F676
:109BA000B14341F0706122B1460D360103FA06F669
:109BB000314300F00046B6F1004F02D11C4EF16176
:109BC00001E01B4E7160F0BD30B500228B071C0F09
:109BD0000F2303FA04F2164B08338C1053F8243089
:109BE0009343134C08348D1044F8253023468C10D1
:109BF00053F824308C07240F00FA04F423430C4C50
:109C000008348D1044F8253030BD0A49DC31086035
:109C10007047000000080140000C014000100140A6
:109C20000014014000180140001C014000200140C8
:109C300000000140000020420E49086070470D49B5
:109C4000486070470B49886070474AF6AA20094966
:109C5000086070474CF6CC400649086070470146E2
:109C60000020044AD2680A400AB1012000E0002026
:109C70007047000000300040DF48006840F00100FD
:109C8000DD49086008464068DC490840DA49486018
:109C900008460068DA490840D74908600846006865
:109CA00020F4802008600846406820F4FE004860E8
:109CB0004FF41F0088607047CF49096821F4803154
:109CC000CD4A11601146096821F480211160B0F578
:109CD000803F03D0B0F5802F0ED106E0C649096859
:109CE00041F48031C44A116007E0C349096841F476
:109CF000A021C14A116000E000BF00BF704710B54D
:109D000001460022002300204A11012A02D1BA4C48
:109D1000236806E0022A02D1B74C236A01E0B64C60
:109D2000636A01F01F02012494401C400CB1012021
:109D300000E0002010BD38B5002000900024002570
:109D400000BF3120FFF7DBFF05460098401C009064
:109D50000098B0F5A06F01D0002DF2D03120FFF7B0
:109D6000CEFF08B1012400E00024204638BD0146A2
:109D70000020A14A106820F0F80040EAC1001060FD
:109D80007047A04908607047024600209A4B586807
:109D900020F47C1042EA01031843974B5860704747
:109DA00098490866704701460020934A506820F0A1
:109DB00003000843506070478F48406800F00C0073
:109DC0007047014600208C4A506820F0F00008439C
:109DD0005060704701460020874A506820F4E060D8
:109DE00008435060704701460020834A506820F4C1
:109DF000605040EAC1005060704729B17E4A527AF3
:109E000002437D4B5A7204E07B4A527A82437A4B7A
:109E10005A7270477B49D83108607047014600206C
:109E2000754A506820F44040084350607047002154
:109E3000714A20321170704A82F82010012802D035
:109E400004280AD104E001216B4A2032117005E098
:109E50000521694A2032117000E000BF00BF704741
:109E60006949086070476449096A0143624A11629E
:109E70007047654944390860704730B500210022B9
:109E8000002400235C4D6D6805F00C0121B104290C
:109E900005D0082923D105E05C4D056022E05B4D2B
:109EA00005601FE0544D6D6805F47012524D6D68E9
:109EB00005F48034022505EB92421CB9544D5543FC
:109EC00005600BE04C4D6D6805F400351DB1504D3B
:109ED0005543056002E04D4D5543056002E04B4D92
:109EE000056000BF00BF444D6D6805F0F001090931
:109EF000484D6B5C0568DD4045603F4D6D6805F47D
:109F0000E061090A434D6B5C4568DD4085603A4D70
:109F10006D6805F46051C90A3E4D6B5C4568DD40D3
:109F2000C560354D6D6805F44041890B3A4D6B5C59
:109F3000C568B5FBF3F5056130BD29B12E4A5269FC
:109F400002432D4B5A6104E02B4A526982432A4B4B
:109F50005A61704729B1284A92690243264B9A6197
:109F600004E0254A92698243234B9A61704729B1E4
:109F7000214AD2690243204BDA6104E01E4AD269C9
:109F800082431D4BDA61704729B11B4AD2680243F4
:109F9000194BDA6004E0184AD2688243164BDA6043
:109FA000704729B1144A12690243134B1A6104E045
:109FB000114A12698243104B1A61704712494039A5
:109FC000086070470F49C86470470B49C8717047F3
:109FD0000948406A40F0807007494862704701466E
:109FE0000020054A92680A400AB1012000E00020E2
:109FF0007047014988727047001002400000FFF866
:10A00000FFFFF6FE000042428004424200127A0046
:10A0100000093D003C0000204C00002010B5044623
:10A02000BE48844208D101218014FFF7ADFF002112
:10A03000A014FFF7A9FF16E0B948844208D1012116
:10A040000014FFF7AEFF00212014FFF7AAFF0AE07B
:10A05000B448844207D10121C013FFF7A2FF0021B9
:10A06000E013FFF79EFF10BD10B50022028802F436
:10A0700041520B884C8823438C882343CC8823434C
:10A080000C8923434C8923438C892343CC89234364
:10A090001A430280838B4FF2FF74234083830B8A21
:10A0A000038210BD2DE9F04F85B005460C464FF0F8
:10A0B000000902274FF000084FF0010B0026B246BE
:10A0C000A88B4FF240010840A88302202884B5F8ED
:10A0D0001C90A068022801D100BF38E0A08810B908
:10A0E0004FF0010B01E04FF0020B8D48854200D18B
:10A0F00000E000BF6846FFF7C0FEDDF800A0E08882
:10A10000B0F5007F0AD14FEA1A2000EB8000400032
:10A11000A168B0FBF1F0401D86B20BE04FEA4B1096
:10A12000BAFBF0F000EB80004000A168B0FBF1F05A
:10A13000401D86B20A20B6FBF0F606F00108A6EB39
:10A140000800C0F34F074FF6FF7000EA0828022FFF
:10A1500001DBFF2F02DD02274FF00008E08840EA14
:10A16000080038432884A088A189084361880843EF
:10A170002188084340F4006040EA0909A5F81C90D2
:10A1800005B0BDE8F08F0021018041808180C18051
:10A19000018141818181C1810721018270470021B4
:10A1A000018041808180C180022181600021818104
:10A1B000704721B1028842F04002028004E0028828
:10A1C0004FF6BF731A400280704721B1828B42F470
:10A1D0008062828304E0828B4FF6FF331A408283D1
:10A1E000704730B5002400230C110125A540ABB207
:10A1F0001AB185881D43858002E085889D4385804E
:10A2000030BD1AB183880B43838002E083888B437F
:10A2100083807047818170470146888970474FF677
:10A22000FF62914204D0028842F48072028004E00E
:10A2300002884FF6FF631A400280704721B182887E
:10A2400042F00402828004E082884FF6FB731A40D9
:10A250008280704702884FF2FF731A4002800288A2
:10A260000A4302807047018841F4805101807047A1
:10A2700021B1028842F40052028004E002884DF6C7
:10A28000FF731A400280704702460020012901D066
:10A29000108B00E0908A70470146088A7047B1F53C
:10A2A000804F04D1028842F48042028004E0028898
:10A2B0004BF6FF731A400280704702460020138954
:10A2C0000B400BB1012000E000207047CA4302811F
:10A2D0007047F0B50246002000240023002501F05D
:10A2E0000F070126BE40B4B20B1101269E40B3B247
:10A2F000968806EA03051689264016B10DB101209D
:10A3000000E00020F0BD10B5002201F00F04012391
:10A31000A3409AB2D343038110BD00000030014036
:10A3200000380040003C004010B50446FE4884421E
:10A3300008D10121C014FFF727FE0021E014FFF728
:10A3400023FEC4E0B4F1804F08D101210846FFF795
:10A3500028FE00210120FFF724FEB8E0F3488442E4
:10A3600008D101210220FFF71CFE00210220FFF787
:10A3700018FEACE0EE48844208D101210420FFF72A
:10A3800010FE00210420FFF70CFEA0E0E948844203
:10A3900008D101210820FFF704FE00210820FFF763
:10A3A00000FE94E0E448844208D101211020FFF728
:10A3B000F8FD00211020FFF7F4FD88E0DF4884421B
:10A3C00008D101212020FFF7ECFD00212020FFF71C
:10A3D000E8FD7CE0DA48844208D101214014FFF70F
:10A3E000D3FD00216014FFF7CFFD70E0D548844213
:10A3F00009D10121C804FFF7C7FD00214FF4002057
:10A40000FFF7C2FD63E0D048844209D1012108056D
:10A41000FFF7BAFD00214FF48010FFF7B5FD56E0BD
:10A42000CA48844209D101214805FFF7ADFD00214A
:10A430004FF40010FFF7A8FD49E0C548844208D159
:10A4400001214020FFF7ADFD00214020FFF7A9FDCD
:10A450003DE0C048844208D101218020FFF7A1FDE2
:10A4600000218020FFF79DFD31E0BB48844208D1E8
:10A4700001218015FFF795FD0021A015FFF791FD43
:10A4800025E0B648844209D101210804FFF77CFD8C
:10A4900000214FF48030FFF777FD18E0B048844288
:10A4A00009D101214804FFF76FFD00214FF400306E
:10A4B000FFF76AFD0BE0AB48844208D10121880414
:10A4C000FFF762FD00214FF48020FFF75DFD10BD16
:10A4D00000220288944B98420ED0994B98420BD0A0
:10A4E000B0F1804F08D0914B984205D0904B9842E4
:10A4F00002D0904B984204D14FF68F731A404B888C
:10A500001A438D4B984207D08C4B984204D04FF69B
:10A51000FF431A40CB881A4302808B8883850B88BF
:10A520000385814B98420BD0854B984208D08B4BCA
:10A53000984205D08A4B984202D08A4B984201D16A
:10A540000B7A038601238382704770B500240022B2
:10A550000023058C4FF6FE7635400584028C8388F7
:10A56000048B4FF68F752C40B51E2C400D882C4364
:10A57000751E2A400D892A434D882A436A4DA842F8
:10A580000BD06F4DA84208D0744DA84205D0744D31
:10A59000A84202D0734DA84213D14FF6F7752A4056
:10A5A0004D892A434FF6FB752A408D882A434FF682
:10A5B000FF652B404FF6FF552B408D892B43CD89EE
:10A5C0002B4383800483CD888586028470BD70B55B
:10A5D000002400220023058C4FF6EF7635400584D9
:10A5E000028C8388048B48F6FF752C404FF6FF459C
:10A5F0002C400D884FF6FF7606EA05252C434FF6D2
:10A60000DF752A400D8906EA05152A434D8806EABA
:10A6100005152A43444DA84202D0494DA8421DD1F8
:10A620004FF67F752A404D894FF6FF7606EA0515ED
:10A630002A434FF6BF752A408D8806EA05152A433E
:10A640004FF6FF352B404FF2FF752B408D8906EA00
:10A6500085052B43CD8906EA85052B43838004833A
:10A66000CD880587028470BD70B5002400220023C8
:10A67000058C4FF6FF6635400584028C8388848BF9
:10A680004FF68F752C404FF6FC752C400D882C43EF
:10A690004FF6FF552A400D894FF6FF7606EA05254D
:10A6A0002A434D8806EA05252A431F4DA84202D0B9
:10A6B000234DA8421DD14FF2FF752A404D894FF618
:10A6C000FF7606EA05252A434FF6FF352A408D8896
:10A6D00006EA05252A434EF6FF752B404DF6FF7519
:10A6E0002B408D8906EA05152B43CD8906EA051511
:10A6F0002B4383808483CD888587028470BD70B5A9
:10A70000002200230024058C4EF6FF763540058498
:10A71000038C8488828B48F6FF752A404FF6FF45EC
:10A720002A400D8820E00000002C01400004004079
:10A7300000080040000C00400010004000140040E1
:10A7400000340140004C01400050014000540140E1
:10A7500000180040001C0040002000400040014064
:10A7600000440140004801404FF6FF7606EA052507
:10A770002A434DF6FF752B400D8906EA05352B431C
:10A780004D8806EA05352B43FA4DA84202D0FA4D12
:10A79000A84208D14BF6FF752C408D894FF6FF7605
:10A7A00006EA85152C4384808283CD88A0F840502A
:10A7B000038470BD828B4FF2FF331A408283828BF9
:10A7C0004FF6FF7303EA01231A4382837047F0B503
:10A7D0000C461546002200210026078C4EF6FF7C11
:10A7E00007EA0C070784828B018C4FF6FF7707EA94
:10A7F000043640F6FF473A404FF6FF7707EA052751
:10A800003A434FF6FF7707EA03373A43D94FB84246
:10A810000ED0D94FB8420BD0B0F1804F08D0D74FEF
:10A82000B84205D0D64FB84202D0D64FB84206D172
:10A830004DF6FF77394046F48057394305E047F637
:10A84000FF57394044F48057394382830184F0BD77
:10A85000828B4FF6F3731A408283828B0A43828382
:10A860007047F0B50C461546002200210026078CE3
:10A870004FF6FF6C07EA0C070784828B018C4FF6BA
:10A88000FF7707EA04264FF60C773A404FF6FF773A
:10A8900007EA03172F433A43B64FB8420ED0B64FDC
:10A8A000B8420BD0B0F1804F08D0B44FB84205D0B9
:10A8B000B34FB84202D0B34FB84206D14FF6FF575C
:10A8C000394046F48077394305E04FF2FF5739406D
:10A8D00044F48077394382830184F0BD028B4FF2C8
:10A8E000FF331A400283028B4FF6FF7303EA012302
:10A8F0001A4302837047F0B50C461546002200212A
:10A900000026078C4FF6EF7C07EA0C070784028BC2
:10A91000018C4FF6FF7707EA041640F6FF473A40EE
:10A920004FF6FF7707EA03373A434FF6FF7707EA18
:10A9300005273A438F4FB8420ED08F4FB8420BD005
:10A94000B0F1804F08D08D4FB84205D08C4FB8423F
:10A9500002D08C4FB84206D14FF6DF77394046F02F
:10A960001007394305E04FF65F77394044F0100790
:10A97000394302830184F0BD028B4FF6F3731A4012
:10A980000283028B0A4302837047F0B50C461546DA
:10A9900000220021068C4FF6FE773E400684028B93
:10A9A000018C4FF60C7632407E1C06EA03162E43CD
:10A9B0003243704EB0420ED06F4EB0420BD0B0F169
:10A9C000804F08D06D4EB04205D06D4EB04202D0DF
:10A9D0006C4EB04206D14FF6FD76314044F0010690
:10A9E000314305E04FF6F576314044F0010631433E
:10A9F00002830184F0BD70B505460C465D48854272
:10AA00000ED05D4885420BD0B5F1804F08D05B4831
:10AA1000854205D05A48854202D05A48854200D125
:10AA200000E000BF208850B92389A28861882846A9
:10AA3000FFF7ABFFE1882846FFF79EFF25E020885F
:10AA400004280AD12389A28861882846FFF753FF8A
:10AA5000E1882846FFF742FF17E0208808280AD13E
:10AA60002389A28861882846FFF7FBFEE1882846F3
:10AA7000FFF7EEFE09E02389A28861882846FFF7E8
:10AA8000A6FEE1882846FFF795FE70BD2DE9F0414E
:10AA900005460C4600260127608808B9022600E01A
:10AAA0000026A088012801D1022700E00127208884
:10AAB000A0B92389A28861882846FFF766FFE1884C
:10AAC0002846FFF759FF23893A4631462846FFF7C3
:10AAD00012FFE1882846FFF701FF13E02389A288CF
:10AAE00061882846FFF707FFE1882846FFF7F6FE52
:10AAF00023893A4631462846FFF747FFE188284632
:10AB0000FFF73AFFBDE8F0810A884B881A438B882B
:10AB10001A43CB881A430B891A434B891A438B89F2
:10AB20001A43A0F8442070474FF6FF71818000213E
:10AB30000180C18041800172704700210180418005
:10AB40008180C180018141818181C1817047002163
:10AB500001804180012181800021C18001817047F5
:10AB60000021018041808180C180018141818181FA
:10AB700070470000002C01400034014000040040F8
:10AB800000080040000C004021B1028842F00102A0
:10AB9000028004E002884FF6FE731A40028070477C
:10ABA00031B1B0F8442042F40042A0F8442005E05E
:10ABB000B0F84420C2F30E02A0F8442070471AB146
:10ABC00083890B43838102E083898B4383817047B0
:10ABD0008182704741EA0203A0F8483070471AB1F9
:10ABE00083890B43838102E083898B438381704790
:10ABF00001894FF6F8721140018170470A46002121
:10AC000001894FF68F73194011430181704730B5A8
:10AC100004460D4629462046FFF7F0FF208940F004
:10AC20000700208130BD2DE9F04104460D4616464F
:10AC30001F46602D06D13B46012231462046FFF7D4
:10AC40005AFE05E03B46012231462046FFF79DFEB5
:10AC500029462046FFF7D2FF208940F007002081D7
:10AC6000BDE8F08130B50C4600210189C9B24FF62C
:10AC7000FF7505EA0325154325432943018130BDAE
:10AC80002DE9F04105460E461746984600244346F6
:10AC90003A4631462846FFF7E5FF2C894FF6F87013
:10ACA000044044F007044FF68F70044044F07004F1
:10ACB0002C81BDE8F081F0B504460D4616461F46CE
:10ACC0003B46324629462046FFF7CCFF208940F418
:10ACD00080402081F0BD0185828270470A460021B4
:10ACE00001884FF68F731940114301807047F0B50A
:10ACF0000C4615461E460021002200230189028BC6
:10AD0000038C4FF6F877394021434FF6FC473A4021
:10AD100040F201173A434FF6DD773B404FF6FF779D
:10AD200007EA06172F433B43018102830384F0BDEA
:10AD30000A460021018B4FF68F731940114301839E
:10AD400070470A460021018B48F6FF7319404FF601
:10AD5000FF7303EA02231943018370470A46002167
:10AD6000818B4FF68F7319401143818370470A46D8
:10AD70000021818B48F6FF7319404FF6FF7303EAF9
:10AD8000022319438183704721B1028842F0800277
:10AD9000028004E002884FF67F731A4002807047F9
:10ADA00021B1828842F00402828004E082884FF65A
:10ADB000FB731A408280704721B1828842F00802FA
:10ADC000828004E082884FF6F7731A4082807047D1
:10ADD00021B1828842F00102828004E082884FF62D
:10ADE000FE731A40828070470A460021018B4FF69D
:10ADF000F77319401143018370470A460021018B04
:10AE00004FF2FF7319404FF6FF7303EA0223194311
:10AE1000018370470A460021818B4FF6F773194072
:10AE20001143818370470A460021818B4FF2FF73E3
:10AE300019404FF6FF7303EA0223194381837047D9
:10AE40000A460021018B4FF6FB7319401143018321
:10AE500070470A460021018B4FF6FF3319404FF629
:10AE6000FF7303EA02231943018370470A46002156
:10AE7000818B4FF6FB7319401143818370470A465B
:10AE80000021818B4FF6FF3319404FF6FF7303EA21
:10AE900002231943818370470A460021018B4FF634
:10AEA0007F7319401143018370470A460021018BCB
:10AEB000C1F30E014FF6FF7303EA02231943018326
:10AEC00070470A460021818B4FF67F73194011436A
:10AED000818370470A460021818BC1F30E014FF632
:10AEE000FF7303EA02231943818370470A46002156
:10AEF000018C4FF6FD7319401143018470470A46D7
:10AF00000021018C4FF6F7731940114301847047FB
:10AF10000A460021018C4FF6DF7319404FF6FF738C
:10AF200003EA02131943018470470A460021018C89
:10AF30004FF67F7319404FF6FF7303EA021319436C
:10AF4000018470470A460021018C4FF6FF531940D7
:10AF50004FF6FF7303EA02231943018470470A4640
:10AF60000021018C4FF2FF7319404FF6FF7303EA83
:10AF700002231943018470470A460021018C4DF6D3
:10AF8000FF7319404FF6FF7303EA0233194301843C
:10AF9000704730B5002301248C40A3B2048C9C433D
:10AFA0000484048C02FA01F5ADB22C43048430BD54
:10AFB00030B5002304248C40A3B2048C9C43048449
:10AFC000048C02FA01F5ADB22C43048430BD70B597
:10AFD0000346002000241846183001258D40ACB2ED
:10AFE0001D8CA5431D8409B1082909D100EB61001E
:10AFF000056825F0700505600568154305600EE0DD
:10B000000D1FC5F34E052844056825F4E04505608D
:10B0100005684FF6FF7606EA02263543056070BDE7
:10B0200021B1028842F00202028004E002884FF659
:10B03000FD731A400280704721B1028842F0040279
:10B04000028004E002884FF6FB731A4002807047CA
:10B0500021B1828842F08002828004E082884FF62B
:10B060007F731A408280704702884FF6F7731A4048
:10B07000028002880A430280704782884FF68F73ED
:10B080001A40828082880A438280704702894FF684
:10B09000F8731A40028102890A43028170470289CB
:10B0A0004FF67F731A40028102890A43028170477A
:10B0B000818470478185704781867047018770471A
:10B0C00081877047A0F84010704702884FF6FF4311
:10B0D0001A40028002880A43028070470146888E27
:10B0E00070470146088F70470146888F70470146B8
:10B0F000B1F8400070470146888C70470146088DC2
:10B10000704702460020138A0B400BB1012000E07B
:10B1100000207047CA430282704730B502460020C3
:10B1200000230024158A05EA0103958905EA010434
:10B1300013B10CB1012000E0002030BDCA430282EF
:10B140007047000010B50446FB48844209D1012134
:10B150008803FEF719FF00214FF48040FEF714FF2B
:10B1600032E0F648844209D101214804FEF719FF74
:10B1700000214FF40030FEF714FF25E0F048844230
:10B1800009D101218804FEF70CFF00214FF4802033
:10B19000FEF707FF18E0EB48844209D10121C804FB
:10B1A000FEF7FFFE00214FF40020FEF7FAFE0BE051
:10B1B000E548844208D101210805FEF7F2FE00218E
:10B1C0004FF48010FEF7EDFE10BD2DE9F04786B07C
:10B1D00005460E460024A24600BFA1460027B089BE
:10B1E00000B100BF2F462C8A4CF6FF700440F08857
:10B1F00004432C82AC894EF6F3100440B0883189A8
:10B200000843718908430443AC81AC8A4FF6FF4080
:10B210000440B0890443AC8201A8FEF72EFEC64864
:10B22000874202D1DDF810A001E0DDF80CA0A8896A
:10B2300000F4004040B10AEBCA0000EB0A1031688C
:10B240004900B0FBF1F807E00AEBCA0000EB0A1076
:10B2500031688900B0FBF1F86420B8FBF0F004011C
:10B260002009642101FB1089A88900F4004040B145
:10B27000322000EBC900B0FBF1F000F007000443FE
:10B2800008E0322000EB09106421B0FBF1F000F07F
:10B290000F0004432C8106B0BDE8F0874FF416512F
:10B2A000016000218180C18001810C214181002148
:10B2B0008181704710B502460020108A4FF2FF03CB
:10B2C00018400B884C8823438C882343CC88234325
:10B2D0001843108210BD0021018041808180C1800F
:10B2E000704721B1828942F40052828104E0828950
:10B2F0004DF6FF731A4082817047F0B50346002473
:10B3000000260025002040F66A17B94200D100BF90
:10B310001846C1F3421401F01F06012707FA06F58B
:10B32000012C01D10C3004E0022C01D1103000E0DE
:10B3300014301AB107682F43076002E00768AF4373
:10B340000760F0BD1AB1838A0B43838202E0838ACF
:10B350008B4383827047028A4FF6F0731A40028251
:10B36000028A0A430282704782894FF2FF731A40B1
:10B37000828182890A438281704721B1828942F0A9
:10B380000202828104E082894FF6FD731A408281B5
:10B390007047028A4FF6DF731A400282028A0A431C
:10B3A0000282704721B1028A42F48042028204E0A4
:10B3B000028A4BF6FF731A4002827047C1F30802FB
:10B3C0008280704701468888C0F3080070478189F1
:10B3D00041F0010181817047028BD2B20283028B5E
:10B3E00042EA012202837047028B02F47F42028309
:10B3F000028B0A430283704721B1828A42F0200205
:10B40000828204E0828A4FF6DF731A40828270479C
:10B4100021B1828A42F01002828204E0828A4FF6D1
:10B42000EF731A408282704721B1828A42F008028B
:10B43000828204E0828A4FF6F7731A408282704754
:10B4400021B1828942F40042828103E08289C2F301
:10B450000E028281704721B1828A42F400628282A8
:10B4600004E0828A4FF2FF731A4082827047828A18
:10B470004FF6FB731A408282828A0A4382827047A7
:10B4800021B1828A42F00202828204E0828A4FF66F
:10B49000FD731A408282704702460020B1F5007F9A
:10B4A00000D100BF13880B400BB1012000E0002049
:10B4B000704701F40072B2F5007F00D100BFCA43AB
:10B4C0000280704770B5024600240023002500204A
:10B4D00040F66A16B14200D100BFC1F3421501F037
:10B4E0001F03012606FA03F3012D02D1968933408A
:10B4F00006E0022D02D1168A334001E0968A3340DD
:10B500000C12012606FA04F41688344013B10CB16B
:10B51000012000E0002070BD10B50022002340F69D
:10B520006A14A14200D100BF0A1201249440A3B2C0
:10B53000DC43048010BD000000380140004400409E
:10B5400000480040004C004000500040094880473F
:10B5500009480047FEE7FEE7FEE7FEE7FEE7FEE7F5
:10B56000FEE7FEE7FEE7FEE704480549054A064B0D
:10B5700070470000939100083181000820B8002036
:10B5800020CA002020BA002020BA002008B5FE48BA
:10B59000C07B002817DC01214020FEF7DBFC4FF6C2
:10B5A000FF70ADF8000010208DF8030003208DF827
:10B5B00002006946F548FEF7F1F9BDF80010F348BE
:10B5C000FEF79BFA53E001214420FEF7C3FC49F645
:10B5D000FF70ADF8000010208DF8030003208DF8F7
:10B5E00002006946E948FEF7D9F9BDF80010E748BE
:10B5F000FEF783FA4FF44050ADF8000010208DF8AC
:10B60000030003208DF802006946E148FEF7C6F901
:10B61000BDF80010DE48FEF770FA01213020FEF779
:10B6200099FC40F69B70ADF8000010208DF80300E7
:10B6300003208DF802006946D648FEF7AFF9BDF841
:10B640000010D448FEF759FA4FF40050ADF800004E
:10B6500010208DF8030003208DF802006946CE48C3
:10B66000FEF79CF9BDF80010CB48FEF746FA08BD7E
:10B67000CA480088401CC949088008460088192823
:10B680001BDB00200880C648007818B90120C44997
:10B69000087002E00020C2490870C148007830B943
:10B6A000C048006820F40050BE49086005E0BD486D
:10B6B000006840F40050BB4908600020BA49087097
:10B6C000FEE3B9480078C0EBC00101EB0010B749B8
:10B6D00001EB400090F82D0048B9B34801780120F3
:10B6E0008840B04909680843AE49086016E2AE4890
:10B6F0000078C0EBC00101EB0010AC4901EB400049
:10B7000090F82800002859D1A7480078C0EBC00164
:10B7100001EB0010A54901EB400090F82D00012835
:10B720002CDBA1480078C0EBC00101EB00109F4961
:10B7300001EB400090F82D000B281FDC9A480078A0
:10B74000C0EBC00101EB0010984901EB400090F8FC
:10B75000260048B194480178012088409149096841
:10B76000814390480160D9E18F48017801208840E9
:10B770008C49096808438B490860CFE18A48007802
:10B78000C0EBC00101EB0010884901EB400090F8CC
:10B79000260048B184480178012088408149096821
:10B7A000084380490860B9E17F480178012088405A
:10B7B0007C49096881437B480160AFE17A480078A1
:10B7C000C0EBC00101EB0010784901EB400090F89C
:10B7D0002D000F280CD074480078C0EBC00101EB9D
:10B7E0000010724901EB400090F82D0019281ED17D
:10B7F0006F486D490978405C01280ED16A4801788C
:10B80000012088406749096881436648016000203B
:10B810006749654A1278885480E1634801780120BD
:10B8200088406049096808435E49086076E15E48DF
:10B830000078C0EBC00101EB00105C4901EB400057
:10B8400090F82D0001282DDB57480078C0EBC0018F
:10B8500001EB0010554901EB400090F82D000A283B
:10B8600020DC51480078C0EBC00101EB00104F49CB
:10B8700001EB4000D0F81E00002809DB4A4801789F
:10B88000012088404749096881434648016045E1F5
:10B8900045480178012088404249096808434149E8
:10B8A00008603BE140480078C0EBC00101EB0010AC
:10B8B0003E4901EB400090F82D00132822D13A4870
:10B8C0000078C0EBC00101EB0010384901EB4000EB
:10B8D000D0F81E0041F28831884209DB32480178F5
:10B8E000012088402F49096881432E48016015E1F5
:10B8F0002D480178012088402A49096808432949D0
:10B9000008600BE128480078C0EBC00101EB001093
:10B91000264901EB400090F82D000B2822D1224847
:10B920000078C0EBC00101EB0010204901EB4000A2
:10B93000D0F81E0040F6C411884209DB1A4801788D
:10B940000120884017490968814316480160E5E0F5
:10B9500015480178012088401249096808431149B7
:10B960000860DBE010480078C0EBC00101EB00107C
:10B970000E4901EB400090F82D000B2839D10A4800
:10B980000078C0EBC00115E05060002000180140B5
:10B990000008014000140140001001405E0000203A
:10B9A0005800002054000020600000205F6F00203D
:10B9B0001417002001EB0010FE4901EB4000D0F805
:10B9C0001E0040F6C411884209DBFB4801780120C3
:10B9D0008840FA4909688143F84801609EE0F648CA
:10B9E000017801208840F54909680843F349086057
:10B9F00094E0F1480078C0EBC00101EB0010ED4984
:10BA000001EB400090F82D000D2822D1EA48007883
:10BA1000C0EBC00101EB0010E64901EB4000D0F89B
:10BA20001E0042F21071884209DBE34801780120D0
:10BA30008840E24909688143E04801606EE0DE48E1
:10BA4000017801208840DD4909680843DB49086026
:10BA500064E0D9480078C0EBC00101EB0010D54983
:10BA600001EB400090F82D00102819D0D248007842
:10BA7000C0EBC00101EB0010CE4901EB400090F893
:10BA80002D0012280CD0CC480078C0EBC00101EB8F
:10BA90000010C84901EB400090F82D00112822D178
:10BAA000C5480078C0EBC00101EB0010C14901EBB3
:10BAB0004000D0F81E004CF25031884209DBBE48ED
:10BAC000017801208840BD4909688143BB48016075
:10BAD00024E0B948017801208840B8490968084342
:10BAE000B64908601AE0B648B349097830F8110041
:10BAF000B0F5006F09DDB048017801208840AF49FA
:10BB000009688143AD48016008E0AB480178012035
:10BB10008840AA4909680843A8490860A6480078EF
:10BB20000B30C0EBC00101EB0010A24901EB40005B
:10BB300090F82D0048B9A048017801208840A1491B
:10BB4000096808439F490860EFE19B4800780B3083
:10BB5000C0EBC00101EB0010964901EB400090F8EA
:10BB6000280090BB944800780B30C0EBC00101EB7B
:10BB70000010904901EB400090F82D0001282FDBC8
:10BB80008D4800780B30C0EBC00101EB00108949F3
:10BB900001EB400090F82D000B2821DC864800784E
:10BBA0000B30C0EBC00101EB0010824901EB4000FB
:10BBB00090F8260050B180480178012088408149E2
:10BBC000096881437F480160AFE12AE07A48017843
:10BBD000012088407B49096808437A490860A4E14C
:10BBE000754800780B30C0EBC00101EB00107149C3
:10BBF00001EB400090F8260048B16F480178012021
:10BC000088407049096808436E4908608DE16A48B8
:10BC10000178012088406B490968814369480160C7
:10BC200083E1654800780B30C0EBC00101EB0010E8
:10BC3000604901EB400090F82D000F280DD05E48C0
:10BC400000780B30C0EBC00101EB0010594901EB4B
:10BC5000400090F82D0019281CD159495648007809
:10BC60000B3031F81000B0F5006F09DA5248017856
:10BC7000012088405349096881435248016054E1DA
:10BC80004D480178012088404E49096808434D49D4
:10BC900008604AE1484800780B30C0EBC00101EB76
:10BCA0000010444901EB400090F82D0001282FDBE3
:10BCB000414800780B30C0EBC00101EB00103D495A
:10BCC00001EB400090F82D000A2821DC3A4800786A
:10BCD0000B30C0EBC00101EB0010364901EB400016
:10BCE000D0F81E00002809DB334801780120884085
:10BCF0003449096881433348016016E12E480178D0
:10BD0000012088402F49096808432E4908600CE14A
:10BD1000294800780B30C0EBC00101EB0010254929
:10BD200001EB400090F82D00132823D12248007821
:10BD30000B30C0EBC00101EB00101E4901EB4000CD
:10BD4000D0F81E0041F28831884209DB1A48017898
:10BD5000012088401B49096881431A480160E4E0DA
:10BD6000154801780120884016490968084315499B
:10BD70000860DAE0104800780B30C0EBC00101EB3E
:10BD800000100C4901EB400090F82D000B282ED13B
:10BD9000094800780B30C0EBC00101EB00100549E9
:10BDA00001EB4000D0F81E0040F6C411884214DBBD
:10BDB000014809E05F6F002060000020540000206F
:10BDC000D416002050000020017801208840F74957
:10BDD00009688143F5480160A7E0F5480178012032
:10BDE0008840F24909680843F04908609DE0F0483E
:10BDF00000780B30C0EBC00101EB0010ED4901EB06
:10BE0000400090F82D000D2823D1E94800780B3030
:10BE1000C0EBC00101EB0010E64901EB4000D0F897
:10BE20001E0042F21071884209DBE14801780120CE
:10BE30008840DE4909688143DC48016075E0DC48E0
:10BE4000017801208840D94909680843D74908602A
:10BE50006BE0D74800780B30C0EBC00101EB00105D
:10BE6000D44901EB400090F82D0010281BD0D04899
:10BE700000780B30C0EBC00101EB0010CD4901EBA5
:10BE8000400090F82D0012280DD0C94800780B30E2
:10BE9000C0EBC00101EB0010C64901EB400090F877
:10BEA0002D00112825D1C24800780B30C0EBC0010D
:10BEB00001EB0010BF4901EB4000D0F81E0000E08C
:10BEC00038E04CF25031884209DBB9480178012052
:10BED0008840B64909688143B448016025E0B44808
:10BEE000017801208840B14909680843AF490860DA
:10BEF0001BE0B149AE4800780B3031F81000B0F5C6
:10BF0000006F09DDAA48017801208840A749096827
:10BF10008143A648016008E0A548017801208840D7
:10BF2000A24909680843A1490860A1480078401C5B
:10BF30009F4908709E4800780B28FFF6C2AB162078
:10BF40009B49087028E29A480078C0EBC00101EBD9
:10BF50000010984901EB400090F82D0058B9944822
:10BF600000780838012101FA00F094490968084373
:10BF7000924908600BE28E480078C0EBC00101EBEB
:10BF800000108C4901EB400090F8280080BB8848E5
:10BF90000078C0EBC00101EB0010864901EB4000C6
:10BFA00090F82D00012830DB81480078C0EBC001FB
:10BFB00001EB00107F4901EB400090F82D000B28A9
:10BFC00023DC7B480078C0EBC00101EB001079490D
:10BFD00001EB400090F8260058B175480078083809
:10BFE0000121814075480068884374490860CEE1AA
:10BFF0002EE06F4800780838012101FA00F06F49FF
:10C00000096808436D490860C1E169480078C0EBE0
:10C01000C00101EB0010674901EB400090F82600D9
:10C0200058B1634800780838012101FA00F06349EB
:10C030000968084361490860A9E15D48007808384B
:10C04000012181405D48006888435C4908609EE1A9
:10C0500057480078C0EBC00101EB0010554901EBD7
:10C06000400090F82D000F280CD051480078C0EB0C
:10C07000C00101EB00104F4901EB400090F82D008A
:10C08000192821D14E484A490978405C01280FD12E
:10C0900047480078083801218140484800688843B3
:10C0A0004649086000204649414A127888546EE1AA
:10C0B0003F4800780838012101FA00F03F4909683B
:10C0C00008433E49086062E139480078C0EBC0018E
:10C0D00001EB0010374901EB400090F82D000128DA
:10C0E00030DB33480078C0EBC00101EB0010314970
:10C0F00001EB400090F82D000A2823DC2C48007842
:10C10000C0EBC00101EB00102A4901EB4000D0F860
:10C110001E0000280ADB26480078083801218140EB
:10C120002648006888432549086030E120480078A7
:10C130000838012101FA00F02049096808431F4925
:10C14000086024E11A480078C0EBC00101EB001040
:10C15000184901EB400090F82D00132832D1144803
:10C160000078C0EBC00101EB0010124901EB400068
:10C17000D0F81E0041F2883188420ADB0C48007872
:10C180000838012181400D48006888430B49086048
:10C19000FDE0074800780838012101FA00F007495E
:10C1A0000968084305490860F1E0000050000020DC
:10C1B000600000205F6F0020D41600205400002093
:10C1C00014170020F8480078C0EBC00101EB001004
:10C1D000F64901EB400090F82D000B2825D1F248DC
:10C1E0000078C0EBC00101EB0010F04901EB40000A
:10C1F000D0F81E0040F6C41188420ADBEA480078F5
:10C20000083801218140EA4800688843E84908600D
:10C21000BDE0E54800780838012101FA00F0E44962
:10C2200009680843E2490860B1E0DF480078C0EBE4
:10C23000C00101EB0010DD4901EB400090F82D003A
:10C240000B2825D1D8480078C0EBC00101EB0010C5
:10C25000D64901EB4000D0F81E0040F6C4118842D8
:10C260000ADBD1480078083801218140D0480068B5
:10C270008843CF4908608AE0CB480078083801211C
:10C2800001FA00F0CA4909680843C94908607EE01C
:10C29000C5480078C0EBC00101EB0010C34901EBB9
:10C2A000400090F82D000D2825D1BF480078C0EB44
:10C2B000C00101EB0010BD4901EB4000D0F81E00A9
:10C2C00042F2107188420ADBB74800780838012131
:10C2D0008140B74800688843B549086057E0B248D4
:10C2E00000780838012101FA00F0B14909680843D3
:10C2F000AF4908604BE0AC480078C0EBC00101EBEF
:10C300000010AA4901EB400090F82D00102819D028
:10C31000A5480078C0EBC00101EB0010A34901EB78
:10C32000400090F82D0012280CD09F480078C0EBF8
:10C33000C00101EB00109D4901EB400090F82D0079
:10C34000112824D198480078C0EBC00101EB0010FF
:10C35000964901EB4000D0F81E004CF25031884263
:10C360000ADB914800780838012181409048006834
:10C3700088438F4908600AE08B480078083801211B
:10C3800001FA00F08A49096808438949086086482B
:10C390000078401C84490870834800781B28FFF609
:10C3A000D2AD1B208049087025E27F480078C0EBA1
:10C3B000C00101EB00107D4901EB400090F82D0019
:10C3C00058B9794800780D38012101FA00F079490F
:10C3D000096808437749086008E273480078C0EBB1
:10C3E000C00101EB0010714901EB400090F82800FA
:10C3F00080BB6D480078C0EBC00101EB00106B49B9
:10C4000001EB400090F82D00012830DB66480078F1
:10C41000C0EBC00101EB0010644901EB400090F853
:10C420002D000B2823DC60480078C0EBC00101EB35
:10C4300000105E4901EB400090F8260058B15A48C0
:10C4400000780D38012181405A48006888435949D5
:10C450000860CBE12EE0544800780D38012101FA44
:10C4600000F054490968084352490860BEE14E484B
:10C470000078C0EBC00101EB00104C4901EB40001B
:10C4800090F8260058B1484800780D38012101FA8B
:10C4900000F048490968084346490860A6E1424857
:10C4A00000780D38012181404248006888434149A5
:10C4B00008609BE13C480078C0EBC00101EB001034
:10C4C0003A4901EB400090F82D000F280CD0364877
:10C4D0000078C0EBC00101EB0010344901EB4000D3
:10C4E00090F82D00192821D133482F490978405C54
:10C4F00001280FD12C4800780D38012181402D48AA
:10C50000006888432B49086000212B48264A12788E
:10C5100081546BE1244800780D38012101FA00F0C4
:10C52000244909680843234908605FE11E480078F0
:10C53000C0EBC00101EB00101C4901EB400090F87A
:10C540002D0001283ADB18480078C0EBC00101EB50
:10C550000010164901EB400090F82D000A282DDC50
:10C5600011480078C0EBC00101EB00100F4901EB4E
:10C570004000D0F81E0000280ADB0B4800780D3878
:10C58000012181400B48006888430A4908602DE179
:10C59000054800780D38012101FA00F005490968C5
:10C5A00008430449086021E1600000205F6F00201B
:10C5B000540000205000002014170020FC48007890
:10C5C000C0EBC00101EB0010FA4901EB400090F80C
:10C5D0002D00132825D1F6480078C0EBC00101EBEF
:10C5E0000010F44901EB4000D0F81E0041F2883100
:10C5F00088420ADBEE4800780D3801218140EE4880
:10C6000000688843EC490860F0E0E94800780D389C
:10C61000012101FA00F0E84909680843E649086089
:10C62000E4E0E3480078C0EBC00101EB0010E14911
:10C6300001EB400090F82D000B2825D1DC48007854
:10C64000C0EBC00101EB0010DA4901EB4000D0F86B
:10C650001E0040F6C41188420ADBD54800780D3828
:10C6600001218140D44800688843D3490860BDE077
:10C67000CF4800780D38012101FA00F0CE49096851
:10C680000843CD490860B1E0C9480078C0EBC0015B
:10C6900001EB0010C74901EB400090F82D000B287A
:10C6A00025D1C3480078C0EBC00101EB0010C1499F
:10C6B00001EB4000D0F81E0040F6C41188420ADBAE
:10C6C000BB4800780D3801218140BB480068884391
:10C6D000B94908608AE0B64800780D38012101FAAE
:10C6E00000F0B54909680843B34908607EE0B048E6
:10C6F0000078C0EBC00101EB0010AE4901EB400037
:10C7000090F82D000D2825D1A9480078C0EBC00174
:10C7100001EB0010A74901EB4000D0F81E0042F2E7
:10C72000107188420ADBA24800780D38012181404F
:10C73000A14800688843A049086057E09C480078F9
:10C740000D38012101FA00F09B49096808439A4914
:10C7500008604BE096480078C0EBC00101EB001088
:10C76000944901EB400090F82D00102819D0904812
:10C770000078C0EBC00101EB00108E4901EB4000D6
:10C7800090F82D0012280CD089480078C0EBC00129
:10C7900001EB0010874901EB400090F82D001128B3
:10C7A00024D183480078C0EBC00101EB001081491F
:10C7B00001EB4000D0F81E004CF2503188420ADBF9
:10C7C0007B4800780D38012181407B480068884310
:10C7D000794908600AE0764800780D38012101FAAD
:10C7E00000F075490968084373490860704800788B
:10C7F000401C6F4908706E4800782028FFF6D5ADC0
:10C800006E480078002804DD6C480078401E6B49B3
:10C8100008706B480078002804DD69480078401EE5
:10C820006749087065480078002806DD624800689E
:10C8300020F480506049086005E05F48006840F4DB
:10C8400080505D4908605E480078002806DD5A483F
:10C85000006820F400605849086005E05648006808
:10C8600040F400605449086056480078002804DD10
:10C8700054480078401E53490870534800780028F7
:10C8800004DD51480078401E4F4908704D4800783B
:10C89000002806DD4D48006820F400604B49086020
:10C8A00005E04A48006840F400604849086046488E
:10C8B0000078002806DD4548006820F48050434990
:10C8C000086005E04148006840F480503F49086036
:10C8D000704710B53E48007808B9012000E00020FC
:10C8E0003B4908700846007800287BD03948C07B57
:10C8F000002806DC3048008881B23748FDF704F98B
:10C900003EE201203549086000203549C1F8B001F8
:10C910002948007800F0010020B101202F493C395E
:10C92000086003E000202D493C3908602248007867
:10C9300000F0020020B1012028493839086003E0E6
:10C9400000202649383908601B48007800F00400B0
:10C9500020B1012021493439086003E000201F493B
:10C96000343908601448007800F0080020B1012034
:10C970001A493039086003E000201849303908604E
:10C980000D48007800F0100020B1012013492C3927
:10C99000086003E0002011492C390860064800783F
:10C9A00000F02000F8B101200C49283908601DE092
:10C9B000600000205F6F0020500000205B0000201E
:10C9C0005C000020590000205A0000205400002084
:10C9D000610000205060002000180140BC0123428B
:10C9E00000002142B3E00020E6490860E6480078F4
:10C9F00000F0400020B10120E249091D086003E079
:10CA00000020E049091D0860DF48007800F0800040
:10CA100020B10120DB490831086003E00020D9493A
:10CA200008310860D848008800F4807020B10120E7
:10CA3000D4490C31086003E00020D2490C31086071
:10CA4000D148008800F4007020B10120CD49103198
:10CA5000086003E00020CB4910310860CA48008814
:10CA600000F4806020B10120C6491431086003E061
:10CA70000020C44914310860C348008800F40060F5
:10CA800020B10120BF491831086003E00020BD49F2
:10CA900018310860BC48008800F4805020B10120A3
:10CAA000B8491C31086003E00020B6491C31086019
:10CAB000B548008800F4005018B10120B34908605F
:10CAC00002E00020B1490860AF48006800F480200F
:10CAD00018B10120AE49086002E00020AC490860AE
:10CAE000A948006800F4003020B10120A849091DC0
:10CAF000086003E00020A649091D0860A2480068FC
:10CB000000F4803020B10120A1490831086003E021
:10CB100000209F49083108609B48008800F40040CD
:10CB200020B101209A490C31086003E000209849A7
:10CB30000C3108609448008800F4804018B101204E
:10CB4000944908601CE100209249086018E192486D
:10CB5000C07B002806DC9148008881B29048FCF731
:10CB6000D3FF0DE1002087492831086001208D495D
:10CB7000C1F8B0018948007800F0010020B101201F
:10CB800080491439086003E000207E4914390860A8
:10CB90008248007800F0020020B101207949103964
:10CBA000086003E000207749103908607B4800786E
:10CBB00000F0040020B1012072490C39086003E044
:10CBC000002070490C3908607448007800F00800B3
:10CBD00020B101206B490839086003E00020694951
:10CBE000083908606D48007800F0100020B101207D
:10CBF0006449091F086003E000206249091F0860BA
:10CC00006648007800F0200018B101205D490860F6
:10CC100002E000205B4908606048007800F04000B6
:10CC200020B101205749091D086003E00020554943
:10CC3000091D08605948007800F0800020B10120EB
:10CC400050490831086003E000204E49083108606F
:10CC50005248008800F4807020B1012049490C310D
:10CC6000086003E0002047490C3108604B48008809
:10CC700000F4007020B1012042491031086003E047
:10CC800000204049103108604448008800F480606A
:10CC900020B101203B491431086003E000203949EC
:10CCA000143108603D48008800F4006020B1012084
:10CCB00034491831086003E0002032491831086017
:10CCC0003648008800F4805020B101202D491C31E5
:10CCD000086003E000202B491C3108602F480088C1
:10CCE00000F4005018B101202849086002E000203B
:10CCF000264908602948008800F4804020B10120BE
:10CD000023492039086003E00020214920390860C8
:10CD10002248008800F4004020B101201C491C3941
:10CD2000086003E000201A491C3908601B480068AD
:10CD300000F4803020B1012015491439086003E067
:10CD400000201349143908601448006800F40030CA
:10CD500020B101200E491039086003E000200C4981
:10CD6000103908600D48006800F4802020B10120CF
:10CD70000749091F086003E000200549091F0860F2
:10CD800010BD00009401234250000020B401214254
:10CD9000A0812242B40122425060002054000020B1
:10CDA000001801400000214208B501210820FDF7CC
:10CDB000D1F80320ADF8000010208DF80300032007
:10CDC0008DF8020069469748FCF7E8FD0321954875
:10CDD000FCF791FE01211020FDF7BCF82020ADF8F2
:10CDE000000010208DF8030003208DF80200694632
:10CDF0008D48FCF7D3FD20218B48FCF77CFE08BD55
:10CE000010B58848006820F00F0086490860084681
:10CE1000006840F0030008600120844908608449EC
:10CE2000C1F88401042002F0E5FB00207F4908607E
:10CE3000042002F0DFFB00207D49C1F8840110BD11
:10CE400010B57848006820F00F0076490860084661
:10CE5000006840F00300086000207449091D086064
:10CE60007349C1F88001042002F0C4FB01206F491E
:10CE7000091D08606E49C1F88001042002F0BAFB68
:10CE800010BD10B500246748006820F00F00654908
:10CE900008600846006840F0080008600120634907
:10CEA000086002F0A7FB01206149C1F8840102F08B
:10CEB000A1FB07E0601CC4B2FA2C03DDFFF7C0FF42
:10CEC000012010BD5948803800680028F2D1574928
:10CED000091D086000BFF4E710B500205349091D83
:10CEE00008605048006820F00F004E49086008466E
:10CEF000006840F00300086000204D49C1F880013F
:10CF0000022002F077FB01204849091D0860022039
:10CF100002F070FB00204649C1F8840110BD10B535
:10CF200000204249091D08603E48006820F00F00BB
:10CF30003C4908600846006840F003000860012092
:10CF40003B49C1F88001022002F054FB012037491F
:10CF5000091D0860022002F04DFB00203449C1F891
:10CF6000840110BD70B504462E48006820F00F0003
:10CF70002C4908600846006840F003000860002063
:10CF80002A49091D0860002517E0E00927490860C3
:10CF90006006040E022002F02DFB01202449C1F896
:10CFA0008401022002F026FB00202049091D0860B0
:10CFB000022002F01FFB681CC5B2082DE5DB70BD26
:10CFC00070B5054600241748006820F00F00154989
:10CFD00008600846006840F008000860002617E076
:10CFE00000201249091D0860022002F003FB012005
:10CFF0000F49C1F884016006040E0C4880380068AF
:10D0000008B1601CC4B2012002F0F4FA701CC6B270
:10D01000082EE5DB15B9FFF782FF01E0FFF75CFFA3
:10D02000204670BD000C014000100140808121426B
:10D030000080214210B5FFF7B7FE10BD70B5044661
:10D040000026FFF7DDFE2546E11704EB116109120A
:10D05000A02202EB4101C8B2FFF784FFFFF711FFE6
:10D06000E11704EB11610912A4EB0121C8B2FFF72B
:10D0700079FFFFF706FFFFF7C3FEA120FFF772FF5E
:10D08000FFF7FFFE0020FFF79BFF0646FFF7D8FEE5
:10D09000304670BD70B504460E4600204949086010
:10D0A000012002F0D2FAFFF7ABFE2546E11704EBB0
:10D0B00011610912A02202EB4101C8B2FFF752FF31
:10D0C000FFF7DFFEE11704EB11610912A4EB012168
:10D0D000C8B2FFF747FFFFF7D4FE3046FFF742FF25
:10D0E000FFF7CFFEFFF7ACFE01203749C1F89401EE
:10D0F000052002F0AAFA70BD2DE9F04105460E4662
:10D100001746002409E0E20026FA02F2D1B22A19F9
:10D1100090B2FFF7BFFF601CC4B2BC42F3DBBDE8B6
:10D12000F0812DE9F04107460C460026002509E074
:10D1300036023919491B491E88B2FFF77FFF0644A2
:10D14000681CC5B2A542F3DB3046BDE8F08110B5DE
:10D15000FF20FFF773FF0446552C01D1002010BDBE
:10D160005521FF20FFF796FFFF20FFF767FF0446DA
:10D17000552C01D10020F2E70120F0E770B50646FA
:10D180000C46154608E03046721C96B2FFF756FF73
:10D1900004F8010B681E85B2002DF4D170BD70B586
:10D1A00005460C46164606E021782846FFF772FF32
:10D1B000681C85B2641C301EA6F101018EB2F3D149
:10D1C00070BD0000940122420000224270B5054665
:10D1D000002406E0601C84B2B4F5803F01DB00202F
:10D1E00070BD02217F48FDF768F80028F2D029467B
:10D1F0007C48FDF70FF806E0601C84B2B4F5803F70
:10D2000001DB0020ECE701217648FDF756F8002805
:10D21000F2D07448FDF700F8C0B2E1E710B504465B
:10D22000704800884FF6C77108406E49088008466C
:10D2300000882043088001216A48FCF7BAFF10BD2E
:10D2400000B587B0012141F20900FCF783FE0121FE
:10D250000846FCF774FC3820ADF8180018208DF84B
:10D260001B0003208DF81A0006A95F48FCF796FB07
:10D27000BDF818105C48FCF73EFC01A8FCF783FFE2
:10D280000020ADF804004FF48270ADF806000020D5
:10D29000ADF80800ADF80A00ADF80C004FF40070CE
:10D2A000ADF80E003820ADF810000020ADF81200E7
:10D2B0000720ADF8140001A94A48FCF7D5FE01216A
:10D2C0004848FCF776FF322002F0BFF90820FFF74C
:10D2D000A5FFFF20FFF77AFF07B000BD10B5044699
:10D2E000424800884FF6C771084040490880084608
:10D2F00000882043088001213C48FCF75AFF10BDFC
:10D3000070B50546002406E0601C84B2B4F5803F89
:10D3100001DB002070BD02213448FCF7CEFF00285D
:10D32000F2D029463148FCF775FF06E0601C84B254
:10D33000B4F5803F01DB0020ECE701212B48FCF72E
:10D34000BCFF0028F2D02948FCF766FFC0B2E1E735
:10D3500000B587B001210820FCF7FCFD01218803FE
:10D36000FCF705FE4FF46040ADF8180018208DF86A
:10D370001B0003208DF81A0006A91B48FCF70EFBC2
:10D380004FF460411848FCF7B6FB0020ADF80400EC
:10D390004FF48270ADF806000020ADF808000220BE
:10D3A000ADF80A000120ADF80C004002ADF80E0007
:10D3B0001820ADF810000020ADF812000720ADF8DD
:10D3C000140001A90948FCF74FFE01210748FCF7AA
:10D3D000F0FEFF20FFF794FF3820FFF77FFF07B034
:10D3E00000BD000000300140000C0140003800404A
:10D3F000B548B6494860B64848607047B3480069C8
:10D4000040F08000B14908617047B048C16801F040
:10D41000010008B10120704701F0040008B10220AA
:10D42000F9E701F0100008B10320F4E70020F2E76B
:10D4300070B5044600BFFFF7E8FF0546012D00D098
:10D4400006E0012002F0D6F8601E84B2002CF2D172
:10D4500000BF04B9FF25284670BD70B505460024FD
:10D4600045F6FF70FFF7E4FF0446C4B9974800692A
:10D4700040F002009549086108464561006940F0A6
:10D480004000086145F6FF70FFF7D2FF0446012C0B
:10D4900005D08E48006920F002008C4908612046C2
:10D4A00070BD70B505460E46FF20FFF7C1FF04466C
:10D4B00094B98648006940F00100844908612E80D3
:10D4C000FF20FFF7B5FF0446012C05D07F48006917
:10D4D00020F001007D490861204670BD01460888A2
:10D4E0007047014601F0010010B90888C0B27047CA
:10D4F00031F8010C000AFAE72DE9F04105460E4625
:10D500001746002407E036F814102846FFF7C9FF35
:10D51000AD1C601C84B2BC42F5DBBDE8F08130B5C7
:10D5200003460C461546002207E01846FFF7D6FFD3
:10D5300024F812009B1C501C82B2AA42F5DB30BDBD
:10D540002DE9F05F80468A461746B8F1006F02D396
:10D550006048804501D3BDE8F09F72B6FFF748FFF1
:10D56000A8F1006B4FEADB25CBF34909C9F58064CC
:10D57000A74200DC3C464EE04FF0006101EBC520C5
:10D580004A145549FFF7CBFF00260BE009EB0600D4
:10D59000514931F810004FF6FF71884200D003E086
:10D5A000701C86B2A642F1DB00BFA6421BDA4FF028
:10D5B000006101EBC520FFF750FF002608E03AF8B4
:10D5C000160006EB0901444A22F81100701C86B2CD
:10D5D000A642F4DB4FF0006101EBC5204A143E493E
:10D5E000FFF78AFF04E0224651464046FFF784FFDA
:10D5F000A74200D110E06D1C4FF000090AEB440A6D
:10D6000008EB4408381B87B2B7F5806F02DD4FF492
:10D61000806400E03C46AFE700BFFFF7EFFE62B674
:10D6200000BF98E730B503460C461546002206E0D9
:10D630001846FFF756FFA0545B1C501C82B2AA424A
:10D64000F6DB30BD13B50446012201A92046FFF7E1
:10D6500077FF1CBD2DE9F05F044689469246002500
:10D660002746C846B4F1006F02D31A48844201D35A
:10D67000BDE8F09F00261DE098F801004FEA002B5E
:10D6800098F8000058441FFA80FB08F10208284669
:10D69000691C8DB2114921F810B0B5F5806F07D122
:10D6A00000254FF480623846FFF726FF07F5006734
:10D6B000B01C86B25645DFD325B12A460749384605
:10D6C000FFF71AFF00BFD3E72301674500200240A0
:10D6D000AB89EFCD00000808940E002094060020CE
:10D6E00010B501215048FDF70CFD01214E48FDF712
:10D6F00011FD10BD7FB505460C4601210220FCF747
:10D7000036FCADF80850ADF804400020ADF80A0032
:10D71000ADF8060001A94448FCF7DAFE1D208DF89B
:10D72000000000208DF8010002208DF80200012089
:10D730008DF803006846FBF7B2FD012211463A4816
:10D74000FDF73DFA01213848FDF71EFA7FBD10B5FF
:10D7500001213648FDF7D5FC012804D13448006882
:10D76000401C33490860334801880088401C314A16
:10D770001080B1F57A7F07DB0020114608802E4823
:10D780000068401C2C4908602C48008841F2883110
:10D79000884205DA29480088401C2849088002E0B0
:10D7A00000202649088026480078401C244908703B
:10D7B000084600780A2804D1FFF78BF8002020499A
:10D7C000087001211948FDF7A5FC10BD7FB505467D
:10D7D0000C4601211020FCF7CAFBADF80850ADF84B
:10D7E00004400020ADF80A00ADF8060001A90F487A
:10D7F000FCF76EFE36208DF8000001208DF8010048
:10D8000003208DF8020001208DF803006846FBF725
:10D8100046FD012211460548FDF7D1F901210348D3
:10D82000FDF7B2F97FBD0000000400400010004089
:10D83000640000206A000020C4010020E8030020EA
:10D840006800002008B501210820FCF783FBC020F8
:10D85000ADF8000010208DF8030003208DF80200C1
:10D860006946FC48FCF79AF84FF48070ADF8000068
:10D8700048208DF8030003208DF802006946F54822
:10D88000FCF78CF840F2CF216420FFF79FFF802146
:10D89000F048FCF732F90A2001F0D7FE8021ED486C
:10D8A000FCF729F90A2001F0D0FE8021E948FCF7B5
:10D8B00024F90A2001F0C9FE8021E648FCF71BF993
:10D8C0000A2001F0C2FE8021E248FCF716F90A2086
:10D8D00001F0BBFE8021DF48FCF70DF90A2001F0C2
:10D8E000B4FE8021DB48FCF708F90A2001F0ADFE08
:10D8F0008021D848FCF7FFF80A2001F0A6FE08BDF9
:10D9000070B505460C4600264021D248FCF7F5F8D4
:10D9100004F01F0040EA05063046FFF757FCFF20E1
:10D92000FFF754FC064604F0800018B1FF20FFF713
:10D930004DFC06464021C748FCF7DDF8304670BD77
:10D940002DE9F04104460D46164600274021C14806
:10D95000FCF7D3F805F01F0040EA04073846FFF74C
:10D9600035FC3046FFF732FC4021BA48FCF7C3F8DB
:10D97000BDE8F08170B505460C464021B548FCF77E
:10D98000BCF83A20FFF722FC05E06D1E0020FFF7EF
:10D990001DFC2070641C002DF7D100202070402158
:10D9A000AC48FCF7A8F870BD70B504460D464021A0
:10D9B000A848FCF7A2F87A20FFF708FC04E0641EF0
:10D9C0002878FFF703FC6D1C002CF8D14021A148FA
:10D9D000FCF791F870BD10B5044604F060009E4954
:10D9E000097888420ED003221F21A020FFF7A8FF4C
:10D9F000C4F341121F218020FFF7A2FF04F0600052
:10DA00009549087010BD10B504462046FFF7E3FFA6
:10DA100021460020FFF774FF10BD70B504460D4687
:10DA20002046FFF7D8FF2A4621464020FFF788FF0F
:10DA300070BD70B505460C4600262946D420FFF778
:10DA4000ECFFE1B2D620FFF7E8FFC4F30721D720AF
:10DA5000FFF7E3FF01E0701C86B2EA20FFF7D3FF77
:10DA600000F0010018B140F6FF708642F3DB70BD94
:10DA700070B504460025FFF7E5FE09E0FF2200210E
:10DA80001046FFF75DFF681C85B20A2001F0DDFD3E
:10DA90001D20FFF7B8FF00F0010010B9B5F5FA7FBF
:10DAA000ECDBB5F5FA7F01DB012070BD00206B498E
:10DAB000086000210820FFF7B0FF00210920FFF7D0
:10DAC000ACFF00210C20FFF7A8FF00210D20FFF77D
:10DAD000A4FF10210A20FFF7A0FF1A210B20FFF757
:10DAE0009CFF11210420FFF798FF1A210520FFF762
:10DAF00094FFFF210620FFF790FF1F210720FFF76B
:10DB00008CFFA1213820FFF788FF3F212820FFF755
:10DB100084FF30212920FFF780FFF9213020FFF713
:10DB20007CFFF7213120FFF778FF0D21C020FFF7A0
:10DB300074FF0021C120FFF770FF3322C221802033
:10DB4000FFF7FEFE1221C620FFF767FF0C21C7205A
:10DB5000FFF763FF1521C420FFF75FFFEE21CA2006
:10DB6000FFF75BFF0521CB20FFF757FF2178E4206B
:10DB7000FFF753FF6178E520FFF74FFFA178E22020
:10DB8000FFF74BFFE178E320FFF747FF2179E02023
:10DB9000FFF743FF6179E120FFF73FFF4FF480710A
:10DBA0000020FFF746FF4FF480711020FFF741FF80
:10DBB0001F20FFF710FFC0221B218020FFF7C0FEAF
:10DBC00004221F218020FFF7BBFEE420FFF71BFF8C
:10DBD0002178884201D1002067E7012065E710B570
:10DBE0007220FFF710FF10BD70B504460D461121DD
:10DBF0000220FFF712FF1A210320FFF70EFF11206A
:10DC00002044C1B20620FFF708FF41F6112020444E
:10DC1000C0F307210720FFF700FF002211467A20FA
:10DC2000FFF78EFE29462046FFF7BEFE08221F2181
:10DC30008020FFF785FE1C20FFF7E5FE00F00200C4
:10DC400030B108221F21A020FFF77AFE03F078FBF5
:10DC500070BD0000000C01406C000020700000202E
:10DC60002DE9F04105460F463920FFF7CCFE10B9EB
:10DC70000020BDE8F0812D4801780020FFF7CDFE9F
:10DC80002A480088C0F307210120FFF7C6FE0021C3
:10DC90003A20FFF735FE2549086000213A20FFF7BA
:10DCA0002FFE2249096841EA00202049086000212E
:10DCB0003A20FFF725FE044600213A20FFF720FE18
:10DCC00044EA0024241F00213A20FFF719FE0646EB
:10DCD00000213A20FFF714FE46EA0026681EA04203
:10DCE00004D203F02DFB6C1E0020C2E706F080007A
:10DCF00020B903F025FB00240020BAE7394620466E
:10DD0000FFF738FE094801780C20FFF786FE074828
:10DD10000088C0F307210D20FFF77FFE40221E215F
:10DD20008020FFF70DFE2046A3E7000070000020D2
:10DD300008B51F20ADF8000010208DF80300022068
:10DD40008DF802006946FE48FBF728FEFD48C07BBF
:10DD500000280EDC4FF44070ADF8000010208DF864
:10DD6000030002208DF802006946F748FBF716FE13
:10DD700011E001214020FCF7EDF84FF4C040ADF870
:10DD8000000010208DF8030002208DF80200694683
:10DD9000EE48FBF703FE01214FF40470FCF7DAF8BC
:10DDA0001020ADF8000000208DF803006946E64819
:10DDB000FBF7F4FD08BD00B585B04FF40040FCF75B
:10DDC0002DF801214802FCF7C5F8002000908DF8DD
:10DDD00004008DF805004FF46020029000200390AD
:10DDE00001208DF810006946D948FBF7E8FA0121B7
:10DDF000D748FBF710FBD648FBF72FFB00BFD448F2
:10DE0000FBF730FB0128FAD0D148FBF735FB00BF08
:10DE1000CF48FBF736FB0128FAD005B000BD08B5A6
:10DE200001210420FCF796F80120ADF8000028201D
:10DE30008DF803006946C248FBF7B0FD052001F0EC
:10DE400004FCC448006818B10120C349087002E00E
:10DE50000020C149087008BD10B5FFF7E0FFFFF7CB
:10DE600067FFFFF7A8FF10BD70B50446C4EBC40000
:10DE700000EB0410B94901EB400090F8235005F085
:10DE80000F05C4EBC40000EB041001EB400090F858
:10DE90002800012870D1C4EBC40000EB041001EB92
:10DEA000400090F82D00142809DBC4EBC40000EBFF
:10DEB000041001EB400090F82D00182814DDC4EB8D
:10DEC000C40000EB0410A54901EB400090F82D00C0
:10DED0000F2809D0C4EBC40000EB041001EB400094
:10DEE00090F82D00192874D1C4EBC40000EB041085
:10DEF0009A4901EB400090F82300C0F30310022878
:10DF000016D19048C07B002807DC012094490860A6
:10DF100000209449C1F8A40106E00120924908605C
:10DF200000209249C1F8B80102209149085515E234
:10DF3000C4EBC40000EB0410884901EB400090F8EA
:10DF40002300C0F30310032817D17E48C07B0028AC
:10DF500007DC00208249086001208249C1F8A40141
:10DF600006E000208049086001208049C1F8B8011E
:10DF700003207F490855F1E12BE0C4EBC40000EB1E
:10DF80000410764901EB400090F82300C0F3031021
:10DF9000012809D10020724908607249C1F8A40122
:10DFA000012073490855D9E16648C07B002806DC8A
:10DFB00001206B4908606B49C1F8A40105E001200C
:10DFC000694908606949C1F8B801002068490855E5
:10DFD000C4E1C4EBC40000EB0410604901EB400055
:10DFE00090F82800012836D1C4EBC40000EB0410DF
:10DFF00001EB400090F82D000B2809D0C4EBC400C1
:10E0000000EB041001EB400090F82D00112822D104
:10E010004C48C07B002807DC0120514908600020E3
:10E020005049C1F8A40106E001204F4908600020D2
:10E030004E49C1F8B80145F0200040B2C4EBC4011C
:10E0400001EB0411454A02EB410181F82300022053
:10E050004749085582E1C4EBC40000EB04103F4976
:10E0600001EB400090F82800012851D1C4EBC40016
:10E0700000EB041001EB400090F82D00132809D0AC
:10E08000C4EBC40000EB041001EB400090F82D003D
:10E0900010283DD12B48C07B002807DC00203049E8
:10E0A000086001202F49C1F8A40106E000202E4994
:10E0B000086001202D49C1F8B801C4EBC40000EB91
:10E0C0000410264901EB400090F8230000F00F00F7
:10E0D000C4EBC40101EB0411204A02EB410181F8B9
:10E0E0002300C4EBC40000EB0410114601EB400018
:10E0F00090F9230040F03000C4EBC40101EB04119F
:10E1000002EB410181F8230003201949085525E15C
:10E11000C4EBC40000EB0410104901EB400090F880
:10E12000280001287DD1C4EBC40000EB041001EBF2
:10E13000400090F82D000C2856D0C4EBC40019E024
:10E14000000801405060002000100140001801400C
:10E150000024014000012142740000205F6F002074
:10E16000A001224200002242B401234200002342C7
:10E170001F75002000EB041001EB400090F82D000B
:10E18000282831D0C4EBC40000EB041001EB4000A0
:10E1900090F82D00292827D0C4EBC40000EB041010
:10E1A00001EB400090F82D002A281DD0C4EBC400DC
:10E1B00000EB041001EB400090F82D000C2813D068
:10E1C000C4EBC40000EB041001EB400090F82D00FC
:10E1D0000D2809D0C4EBC40000EB041001EB400093
:10E1E00090F82D00122840D1FE48C07B002806DCA4
:10E1F0000020FD490860FD49C1F8A40105E00020A8
:10E20000FB490860FB49C1F8B801C4EBC40000EB4E
:10E210000410F94901EB400090F8230000F00F00D2
:10E2200000E022E0C4EBC40101EB0411F24A02EB6E
:10E23000410181F82300C4EBC40000EB0410114637
:10E2400001EB400090F9230040F01000C4EBC40142
:10E2500001EB041102EB410181F823000120E749A1
:10E2600008550A2001F0F1F978E0C4EBC40000EB96
:10E270000410E14901EB400090F82D00092809D075
:10E28000C4EBC40000EB041001EB400090F82D003B
:10E290000A282AD10520D9490855C4EBC40000EB4F
:10E2A0000410D54901EB400090F8230000F00F0066
:10E2B000C4EBC40101EB0411CF4A02EB410181F828
:10E2C0002300C4EBC40000EB0410114601EB400036
:10E2D00090F9230040F05000C4EBC40101EB04119D
:10E2E00002EB410181F8230038E0BE48C07B0028E2
:10E2F00006DC0120BC490860BC49C1F8A40105E066
:10E300000120BB490860BB49C1F8B801C4EBC40097
:10E3100000EB0410B84901EB400090F8230000F036
:10E320000F00C4EBC40101EB0411B34A02EB41013D
:10E3300081F82300C4EBC40000EB0410114601EB8C
:10E34000400090F92300C4EBC40101EB041102EB7F
:10E35000410181F823000020A849085570BD70B51F
:10E3600004460D46002602212046FBF70EFA05233F
:10E37000012229462046FBF7BAF801212046FBF787
:10E380008AF800BF02212046FBF7F6F90028F9D0F1
:10E390002046FBF713F90646304670BD2DE9F047DD
:10E3A0004FF000084FF0010A95480078C0EBC0011B
:10E3B00001EB0010904901EB400090F82D00192866
:10E3C0002ED000251EE00E218E48FFF7C8FF044620
:10E3D000A044BAF1010F04D12646A1464FF0000A2D
:10E3E0000BE0A64201DD304600E020460646A1458E
:10E3F00001DA484600E020468146012001F025F977
:10E40000681CC5B20C2DDEDBA8EB0600A0EB0900F2
:10E410000A21B0FBF1F07C49794A127821F8120008
:10E4200077480078C0EBC00101EB0010724901EBA6
:10E43000400090F82D000F280CD071480078C0EBF8
:10E44000C00101EB00106C4901EB400090F82D0079
:10E45000192844D16C486A49097830F811006B4991
:10E46000674A127821F81200654800780B2836DBDD
:10E4700067486349097830F811006449604A1278A6
:10E4800031F81210884220DD61485D49097830F882
:10E4900011005E495A4A127831F81210401AB0F54C
:10E4A000FA6F12DD4F4840305549097850F8310075
:10E4B000401C4C494031524A127841F83200012147
:10E4C00054484F4A127820F8121050484C490978A5
:10E4D00030F811004E494A4A127821F81200484893
:10E4E0000078401C4649087008460078202801DB67
:10E4F00000200870424800780B282ADA27E04048BC
:10E500000078C0EBC00101EB00103B4901EB40007B
:10E5100090F82D000F280CD039480078C0EBC001CE
:10E5200001EB0010344901EB400090F82D00192850
:10E530000CD1642001F089F831480078401C304942
:10E540000870084600780B2801D101E000E0D6E70A
:10E5500000BF3148FBF7CBFA07464FF6E0700740A3
:10E560002748007847EA00012B48FBF7CDFA2448FA
:10E570000078FFF779FCBDE8F0871FB5044604EB8F
:10E58000840000EBC400254908448088ADF80C00E5
:10E5900048208DF80F0003208DF80E0004EB840155
:10E5A00001EBC4011D4A1144086803A9FBF7F6F901
:10E5B00004EB840202EBC402184B1A44918804EB6A
:10E5C000840202EBC4021A441068FBF794FA04EBCD
:10E5D000840202EBC402114B1A44D17904EB840289
:10E5E0001EE0000050600020A001224200002242F4
:10E5F000B4012342000023425F6F00201F750020FA
:10E60000B600002000240140D4160020201700206E
:10E61000760000209416002000080140A027020880
:10E6200002EBC4021A449079FBF7CEFA04EB8400A3
:10E6300000EBC4007D490844D0F809000190002097
:10E640008DF808000C208DF8090001208DF80A00D3
:10E6500001A8FBF7C3F804EB840000EBC400734986
:10E660000844007A8DF8000000208DF80100012098
:10E670008DF802008DF803006846FAF710FE1FBD02
:10E680006B48006800F0010010B101206849086083
:10E690006848D0F88800401C6649C1F8880001200D
:10E6A000654948726549488270476148006800F0D2
:10E6B000020010B102205E4908605E48006F401CF5
:10E6C0005C49086701205D4988815B498871704712
:10E6D0005748006800F0040010B104205449086055
:10E6E0005448806F401C5349886701205349C881B2
:10E6F0005149C87170474E48006800F0080010B1D9
:10E7000008204B4908604B48806E401C4949886688
:10E7100001204A4948814849487170474448006887
:10E7200000F0800060B18020414908604148006CE1
:10E73000401C404908640120404908803E49087057
:10E740003B48006800F0400060B140203849086054
:10E750003848806C401C374988640120374948801C
:10E76000354948703248006800F0200060B1202030
:10E770002F4908602F48006D401C2E490865012074
:10E780002E4988802C49887070472948006800F419
:10E79000006068B14FF40060254908602548806D2D
:10E7A000401C2449886501202449C8802249C8703A
:10E7B0001F48006800F4805078B14FF480501C4925
:10E7C00008601C48D0F88000401C1A49C1F880003D
:10E7D00001201A490882184908721548006800F497
:10E7E000806068B14FF48060114908601148006E84
:10E7F000401C104908660120104908810E49087123
:10E800000B48006800F4804078B14FF4804008491C
:10E8100008600848D0F89000401C0649C1F89000F4
:10E82000012006498882044988727047A02702089F
:10E83000140401405060002014170020941600209A
:10E8400010B5002407E004EB8401F94A02EB8100D3
:10E8500000F0FCFC641C0A2CF5D3F64800F0F6FC32
:10E86000F54800F0F3FCF54800F0F0FCF44800F047
:10E87000EDFCF44800F0EAFCEE48F3490860EE488D
:10E88000F249086010BD2DE9F04104460E461546D8
:10E890009846069F1022314604F1340011F073FCB3
:10E8A0000021432001550A2D00D30925E562201DD2
:10E8B00000F0D9FC04F1180000F0D5FC2461C5F18A
:10E8C0000A00A0616462BDE8F08170B505460E469D
:10E8D000442000F05FFD044694B11EB9A80000F08A
:10E8E00059FD00E030462063206B20B9204600F03F
:10E8F000B2FD002404E0A900A522206B11F0F2FB78
:10E90000204670BD2DE9FF4F81B0804615469946DF
:10E91000DDE90E7A28461099FFF7D7FF0446002C50
:10E9200056D0681E216B01EB800B2BF0070B009576
:10E930003A462046119B0299FFF7A5FF4A464146F9
:10E94000584600F0CDFC2060BAF1000F01D0CAF8A3
:10E95000004000F0F5FCBE480068401CBC4908605F
:10E96000BC48006840B9BB480460084600680128FC
:10E970000CD1FFF765FF09E0B748006830B9B5482A
:10E980000068C06AB84201D8B2480460B349E06A7E
:10E990000968884202D9B149E06A0860B048006855
:10E9A000401CAF490860AF49E06A0968884202D953
:10E9B000AC49E06A0860E16A01EB81019C4A02EB24
:10E9C0008100211D00F052FC012600F0C2FC01E094
:10E9D0004FF0FF36012E09D19F48006830B19D48A5
:10E9E0000068C06AB84201D200F0A4FC304605B00D
:10E9F000BDE8F08F70B5044600F0A2FC95480068B1
:10EA0000844200D1002414B99248006800E02046F6
:10EA10000546281D00F052FCA86A18B105F118003F
:10EA200000F04CFC291D864800F020FC8E48006850
:10EA3000401C8D4908608A480068401C884908606D
:10EA400000F087FC8448006810B10CB900F072FC3B
:10EA500070BD70B585480068002866D1844800689C
:10EA6000401C834908600846006808BB764908686E
:10EA700076490968744A1160744908607D490968DB
:10EA8000491C7C4A116070490968096809B901216B
:10EA900000E0002121B14FF0FF31774A116006E01C
:10EAA00069490968C968CC68734A6168116000BF28
:10EAB0006F48006870490968884235D300BF6248D2
:10EAC0000068006808B9012000E0002020B14FF084
:10EAD000FF306949086026E05B480068C068C46888
:10EAE000656863480068A84202D2634805601AE07E
:10EAF000201D00F0E3FBA06A18B104F1180000F03B
:10EB0000DDFB5849E06A0968884202D95549E06A44
:10EB10000860E16A01EB8101454A02EB8100211D99
:10EB200000F0A4FBCBE700BF04E054480068401CA1
:10EB30005249086070BD70B5002500F001FC4B48DB
:10EB40000068401E494908600846006800284CD10A
:10EB50003F480068002848D0002621E03748C068B8
:10EB6000C46804F1180000F0A9FB201D00F0A6FB0A
:10EB70003C49E06A0968884202D93A49E06A08607B
:10EB8000E16A01EB81012A4A02EB8100211D00F0BC
:10EB90006DFB3049E06A0968C96A884200D30126E2
:10EBA0002648006808B9012000E000200028D5D0E0
:10EBB0003248006860B106E0FFF74BFF2F4800685D
:10EBC000401E2E4908602D4800680028F4D1012617
:10EBD000012E03D02A480068012805D10125002014
:10EBE0002749086000F0A6FB00BF00F0B2FB2846F2
:10EBF00070BD10B504461748006844601C480068A2
:10EC0000844207D213480168091D1048006800F0CB
:10EC10003BFB0CE00F480168091D0B48006800F041
:10EC200033FB15480068844201D21348046010BDCC
:10EC300060170020281800203C18002050180020E1
:10EC40006418002078180020BC000020C0000020BC
:10EC5000C8000020B8000020D8000020D00000200C
:10EC6000EC000020D4000020C4000020DC000020C4
:10EC7000CC000020E8000020F0000020E000002090
:10EC8000E4000020F9480068401CF849086070471B
:10EC90002DE9F04104460F464FF00008FFF7F2FF60
:10ECA0002068C519F24920680968884209D9206896
:10ECB000A8420FD9EE48006885420BD94FF00108F1
:10ECC00008E02068A84203D8E9480068854201D9D5
:10ECD0004FF001082560B8F1000F07D0E548006843
:10ECE000001D00F0EBFA2846FFF783FFFFF723FF34
:10ECF00006460EB900F01EFBBDE8F08170B5044673
:10ED000000267CB1FFF7BEFFD94800680519D94835
:10ED10000068001D00F0D2FA2846FFF76AFFFFF7EF
:10ED20000AFF06460EB900F005FB70BD70B504463B
:10ED300000F006FB14B9CF48006800E02046064604
:10ED4000F56A00F006FB284670BD2DE9F041064645
:10ED50000D464FF000080A2D00D3092500F0F0FA07
:10ED6000C4480068864200D1002616B9C148006830
:10ED700000E030460446E76AAF422DD0BD4203D9D9
:10ED80002EB14FF0010802E00EB94FF00108E56224
:10ED9000C5F10A00A06107EB8701B74A02EB8101C8
:10EDA0006069884213D1201D00F088FAB349E06AF7
:10EDB0000968884202D9B149E06A0860E16A01EB5A
:10EDC0008101AD4A02EB8100211D00F04FFAB8F13C
:10EDD000010F01D100F0AEFA00F0BBFABDE8F081FE
:10EDE000A248006818B10120A549086025E004E0A8
:10EDF000A2480068401EA1490860A048006800EBD6
:10EE000080009D4951F820000028F1D09B490968F5
:10EE100001EB8101984A02EB810041684968416039
:10EE200000F1080142688A4202D1416849684160A4
:10EE30004168C9688F4A116000BF704770B50446C9
:10EE400000F07EFA8B480068844200D1002414B997
:10EE50008848006800E020460546281D00F02EFA8C
:10EE6000A86A18B105F1180000F028FA291D854894
:10EE700000F0FCF900F06DFA8CB98348006810B11D
:10EE800000F058FA0BE07F48006880490968884222
:10EE900003D100207749086001E0FFF7A1FF70BDB2
:10EEA00010B5014600200A46764C5369A34201D1B1
:10EEB000012300E0002383B1754C936AA34201D182
:10EEC000012300E00023012B07D0936A0BB9012333
:10EED00000E00023012B00D1012010BD70B50546D4
:10EEE0002C4644B363480068844224D000F028FADA
:10EEF0002046FFF7D5FF01281BD1201D00F0DEF9C9
:10EF00005E49E06A0968884202D95C49E06A0860A3
:10EF1000E16A01EB8101584A02EB8100211D00F0FA
:10EF2000A5F95449E06A0968C96A884201D300F02A
:10EF300001FA00F00EFA70BD70B5054600262C46A9
:10EF40002046FFF7ADFF012826D148480068F0B9F8
:10EF50004849E06A0968C96A884201D3012000E093
:10EF600000200646201D00F0A9F94449E06A09681E
:10EF7000884202D94149E06A0860E16A01EB8101F7
:10EF80003D4A02EB8100211D00F070F904E004F11C
:10EF900018013F4800F06AF9304670BD10B50446CC
:10EFA000206B00F058FA204600F055FA10BD70B5FD
:10EFB0003848006818B3FFF765FE3748006808B99D
:10EFC000012000E000200546FFF7B5FDBDB900F0C7
:10EFD000B7F93148C068C468201D00F06FF92B48AC
:10EFE0000068401E294908602A480068401E2949D7
:10EFF000086000F0AEF92046FFF7D0FF00BF70BDFB
:10F0000000BFFFF7D4FF1C4800680128F9D900F0C1
:10F0100091F9F6E71FB50020009001900290034699
:10F0200080221EA103901F48FFF76CFC0446012CB0
:10F0300009D1F9F749F901201349086000200C496A
:10F04000086000F061F91FBD10B5F9F73DF9002027
:10F050000D49086000F06DF910BD10B500F070F9B1
:10F060000348046800F075F9204610BDDC0000205C
:10F07000CC000020B800002060170020D400002041
:10F08000E400002078180020D8000020C8000020EC
:10F0900050180020C40000206418002049444C454A
:10F0A0000000000001F0000870B50025F9F70CF928
:10F0B0005B480468F9F70FF9204670BD59480068AD
:10F0C000704770B506460C465748016818313046FF
:10F0D00000F0DAF854480068001D00F0EFF8601CFA
:10F0E00030B951480168091D504800F0BFF805E0EB
:10F0F0004B48006805192846FFF77BFD70BD70B5C9
:10F100000646F068C46804F1180000F0D7F84848D3
:10F110000068A0B9201D00F0D1F84649E06A0968EE
:10F12000884202D94349E06A0860E16A01EB810143
:10F13000414A02EB8100211D00F098F804E004F13F
:10F1400018013E4800F092F83749E06A0968C96A38
:10F15000884201D3012500E00025284670BD3849CA
:10F16000096801602E4909684160704770B504461E
:10F170000D4600F0E5F82868401C08B900261FE09D
:10F180002F4920680968884206D0254960680968C7
:10F19000884201D8012613E0214960680968081AED
:10F1A000296888420BD228681D4A61681268511A82
:10F1B000401A28602046FFF7D2FF002600E0012613
:10F1C00000F0C7F8304670BD01201E490860704746
:10F1D0000146002002E0491C421C90B20A78A52A90
:10F1E000F9D0800870472DE9F041044614B90E4863
:10F1F000006800E0204607463D6B2846FFF7E8FF21
:10F2000006463046BDE8F0810F49096809B900207B
:10F2100005E00749096809B9012000E002207047AC
:10F22000CC000020C8000020B80000207818002082
:10F23000DC000020D40000206017002050180020BF
:10F24000E8000020E4000020D800002000F10801C0
:10F2500041604FF0FF31816000F10801C160016140
:10F2600000210160704700210161704742685368C6
:10F270004B6043688B6053689960516041600861DE
:10F2800003685B1C0360704710B502460B685C1C8A
:10F290000CB9106907E002F1080000E0406844681A
:10F2A00024689C42FAD944684C604C68A16088602C
:10F2B00041600A611468641C146010BDD0E9013219
:10F2C0009A60D0E901235A6001694A68824201D1FB
:10F2D00082684A60002202610A68521E0A60704712
:10F2E000001F4FF080730360001F0160001F0023A8
:10F2F0000360143802602038704723484FF0E02143
:10F30000486107200861704710B52048006840F444
:10F310007F001E4908600846006840F07F40086092
:10F32000FFF7EBFF00201A490860F8F7A5FF00205F
:10F3300010BD70474FF0805014491C390860704769
:10F3400010B5F8F7C1FF12480068401C104908606A
:10F3500010BD10B50E480068401E0D4908600846F3
:10F36000006808B9F8F7B7FF10BD10B54FF080502E
:10F3700006491C3908600024F8F7A6FFFFF769FB6F
:10F38000F8F7A9FF10BD00003F19010020ED00E0D3
:10F39000F40000202DE9F04104464FF00008FFF78B
:10F3A00071FC3D48006898B93C493D4A1160002114
:10F3B00051604FF440513B4A516000211160374881
:10F3C0004FF440514160114601600120324908600C
:10F3D00044B1103404F0070020B104F00700C0F17C
:10F3E00008000444002C31D0B4F5405F2ED22C4FDD
:10F3F0003846056801E02F462D686868A04202D2B1
:10F4000028680028F7D1274885421FD0386800F1C6
:10F410001008286838606868001B202810D92E1949
:10F420006868001B70606C6071681D4800E00068CF
:10F43000026852688A42FAD302683260066000BFEE
:10F44000194968680968081A17490860FFF773FBCB
:10F450004046BDE8F08170B506463546B6B1103D70
:10F460002C46FFF70FFC61680D4800E00068026859
:10F4700052688A42FAD30268226004600A496068CE
:10F480000968084408490860FFF755FB70BD064845
:10F4900000687047704700000C01002090180020A1
:10F4A000F8000020000100200801002000BF704784
:10F4B00000BF704770B504460D460120384908600A
:10F4C00000BF40213748FBF7E7FF0028F9D0A1B281
:10F4D0003448FBF773FF002031490860204670BDB7
:10F4E00010B586B00446012144F20400FAF732FD5B
:10F4F0002C48FBF727FE4FF40070ADF814000320F2
:10F500008DF8160018208DF8170005A92648FAF77F
:10F5100045FA4FF48060ADF8140004208DF8170010
:10F5200005A92148FAF73AFA4FF48070ADF81400B3
:10F5300010208DF8170005A91B48FAF72FFA4FF491
:10F5400080711948FAF7D7FA25208DF800000020BD
:10F550008DF801008DF8020001208DF80300684647
:10F56000F9F79DFE01940020ADF80800ADF80A00FF
:10F57000ADF80C00ADF810000C20ADF80E0001A99C
:10F580000848FBF722FE012240F225510548FBF70F
:10F59000B4FE01210348FBF7A4FE06B010BD000035
:10F5A000A0012142003801400008014010B54FF091
:10F5B000E022126922F004024FF0E0231A61C3171F
:10F5C00000EB5373C3F3C7032F4C2370C31700EB37
:10F5D0005373D9104FF47A72514301222B4B1A8086
:10F5E0004FF0E0225161126942F001024FF0E02336
:10F5F0001A6110BD2DE9F047074600264FF0E020C4
:10F60000D0F814902048007807FB00F800BFFFF7FF
:10F6100097FE4FF0E020856911E04FF0E02084690B
:10F62000AC420CD0AC4202D2281B064403E0A9EB4A
:10F630000400284406442546464500D300E0ECE794
:10F6400000BFFFF786FEBDE8F08770B50446FFF700
:10F65000DBFD88B10D480088844206DB0B4800883A
:10F6600094FBF0F52846FFF749FB0848008894FB17
:10F67000F0F100FB114084B24FF47A7104FB01F009
:10F68000FFF7B8FF70BD0000160100201801002030
:10F6900070B504460D46656001F04CFE206070BDFB
:10F6A000D0E9001211440160704710B5044601F022
:10F6B00041FE206010BD10B5044601F03BFE2168FC
:10F6C000401A6168884201DB012010BD0020FCE780
:10F6D000F74908807047C2780A44F64BDA7082789E
:10F6E00002EB21229A7042785A7002781A701A46F8
:10F6F0009278B2EB212F0ADA1A465278521C5A70CD
:10F700001A4652781AB91A461278521C1A70E94AE7
:10F71000D278CBB29A4212DAE64A9278521CE54B82
:10F720009A701A46927852B91A465278521C5A70F8
:10F730001A4652781AB91A461278521C1A70704733
:10F74000F0B50B46144619461E19751E0BE04E788F
:10F750000F7806EB0726B2B28618B0B2904201DAF3
:10F76000461CB0B2891CA942F1D3A9420AD10E7835
:10F77000002707EB0626B2B28618B0B2904201DA33
:10F78000461CB0B2F0BD0146080240EA212080B21A
:10F79000704770B504460D462A4621460020FFF703
:10F7A000CFFF0646FFF7EFFF70BD10B51422C24928
:10F7B0000020FFF7C5FF044614B94FF6FF7010BDD7
:10F7C0002046FFF7E0FFFAE770B50446BA480E3866
:10F7D000417C007C01EB0020143885B2281986B2E8
:10F7E0000822B5490C313046FFF7AAFF06462A46E3
:10F7F000B14914313046FFF7A3FF064616B94FF65C
:10F80000FF7070BD3046FFF7BEFFFAE710B5062067
:10F81000FFF7DAFF10BD10B51120FFF7D5FF10BDBF
:10F820000020A64908700AE00020A549A34A1278E2
:10F8300021F81200A1480078401CA04908709F4898
:10F8400000781E28F0DB00209C49087012E00020A0
:10F850009A49097801EB81019A4A02EBC101487685
:10F8600014219948954A1278815494480078401C94
:10F8700092490870914800781E28E8DB4FF48060B8
:10F880009249088000208D4908700BE000209049C3
:10F890008A4A127801EB8211888088480078401CDF
:10F8A00086490870854800780A28EFDB70470020F9
:10F8B00017E000EB8001834A02EBC101497E71B180
:10F8C0008149095C491E804A11541146095C31B9CD
:10F8D000002100EB80027B4B03EBC2025176411CFE
:10F8E000C8B20528E5DB704730B504460D4600BFB9
:10F8F00076480088401C7549088008460088B0F5A5
:10F90000FA4F02DB4FF48050088000206B490870EA
:10F9100015E06A48007800EB80006A4901EBC002FC
:10F92000507E38B169480088FFF72DFF91888842E2
:10F9300000D1DDE761480078401C604908705F48ED
:10F9400000781E28E5DB002200205C49087018E0E2
:10F950005A48007800EB80005A4901EBC003587EFA
:10F9600008B91A4611E0587E072805D11AB1987EC9
:10F97000917E884200DD1A4650480078401C4F496D
:10F9800008704E4800781E28E2DB00BF0AB900204C
:10F9900030BD022050764F48007810734D484178B2
:10F9A000517381789173C178D17340F2CA705082DB
:10F9B0009082012010820020D076012090760320D2
:10F9C0001076002090751020D07540480088FFF711
:10F9D000DAFE9080D58000BF20881080608850803B
:10F9E00000BF1046D4E730B503460C4600BF374889
:10F9F0000088401C3549088008460088B0F5FA4F59
:10FA000002DB4FF48050088000202C49087011E080
:10FA10002E480088FFF7B7FE2D49284D2D7801EBC1
:10FA200085118988884200D1E1E724480078401C8C
:10FA300022490870214800780A28E9DB00220020CA
:10FA40001E49087011E022481C49097800EB81101A
:10FA5000808828B91E481949097800EB811208E00E
:10FA600016480078401C15490870144800780A2888
:10FA7000E9DB00BF0AB9002030BD1448007800025D
:10FA80001249098840EA21209080D48013B90020CF
:10FA9000106005E000BF188810805888508000BFB3
:10FAA000402010721046E7E70021044A117026E05A
:10FAB0004C010020540100209E48002058010020E5
:10FAC000445500209450002034580020520100205A
:10FAD000805500204E010020FD49FE4A127831F881
:10FAE0001210814206D10021F94AFA4B1B7822F804
:10FAF00013107047F7490978491CF64A1170F54907
:10FB000009781E29E8DB00BFF3E70021F14A1170F4
:10FB100010E0EF49EF4A127831F8121029B9EC4998
:10FB2000EC4A127821F812007047EA490978491C1A
:10FB3000E84A1170E74909781E29EADB00BFF3E7BC
:10FB400010B504462146E44800680830FFF7C3FDBD
:10FB5000E2480078E04909680872E0484178DE48E8
:10FB600000684172DD488178DB4800688172DB48BB
:10FB7000C178D9480068C17210BD7CB50546D64829
:10FB80000468042D00D15DE3D548D6490860D64904
:10FB90000860032D0FD1607E00F00F00032808D10C
:10FBA000208A30B90820D149087001F060FD01F0C9
:10FBB00010B801F08FB9022D74D1CD48C078401C27
:10FBC000C0B2CB49C87078B908468078401CC0B232
:10FBD000887048B908464078401CC0B2487018B9CF
:10FBE00008460078401C08700020C2490880C249BD
:10FBF0000880607E072802D0607E052808D1A07E9C
:10FC0000401CA076A07E782862D1002060765FE05C
:10FC1000607E00285CD0208A00284ED0A17E481E3D
:10FC2000A076002954D1E07E082808D0607E022802
:10FC300002D0607E012810D1E07E05280DD1002081
:10FC400060768020A949087001F011FD1421A448B4
:10FC5000363880F82F1001F0ABB8E07E042801DDC3
:10FC6000042000E0E07E03218140A176E07E401C7C
:10FC7000E076A248C08C401C81B2A048C184607E5E
:10FC800000F00F00092823D2DFE800F02205060D5E
:10FC9000142215221600FDE300219148363880F821
:10FCA0002F10F8E315E004209049087001F0DFFC04
:10FCB00000F0D1BF00BF00BFEEE3607E00F00F0098
:10FCC000032805D108208949087001F0D0FC6EE7AF
:10FCD0006FE7052D18D18A480068808898B1002008
:10FCE0007D4908607E480C387E4908607E4908607E
:10FCF0000020814908807F49088008207B490870DE
:10FD000002F030FC9EE254E77C484088401C7B496E
:10FD1000488073483638807B45280BD008460088D9
:10FD2000401C08800846C088401CC88075A001F0AF
:10FD3000C5FC3EE76A483638417C007C01EB002078
:10FD40006C490988884208DC65483638417C007C6B
:10FD500001EB00206749088003E074A001F0AEFCCD
:10FD600027E75F483638007D00F03F0018B95C484F
:10FD70003638407D60B161480088401C5F4908808A
:10FD800008468089401C888174A001F097FC10E728
:10FD90007848008878490988884205D175484088A4
:10FDA00075494988884235D04D483638C07D11287C
:10FDB0001CD14B483638C08B70490988884206D11F
:10FDC00047483638008C6D49498888420DD04448F0
:10FDD0003638C08B6A490988884207D1404836388E
:10FDE000008C67494988884200D111E13C48363887
:10FDF000C08B60490988884206D139483638008C62
:10FE00005C494988884205D03C480088401C3B49F1
:10FE10000880CEE6FFF7C9FC4FF6FF7188420CD090
:10FE200036480088401C354908800846C089401C77
:10FE3000C88154A001F042FCBBE629483638C07D99
:10FE4000062800D151E226483638C07D112800D15D
:10FE5000DEE023483638C07D01280CD027480088D2
:10FE6000401C264908800846008A401C08824AA097
:10FE700001F024FC9DE62148808A401C81B21F4885
:10FE800081821748363890F8220008280ED01B4887
:10FE9000408A401C194948820846008B401C81B2A8
:10FEA0001648018343A001F009FC82E600210C48BA
:10FEB000363880F82210808C4FF6F771884205DBC7
:10FEC00007483638808C093081B27FE081E000003D
:10FED0004455002058010020440100205401002016
:10FEE000C6480020340100203801002040010020D5
:10FEF0004E0100203C0100203E010020005800205F
:10FF00004801002069703A20696E76616C6964204E
:10FF100076657273696F6E206F72206865616465C3
:10FF200072206C656E6774682E00000069703A205C
:10FF30007061636B65742073686F7274657220748E
:10FF400068616E207265706F7274656420696E20DE
:10FF50004950206865616465722E000069703A201E
:10FF6000667261676D656E742064726F707065642F
:10FF70002E0000001C01002034280208302802084E
:10FF80002801002069703A2062616420636865631B
:10FF90006B73756D2E0D0A0069703A206E65697479
:10FFA00068657220746370206E6F722069636D7073
:10FFB0002E0D0A0069636D703A206E6F74206963BC
:10FFC0006D70206563686F2E0D0A0000FC48818407
:10FFD00005E0FB48808C083081B2F948818400BF7D
:10FFE000F748418BC183818B018400BF00BFF54876
:10FFF0000188F3484183F3484188F148818300BF79
:020000040801F1
:10000000F148C08A401C81B2EF48C18200F059BF5C
:10001000EE4800881C38ED490880E9482A30EC4950
:1000200008602A38008D88B1FFF7F5FB4FF6FF71A5
:1000300088420BD0E448808D401CE34988850846FF
:10004000408E401C81B2E0484186B2E5E148E24979
:100050000860DBE0E0480068808800287ED0D8484F
:10006000808CDD4909688988884277D1DA48006840
:100070000088DA490988884206D1D7480068408854
:10008000D649498888423FD0D34800680088D4497F
:100090000988884206D1D04800684088D0494988FC
:1000A000884231D0C648408BCB49096809888842CC
:1000B00006D1C348808BC84909684988884223D043
:1000C000BF48C08BC6490988884205D1BC48008C0E
:1000D000C3494988884217D0B948C08BB9490988B3
:1000E000884205D1B648008CB649498888420BD071
:1000F000B348C08BBB49098888422FD1B048008CD7
:10010000B849498888427CD1B3480068C08860B14A
:10011000AB48808CB04909688988884270D1AE4864
:1001200000688088B0F5884F6AD0A548408CAA49FD
:100130000968C88000BFA248408BADF80400A04801
:10014000808BADF8060000BFA748006800909DF8BE
:1001500004009DF80010C1F1FF0100E051E00843E8
:100160008DF804009DF805009DF80110C1F1FF0114
:1001700008438DF805009DF806009DF80210C1F1B6
:10018000FF0108438DF806009DF807009DF8031055
:10019000C1F1FF0108438DF80700BDF80400914943
:1001A0000988884205D1BDF806008E4949888842F1
:1001B00019D0894800680079000287490968898850
:1001C00040EA212080B240F2D24188420BD100BFE8
:1001D00083480088804909680880814840887E49B2
:1001E000096848800BE000BF7548408B7A49096870
:1001F00008807348808B78490968488000BF00BF39
:100200000EE0754800684030734908607248016824
:1002100076488142FFF41EAF75A001F04FFAC8E4A2
:1002200000207C49086002207B49087064482A301D
:10023000674908607949086000207949088002F020
:1002400091F900BF7648008800B9B2E4744800888C
:100250001C305E4908800846008801125848017425
:100260005A480178564841741121C1756C4800887C
:100270000830C0F307216A480078083041EA0020BE
:1002800081B24F48C18400210185534800688188AC
:100290004B48418450480068C1884948818400BF68
:1002A00048480188464841834648418844488183FC
:1002B00000BF00BF4848006801884148C1834648E4
:1002C000006841883E48018400BF363040490860DC
:1002D000FFF7A1FAC04381B239480185008D18B9F2
:1002E0004FF6FF7136480185F8E33748808B401C94
:1002F00081B235488183FFF789FA4FF6FF71884252
:100300000ED03148408B401C2F4948830846008C52
:10031000401C81B22C48018442A001F0CFF948E48E
:10032000454C17E0607EA0B12548808CA1888842AA
:100330000FD12348408CE18888420AD12048408B65
:100340002188884205D11E48808B6188884200D16F
:1003500005E2283439488442E4D9194890F82F003E
:1003600000F03F00022800D021E01548808C34497D
:1003700008800020334908700EE03348314909787D
:1003800030F811002E490988884200D1E6E02D4856
:100390000078401C2B4908702A4800781E28ECDBA6
:1003A0000948408D401C81B20748418500BF044880
:1003B00090F82F0000F0040000B189E446E000004E
:1003C000904800201C010020005800203C01002023
:1003D0003401002080550020480100203428020804
:1003E00030280208280100202401002000580020A5
:1003F0007564703A206E6F206D61746368696E6712
:1004000020636F6E6E656374696F6E20666F756EC4
:100410006400000044010020400100203801002059
:100420003E0100207463703A206261642063686555
:10043000636B73756D2E0000945000201C550020D6
:100440005A0100205801002044550020FE48808CAD
:10045000401C81B2FC4881841421FC4880F82F1094
:100460002820FB4908805021F84880F82E1090F889
:100470002900F8490870F54890F82D1080F82910E7
:10048000F4480178F14880F82D1090F82800F149DF
:10049000087002E042E146E13FE3EC4890F82C109E
:1004A00080F82810EB480178E84880F82C1090F884
:1004B0002700E8490870E54890F82B1080F82710CD
:1004C000E4480178E14880F82B1090F82600E149D3
:1004D0000870DE4890F82A1080F82610DD48017870
:1004E000DA4880F82A1090F82D00401CC1B2D74895
:1004F00080F82D10B1B990F82C00401CC1B2D3483F
:1005000080F82C1071B990F82B00401CC1B2CF4874
:1005100080F82B1031B990F82A00401CC1B2CB48AA
:1005200080F82A10C948408CCB490880C748818C84
:100530004184C9480188C548818400BF418BC1837B
:10054000818B018400BF00BFC4480188BF4841833C
:10055000C2484188BD48818300BFEFE300240020EA
:10056000BC49087030E0BB48007800EB8000BC4913
:1005700001EBC000407E30B9B648007800EB800047
:1005800001EBC00424E0B348007800EB8000B449DC
:1005900001EBC000407E072811D14CB1AD48007876
:1005A00000EB800001EBC000807EA17E884206DD6A
:1005B000A848007800EB8000A94901EBC004A548D9
:1005C0000078401CA3490870A24800781E28CADBA6
:1005D00000BF4CB99C48008D401C81B29A480185EF
:1005E000A0A001F06BF814E4A74804600320A076F3
:1005F00020760020A0750420E0750020E076934866
:10060000808CA0809148408CE08000BF8F48408B58
:1006100020808E48808B608000BF012060769B48E0
:10062000007820739948417861738178A173C1780B
:10063000E17301202082854890F82910E17290F83A
:100640002810A17290F82710617290F8260020728D
:100650000120FFF775FA7D4890F82E0000F0F000B9
:1006600050285ADD00207B4908704AE0794800781C
:1006700036307649085C864908700846007800B92B
:100680004AE083480078012805D172480078401C70
:100690007049087035E07E480078022820D16D4806
:1006A000007837306949085C042819D16948007816
:1006B0003930095C674800783830644A105C41EA98
:1006C0000020654908800846008840F2CA718842C7
:1006D00001DD084601E0604800886082A0821BE0DE
:1006E0005C48007837305949085C00B914E0594833
:1006F000007837305549085C56490978084455490F
:100700000870524890F82E000521C1EB2010514985
:100710000978B1EB800FA9DB00BF00BF10214B4867
:1007200080F82F1000BF494890F82F0040F00201D8
:10073000464880F82F10022180F83610042180F8F6
:100740003710072180F83810CA2180F839102C2082
:100750003F49088060213D4880F82E1031E34A4827
:10076000046000204B490870384890F82F0000F0D2
:10077000040050B10020607647A000F09FFF2020C9
:100780004449087000F073FFA4E3304890F82E004D
:10079000001180002F4908702D4800880978401A00
:1007A00014382B490880607E00F00F00022806D123
:1007B000264890F82F0000F03F00122822D024484D
:1007C0000088002805DC214890F82F0000F0030085
:1007D000C0B11E4890F82600217A884211D11B48EA
:1007E00090F82710607A81420BD1184890F82810B1
:1007F000A07A814205D1154890F82910E07A81420B
:1008000000D0D0E2114890F82F0000F01000C8B1DD
:10081000208AB8B1218A04F10C00FEF75CFF0B4876
:1008200090F82A002649097888420BD1074890F8A9
:100830002B002349497888427DD1044890F82C0048
:100840001F493FE077E0000000580020904800205A
:100850003C010020580100205A0100201C0100200A
:10086000945000207463703A20666F756E64206E39
:100870006F20756E7573656420636F6E6E6563744B
:10088000696F6E732E000000440100204E010020AD
:1008900059010020400100207463703A20676F7492
:1008A0002072657365742C2061626F7274696E6763
:1008B00020636F6E6E656374696F6E2E00000000BA
:1008C000540100208978884235D1FA4890F82D00EB
:1008D000F949C97888422ED1F74800782073F64844
:1008E000417861738178A173C178E173E07ED8B9F2
:1008F000217EA27E891A48B2A17DA0EBE10148B217
:10090000A17D0144A175002801DA414248B2E17D90
:10091000A0EBA10148B2E17D0144E175E17DA27D3A
:1009200001EBE201217600BF0120E4490870207E3E
:10093000A07600202082607E00F00F0009286AD295
:10094000DFE800F0690525BFF4F3F2F1F000DB48C1
:10095000007800F00100C8B1032060764020D7493C
:10096000087000202082D6480088002808DD08464C
:10097000007840F002000870D1480088FFF7E0F8E6
:100980000020D049088000F072FE22E1A2E2CB48AC
:10099000007800F00100E8B3C64890F82F0000F09E
:1009A0003F00122836D1C34890F82E0000F0F00026
:1009B00050285DDD0020C44908704DE0C248007831
:1009C0003630BC49085CC14908700846007800B957
:1009D0004DE0BE480078012805D1BB480078401C96
:1009E000B949087038E0B9480078022823D1B648E0
:1009F00000783730AF49085C04281CD1B248007831
:100A00003930095CB04800783830AA4A105C41EAB5
:100A1000002001E04BE0C4E1AD49088008460088B1
:100A200040F2CA71884201DD084601E0A84800880A
:100A30006082A0821BE0A448007837309D49085CA2
:100A400000B914E0A048007837309A49085C9E4904
:100A5000097808449C490870964890F82E000521B2
:100A6000C1EB201098490978B1EB800FA6DB00BFDD
:100A7000032060768F4890F8260020728D4890F809
:100A80002710617290F82810A17290F82910E17275
:100A90000120FFF755F84220884908700020208285
:100AA000874908808749088000F0E1FD91E0202017
:100AB0008249087000F0DBFD00208649096848760D
:100AC00075E47C4890F82F0000F0010078B3607E58
:100AD00000F0100058BB208A08B1FBE1CCE1784956
:100AE0000988491C88B2FFF72BF87448007840F059
:100AF00010007249087072480088002804DD08461A
:100B0000007840F00200087000F0B1FD0120208262
:100B1000082060760020E07600BF1121654880F84B
:100B20002F1045E1B9E031E131E10EE1D8E0FFE716
:100B3000604890F82F0000F02000B8B15D4890F8B0
:100B4000351090F8340041EA0020634909680844F0
:100B500061490860574890F8351090F8340041EA30
:100B6000002057490988081A5549088054480088C8
:100B700000280DDD607E00F0100048B94F48007875
:100B800040F002004D4908704D480088FEF7D8FF3C
:100B9000484890F8311090F8300001EB00204C49A3
:100BA0000880A08A0988884202DB4948008810B979
:100BB000A08A474908804648008860823F480078FC
:100BC00000F00300F0B300203E49088000F04FFD24
:100BD00000BF3A48007800F0200040B100203949B9
:100BE000088060761421334880F82F10E0E0334805
:100BF000007800F0100068B1002032490880012020
:100C00002082042060760020E0761121294880F8B7
:100C10002F10CDE02B480088002819DD27480078E8
:100C200000F0010008B100202082208A68B9608AA3
:100C300024490988884202DA608A224908802148CA
:100C4000008800E028E0208202E0208A1D49088018
:100C50000020E07600BF214800681F49086019485D
:100C6000008800280BDD208A002808DD208A283033
:100C70001349088018210F4880F82F109CE00F4876
:100C8000007800F0020038B128200D4908801021BA
:100C9000084880F82F108FE01CE10848007800F029
:100CA000010030B10020607610200449087000F087
:100CB000DEFC76E090480020540100204001002036
:100CC0003C0100203E010020580100205901002075
:100CD0005A01002044010020340100203801002086
:100CE00089480088002803DD87480088FEF728FF30
:100CF000864890F82F0000F00100A8B184480078E1
:100D000000F0010028B1072060760020A076208244
:100D100001E0062060760120FEF712FF10207C49DA
:100D2000087000F0A4FC3EE07948007800F0010073
:100D300028B10520607600202082CBE083E0724855
:100D40000088002800DD2EE0C4E06F4800880028FD
:100D500003DD6D480088FEF7F3FE6C4890F82F0025
:100D600000F0010060B1072060760020A07601202D
:100D7000FEF7E6FE10206649087000F078FC12E0ED
:100D800061480088002800DD0DE0A3E00BE060482A
:100D9000007800F0010018B1072060760020A076EE
:100DA00000BF00BF96E01021584880F82F1000BF08
:100DB00028205549088000BF5021544880F82E1043
:100DC00000BF217A514880F82A10617A80F82B10F0
:100DD000A17A80F82C10E17A80F82D10217B80F820
:100DE0002610617B80F82710A17B80F82810E17B1A
:100DF00080F829100621C175A1884184E188818489
:100E000000BF4448018841484183424841883F48E7
:100E1000818300BF00BF2188C1836188018400BF36
:100E2000607E00F0100030B10021384880F83110A9
:100E300080F8301006E00721344880F83010CA21CD
:100E400080F8311000BF4021304881752E4800885D
:100E500001122E4801742C4801782C48417400215D
:100E600080F8351080F834104186FEF7CFFCC0437F
:100E700081B22648418600BF45202449887300215D
:100E80002248C1734175017523480088401C2249DE
:100E900008800846008801121C4881741E480178A9
:100EA0001A48C17400210183FEF77FFCC04381B260
:100EB000164801831948C08B401C81B21748C18372
:100EC00000BF16488088401C1449888000201049C3
:100ED00008707CBD00200C4908800D49087000BFD7
:100EE000F7E770B504460D46002D0CDD0C490D806A
:100EF0000C480068844206D008460288214609480A
:100F000000680FF078F870BD3C0100209048002088
:100F1000400100201C0100204C010020005800204E
:100F20003E010020380100200020F34908700DE048
:100F3000F148007800EB4000F04901EB800000210F
:100F40000160ED480078401CEB490870EA480078E1
:100F50000828EDDB7047EA490978491CE84A117016
:100F60000021E54A117017E0E349097801EB4101DE
:100F7000E24A02EB810001884288114339B1817A4B
:100F8000DF4A1278511A782901DB00210160DA4921
:100F90000978491CD84A1170D74909780829E3DB38
:100FA000704710B502460023D34C23701FE0D24B8C
:100FB0001B7803EB4303D14C04EB830003888BB114
:100FC00043887BB113880488A3420BD1538844889B
:100FD000A34207D10B6843608B880381C84B1B7801
:100FE000837210BDC44B1B785B1CC34C2370C24B77
:100FF0001B78082BDBDB0023BF4C237010E0BE4BBB
:101000001B7803EB4303BD4C04EB8300038813B947
:10101000438803B908E0B84B1B785B1CB64C2370BF
:10102000B54B1B78082BEADB00BFB34B1B78082BB2
:1010300034D10023B34C2370B34C2370AE4C2370D7
:101040001DE0AD4B1B7803EB4303AC4C04EB83007A
:10105000837AAB4C2478E31AAA4C2478A34209DDA6
:10106000837AA74C2478E31AA64C2370A24B1B78F2
:10107000A54C2370A04B1B785B1C9F4C23709E4B90
:101080001B78082BDDDBA04B1B789B4C2370234681
:101090001B7803EB4303994C04EB83001368036054
:1010A0000B6843608B880381954B1B78837200BF6C
:1010B00097E710B5954800882A2803D20020934965
:1010C000088010BD0020914908809148808AB0F5C1
:1010D000807F03D0B0F5007F54D141E08C48C08CB4
:1010E0008C49098888423AD18948008D89494988C4
:1010F000884234D186491631881DFFF752FF4FF4DC
:101100000070834988820846D1F816200262498B14
:10111000818481490A68C0F81620898841837E4904
:101120000A68C0F806208988418101460A6A02607F
:10113000898C8180808B7649C8840846C18B018563
:101140007448008872498883724841887048C18316
:101150004FF4C1606E4988812A206C49088011E0F3
:101160006B48C08C6B49098888420AD16848008D59
:1011700068494988884204D165491631881DFFF7BE
:1011800010FF00BF00BF00BF9BE710B56048C08BD9
:101190006249098888420CD15D48008C5F494988C2
:1011A000884206D15A485E490A680260898881806F
:1011B00091E05748C08B5B49098808405549098828
:1011C000584A1288114088420BD15148008C554929
:1011D000498808404F494988524A528811408842FC
:1011E00008D000BF50480088504908804E484088C9
:1011F000488008E000BF4648C08B4C4908804448FE
:10120000008C488000BF00203B49087016E03A4837
:10121000007800EB4000394901EB80044348008826
:101220002188884205D1414840886188884200D1A0
:1012300008E031480078401C2F4908702E4800789B
:101240000828E4DB00BF2C48007808283ED1FF22A4
:1012500006212F480EF046FF2D48002101628184AF
:101260002D490A68C0F80620898841812A490A6800
:10127000C0F816208988418300BF2C480088244983
:10128000C8842A4841882248018500BF00BF214800
:1012900000881F4988831F4841881D48C18300BFBB
:1012A0004FF480701A498882C8810820088206207D
:1012B00088740420C8744FF4C160888101F136003D
:1012C0001B4908602A201149088010BD1048616838
:1012D0000160218981800E480F490A68C0F8062004
:1012E0008988418108200A498881084800880E3091
:1012F0000649088000BFE8E760010020525800203E
:101300006201002063010020610100203C010020F7
:10131000904800201C0100202C0100203E280208DB
:101320003828020824010020200100205C01002050
:10133000340100200148006870470000640000206C
:101340007CB50025A948FCF793FB0546002405E081
:10135000A648005DA6490855601CC4B2062CF7DB00
:1013600040F276411420FCF764FBFEF759FA9F48DF
:10137000143890F82F0000287ED100BF9B48143805
:10138000C07E9A491439897E40EA012001029748BB
:101390001438C07E954A143A927E40EA022041EA0F
:1013A000202080B2ADF8000090481438417F007FC3
:1013B00041EA002001028D481438427F007F42EA52
:1013C000002041EA202080B2ADF8020000BF00BF3B
:1013D000BDF8000087490880BDF80200488000BFC2
:1013E00000BF8248143890F824008049143991F8DD
:1013F000231040EA012001027C48143890F82400B0
:101400007A4A143A92F8232040EA022041EA202046
:1014100080B2ADF800007548143890F8261090F8A6
:10142000250041EA002001027048143890F8262077
:1014300090F8250042EA002041EA202080B2ADF871
:10144000020000BF00BFBDF800006B490880BDF876
:101450000200488000BF00BF6448143890F82000A4
:1014600062491439C97F40EA012001025F481438FB
:1014700090F820005D4A00E0A0E0143AD27F40EAF4
:10148000022041EA202080B2ADF80000574814380D
:1014900090F8221090F8210041EA00200102534800
:1014A000143890F8222090F8210042EA002041EA06
:1014B000202080B2ADF8020000BF00BFBDF80000E0
:1014C0004E490880BDF80200488000BF47481438E4
:1014D000807E8DF8040045481438C07E8DF80500E4
:1014E00042481438007F8DF8060040481438407F89
:1014F0008DF807009DF804003C491439C97FC1F1FB
:10150000FF0108438DF804009DF8050037491439A0
:1015100091F82010C1F1FF0108438DF805009DF8F6
:1015200006003249143991F82110C1F1FF01084336
:101530008DF806009DF807002C49143991F8221007
:10154000C1F1FF0108438DF8070000BF9DF80500B9
:101550009DF8041040EA012000029DF805109DF856
:10156000042041EA022140EA2120254908809DF813
:1015700007009DF8061040EA012000029DF80710C0
:101580009DF8062041EA022140EA21201C494880BA
:1015900000BF0120FEF759F81449143991F82810BA
:1015A0000902124A143A128D41EA222188B2FEF74A
:1015B000ACFA00F015FE04F030FE05E006210B4801
:1015C00000F0D7FA00F0FCFA28467CBD10B50D49B2
:1015D00040F2EE50FCF744FB80B210BD10B5094953
:1015E00009480088FCF700FB10BD00006460002083
:1015F0002C0100201C0100202001002024010020DB
:1016000028010020904800203C0100202DE9F041F5
:1016100007460E46002525E005EB8500284901EB2D
:10162000C0040422394620460EF076FC68B9E088F2
:10163000B0420AD1607E10B1607E072803D14FF01E
:10164000FF30BDE8F08168B2FBE70422394620464E
:101650000EF062FC20B9A088B04201D168B2F0E778
:10166000681CC5B21E2DD7DB4FF0FF30E9E710B57F
:101670004FF0FF3400BF134890F8280000021149D2
:10168000098D40EA212080B20F4909688988884283
:1016900013D100F0C6FC0C48006881880A48006835
:1016A000FFF7B4FF0446002C07DB0848007800F081
:1016B000020010B114200649085510BD7047000003
:1016C0009450002050600020440100204001002080
:1016D00034580020352200F8012B012200F8012B9C
:1016E00000F8011B70470146362001F8010B042069
:1016F00001F8010BFE48C0690860081D70470146EB
:10170000322001F8010B042001F8010BF848406A6F
:101710000860081D7047372100F8011B032100F8FD
:10172000011B012100F8011B032100F8011B062108
:1017300000F8011B7047FF2100F8011B704710B52E
:101740000446012020706070E948007EA0700020EF
:10175000E070E8480068606000202081802060819F
:10176000E5480068E060002020616061A061E04819
:101770008269416904F11C000EF03DFCDC4A92696B
:10178000C2F11001DA4A936904F11C0298180EF0B4
:10179000B1FC402104F12C000EF0ACFC802104F1DE
:1017A0006C000EF0A7FCD5490968C4F8EC1010BD18
:1017B00070B5D34805682846FFF7C1FF012105F140
:1017C000F000FFF787FF04462046FFF7A4FF04461A
:1017D0002046FFF7B0FF0446C9480068211AC848F0
:1017E0000068FFF77EFB70BD70B5C54805682846E8
:1017F000FFF7A5FF032105F1F000FFF76BFF04469B
:101800002046FFF770FF04462046FFF778FF0446A6
:101810002046FFF790FF0446B9480068211AB848EF
:101820000068FFF75EFB70BD30B50246531800201C
:1018300031E01478332C24D006DC012C0BD0032C9F
:101840000ED0062C23D110E0352C13D0362C13D01B
:10185000FF2C1CD11AE0A64CD2F80250A56216E06B
:10186000A34CD2F80250256311E0A14CD2F80250EB
:10187000E5620CE090780AE09D4CD2F80250E561F8
:1018800005E09B4CD2F80250256200E030BD00BF5D
:101890005478A41C22449A42CBD300BFF6E710B57B
:1018A000974804682078022817D104229149201D06
:1018B0000EF032FB88B98E488269416904F11C0040
:1018C0000EF02AFB48B98A48216941628D48018897
:1018D00004F1F000FFF7A8FF10BD0020FCE7002096
:1018E0008349496888808848817EC07E01EB00205A
:1018F0007F4988848448017F407F01EB002081B2CA
:101900007B48C1848048C17F90F8200001EB002013
:10191000774908857C4890F8211090F8220001EB67
:10192000002081B272484185774890F8231090F8E2
:10193000240001EB00206E498885734890F825103B
:1019400090F8260001EB002081B26948C1856E48FD
:1019500090F8231090F8240001EB002064490886D9
:10196000694890F8251090F8260001EB002081B21C
:101970005F484186704710B5012400BF5C4800886D
:10198000B0F5BE7F69D005DC58B1A0F25310002835
:101990006FD11AE0B0F5D77F6CD0B0F5DA7FF7D110
:1019A000DCE00120524988704FF47A70088200BF51
:1019B000FFF7FEFE4E48018A0830FDF769FE00BFC2
:1019C00040F253104A49088000BF5048007800F0A8
:1019D000020030B946480830FDF76DFE08B9002016
:1019E00010BD00BF4948007800F0020030B1FFF799
:1019F00056FF022802D13E49887017E03C48008A11
:101A00004EF66021884207DA3948008A4FF6FF71A6
:101A100001EA4000364908823548008AB0F57A5F0D
:101A200000DB54E0324880780228C1D100BF4FF477
:101A30007A702F49088200203449087000BF00BF27
:101A4000FFF7D2FE2A48018A0830FDF721FE00BFC9
:101A50004FF4BE702649088000BF2C48007800F083
:101A6000020040B922480830FDF725FE18B90020D1
:101A7000B6E778E062E000BF2448007800F002009A
:101A800038B1FFF70CFF052803D1032018498870EF
:101A90001BE01748008A42F21071884206DC1448A5
:101AA000008A00F57A701249088204E000BF002025
:101AB0000F49088094E70E48008AB0F5FA5F00DB12
:101AC00005E00B4880780328BAD100BF02E0FFF799
:101AD00006FF00BF064800F071FD054890F822009F
:101AE00002020348408C42EA1022014810E0000044
:101AF000B4580020422802081C0100204628020891
:101B0000340100203C0100205060002040010020F2
:101B100090F820000002354B1B8C40EA132002EBAA
:101B20000040322200FB02F130480830FDF7B0FDE2
:101B300000BF4FF4D7702D49088000BF2B480830F4
:101B4000FDF7B9FD08B900204AE700BF77E700BFFD
:101B500000244FF4DA702549088000BF0CB9032037
:101B60003EE700BFF3E700BF0020204908800220C5
:101B700036E738B504460D461C48446185610020AF
:101B80001A49887000BF4FF6FF70ADF80000ADF83D
:101B9000020000BF4FF486416846FDF724FF134959
:101BA00048600846406818B14FF48840496888800A
:101BB00000200E49088038BD10B5FFF7DCFE10BDCF
:101BC00008B50A48807878B900BF0020ADF8000059
:101BD000ADF8020000BF00BFBDF800000449088056
:101BE000BDF80200488000BF08BD0000B4580020C6
:101BF0001C010020014600BF11F8012B02E0491C26
:101C0000501EC2B2002AFADC08780028F4D1481C21
:101C100070472DE9F0410020CB49087071E0CA48B7
:101C20000078C0EBC00000EB4000C84901EB400465
:101C30002078012802D0207802285CD12078022860
:101C400011D16078401EC0B2607058B9A078401CB5
:101C5000C0B2A070082802D1042020704CE0A07807
:101C6000607006E048E002202070012060700020D3
:101C7000A070B7480768002038607860B860B24844
:101C80000078FDF780FD38800120B8700002B88030
:101C9000AF48006800F10C05661D761E00BF761C7B
:101CA000A8466D1C0020AB49087008E03078287009
:101CB0006D1CA8480078401CA6490870761C307836
:101CC0002E2802D030780028F0D1A248007888F879
:101CD000000030780028E2D19F480168296000792F
:101CE0002871681D9A4A1278801AC1B29848006813
:101CF000FFF7F7F809E000BF93480078401C9249CD
:101D0000087091480078042889DB00BFBDE8F081A5
:101D10002DE9F0418E4807683888FDF734FD8F497A
:101D2000087008460078C0EBC00000EB400087490F
:101D300001EB40068948007804284DDA3078022803
:101D40004AD103203070F87800F00F0030713079FC
:101D500018B104203070BDE8F081B888FDF713FD9C
:101D60007F490870084600780870F888FDF70BFD79
:101D70007C490870764800680C30FFF73BFF041D73
:101D800026E0207800F0C00008B1A41C03E0204643
:101D9000FFF730FF044625462888B0F5807F0CD138
:101DA0006888B0F5807F08D12889B0F5806F04D1AC
:101DB0006889F084A9893185CDE72889FDF7E3FC9E
:101DC00004F10A01441867480078401E654908700C
:101DD000644800780028D4DC00BFBCE710B5624836
:101DE0000068C088B0F5545F0DD16048007800F0FD
:101DF000080008B1FFF70DFF5C48007800F0020012
:101E000008B1FFF785FF10BD70B5054600205849A1
:101E10000870584908705849087022E05648007800
:101E2000C0EBC00000EB4000484901EB40042078C3
:101E300000B91AE0E07851490978081A4D49097843
:101E4000884209DDE0784D490978081A4949087047
:101E5000494800784649087047480078401C464980
:101E60000870454800780428D8DB00BF4248007855
:101E700004280CD13E4800783F4908700846007895
:101E8000C0EBC00000EB4000304901EB40042946A4
:101E9000601D0EF06DF80120207038480078E07069
:101EA00036480078401C3549087070BD70B505464D
:101EB00000203349087018E031480078C0EBC000BA
:101EC00000EB4000214901EB40042078032807D1B2
:101ED000611D28460EF082F910B904F1260070BD8C
:101EE00027480078401C26490870254800780428B7
:101EF000E2DB0020F3E72348006808B900207047C0
:101F000020480068FBE71F49096819B100211D4AF4
:101F100012689180704700201B4908700EE0032072
:101F200019490978C1EBC10101EB4101074A02F8E7
:101F3000110015480078401C1349087012480078B9
:101F40000428ECDB704770476C010020E858002043
:101F5000340100206D0100206E0100207501002079
:101F6000730100207401002048010020400100207E
:101F70007801002077010020760100206401002014
:101F800079010020680100207A01002010B56C481A
:101F9000006800F11C04A068002803DDD4E90101F9
:101FA000FEF79FFF10BD10B56548006800F11C04E6
:101FB0000020A06063A0FFF781FB10BD10B5604852
:101FC000006800F11C046448007840F08000624919
:101FD000087062A0FFF772FB00202070A06010BDA7
:101FE00010B55D48007820F080005B49087061A062
:101FF000FFF764FB10BD10B55748007820F0800053
:102000005549087061A0FFF759FB10BD10B5524843
:10201000007820F080005049087062A0FFF74EFB66
:1020200010BD70B500254648006800F11C046348E7
:10203000007800F0200008B1FFF7E8FF5F48007863
:1020400000F0800008B1FFF7D6FF5C48007800F090
:10205000100008B1FFF7C4FF5848007800F04000B6
:1020600008B1FFF7ABFF5548007800F0010008B158
:10207000FFF799FF5148007800F0020000283BD09C
:102080004F4802884F4801684F480DF0B4FF4E4852
:102090000078EE281AD14C484078102816D14A48CA
:1020A000807898B94848C07880B94748007968B9BD
:1020B0004548407950B94448807938B94248C07998
:1020C00020B9012501204149087015E03E4880797A
:1020D0003F490979884203D03B488079FF280BD1DA
:1020E00002203C49087001253749012001F0CDFB51
:1020F0003549012000F05DFD3048007800F0040013
:1021000098B92E48007800F0020070B92B4800788A
:1021100000F0010048B92948007800F0400020B9DB
:102120002648007800F0080040B1012D04D12A486B
:1021300060602A480088A060FFF728FF70BD00009B
:10214000440100207463705F73657276657220616C
:10215000636B6564210D0A007C0100207463705F6D
:1021600073657276657220636F6E6E656374656405
:10217000210D0A007463705F736572766572206367
:102180006C6F736564210D0A000000007463705F5A
:102190007365727665722074696D656F7574210D53
:1021A0000A0000007463705F736572766572206167
:1021B000626F72746564210D0A0000004001002006
:1021C0003C01002034010020905900200000002034
:1021D000506000205C000020BC5A00207E010020DE
:1021E00010B54DF20420FDF790FC4DF20420FE499D
:1021F000888010BD10B504463C21FC480DF07AFFE4
:102200001CB96520F949087004E0012C02D167204F
:10221000F64908700020F5494870F54800780871C3
:10222000F34840788871F24880780872F048C078A6
:102230008872EF48807B0873ED4800798873EC481A
:10224000807E0874EA48C07E8874E948007F08757B
:10225000E748407F8875E64890F828000876E4480B
:10226000008D00124876002088764820C87600202D
:102270000877DF48C07B487700208877C87781F8E7
:10228000200081F82100DB480088000A81F8220044
:10229000D848007881F82300D748007881F82400D6
:1022A0001422D649D14825300DF0A5FED14800684A
:1022B000000ECE4981F83900CE480068000C81F844
:1022C0003A00002081F83B003C21C848FEF709FE97
:1022D0000120CB49087010BD70B50024C9480078B2
:1022E00000F00200002842D0C74806783246C748AE
:1022F0000168C7480DF07FFEC5480078642837D1D3
:102300000120BF49087000BF24E0A000401CC04964
:10231000085CB749897E88421AD1A000801CBC495C
:10232000095CB348C07E814212D1A000C01CB849EC
:10233000095CAF48007F81420AD1A000001DB4496A
:10234000095CAB48407F814202D10020AC49087053
:10235000601CC4B2F11706EB9171B4EBA10FD4DB92
:10236000A74800780028BED00020FFF743FFF8E020
:10237000A74800786628FAD1A54840789C49897E0C
:102380008842F4D1A24881789948C07E8142EED13A
:102390009F48C1789648007F8142E8D19C480179E6
:1023A0009348407F8142E2D19948407C9049097826
:1023B000884211D19648807C8D49497888420BD15A
:1023C0009348C07C8A498978884205D19048007D2D
:1023D0008749C97888420FD08D48407C0028C6D1F3
:1023E0008B48807C0028C2D18948C07C0028BED19F
:1023F0008748007D0028BAD105240120FFF7FAFEA6
:1024000000207B4988772146641C8148405C7849DC
:1024100088762146641C7E48415C7548C176214619
:10242000641C7B48415C724801772146641C7848F3
:10243000415C6F484177807E6D4981F82B000846EA
:10244000C17E80F82C10017F80F82D10417F80F82C
:102450002E102146641C6E48405C6549C8772046B2
:10246000611CCCB26A49095C614880F820102046A2
:10247000611CCCB26649095C5D4880F82110204699
:10248000611CCCB26249095C594880F82210C07FB7
:10249000574981F83000084690F8201080F8311034
:1024A00090F8211080F8321090F8221080F8331044
:1024B0002046611CCCB25649085C4D4981F8230086
:1024C0002046611CCCB25249095C494880F824106E
:1024D0002046611CCCB24E49095C454880F8251065
:1024E0002046611CCCB24A49095C414880F826105C
:1024F00090F823003E4981F83400084690F82410F3
:1025000080F8351090F8251080F8361090F82610D5
:1025100080F8371001203F4908703548807E00B3AD
:102520003348C07EE8B13248407FD0B1002516E084
:102530002F4A1A32515D05F12F00FAF7ABFD2C4AF4
:102540001F32515D05F13300FAF7A4FD284A23320A
:10255000515D05F13700FAF79DFD681CC5B2042DE9
:10256000E6DB70BD10B5224890F83C00000220491F
:10257000898F40EA212084B22748006880884DF284
:102580000421884202D1FFF7A7FE06E02248006836
:102590008088A04201D103F063FE1F480068C08814
:1025A000B0F5545F05D0B0F5864F05D1FFF704FBB9
:1025B00002E0FFF713FC00BF00BF10BD38B50446B2
:1025C00000BFA08C15490880E08C488000BF00BF88
:1025D000208D13490880608D488000BF00BF208E89
:1025E00010490880608E1FE080550020E85B0020C5
:1025F00050600020040000208E010020C0620020F6
:1026000080010020400100203C0100203401002016
:10261000245C002082010020480100201C010020D1
:102620002401002020010020488000BF04F12C007C
:10263000FFF769FCFFF7D4FDB14991F828100902B2
:10264000AF4A128D41EA222188B2FDF75EFA0422D8
:10265000AC49AB481A300DF05FFC002846D0A949C0
:102660000888FDF790F8001288B9A6490888FDF798
:102670008AF8C0B258B9A3494888FDF784F8001217
:1026800028B9A0494888FDF77EF8C0B270B39D49CB
:102690000888FDF778F800129949887699490888E2
:1026A000FDF771F8C1B29648C17696494888FDF7A2
:1026B0006AF801129248017792494888FDF763F859
:1026C000C1B28F484177817E2F20FAF7E3FC8C4816
:1026D000C17E3020FAF7DEFC8948017F3120FAF70D
:1026E000D9FC8748417F3220FAF7D4FC042286497E
:1026F00083481F300DF010FC00284CD08249088818
:10270000FDF741F8001288B97F490888FDF73BF8CA
:10271000C0B258B97C494888FDF735F8001228B98D
:1027200079494888FDF72FF8C0B2A0B376490888E8
:10273000FDF729F800127249C87773490888FDF738
:1027400022F8C1B26E4880F820106F494888FDF722
:102750001AF801126A4880F821106B494888FDF781
:1027600012F8C1B2664880F82210C17F3320FAF710
:1027700091FC634890F820103420FAF78BFC6048F5
:1027800090F821103520FAF785FC5D4890F822106A
:102790003620FAF77FFC04225C49594823300DF0BB
:1027A000BBFB00284ED059490888FCF7ECFF00120B
:1027B00088B956490888FCF7E6FFC0B258B95349B2
:1027C0004888FCF7E0FF001228B950494888FCF718
:1027D000DAFFC0B2B0B34D490888FCF7D4FF00124D
:1027E000474981F8230049490888FCF7CCFFC1B26A
:1027F000434880F8241045494888FCF7C4FF01127B
:102800003F4880F8251041494888FCF7BCFFC1B219
:102810003B4880F8261090F823103720FAF73AFC4E
:10282000374890F824103820FAF734FC344890F8F0
:1028300025103920FAF72EFC314890F826103A205E
:10284000FAF728FC2E48807E8DF800002C48C07EC8
:102850008DF801002A48007F8DF802002848407F4B
:102860008DF803009DF800002549C97FC1F1FF01E3
:1028700008438DF800009DF80100214991F82010CF
:10288000C1F1FF0108438DF801009DF802001C49C9
:1028900091F82110C1F1FF0108438DF802009DF865
:1028A0000300174991F82210C1F1FF0108438DF888
:1028B000030000BF9DF801009DF8001040EA0120D0
:1028C00000029DF801109DF8002041EA022140EA33
:1028D00021200F4908809DF803009DF8021040EA6E
:1028E000012000029DF803109DF8022041EA022118
:1028F00040EA21200649488000BF03F08EFC38BD25
:10290000506000201C010020240100202001002034
:10291000280100200020FE490860FE490870FE4999
:102920000870704770B540F22551FC48F8F7CAFDB1
:10293000012878D10220FA490870FA48807C0328DF
:1029400073D1F4480078FA280BDAF448F8F73AFD26
:10295000C1B2F0480578681CEE4A1070F248415543
:1029600001E0FFF7D7FFEB480078012807D1FA20F4
:10297000EE490870EE480078EE490870A4E0E5489A
:102980000078032807D1E84840781928F6D10620B6
:10299000E649087098E0DF480078042813D1E2483F
:1029A000C078E149897800EB01200A28E6D1DE48A9
:1029B00040780628E2D10C20DC490870DC48007819
:1029C000DC49087080E0D348007807281ED1D6483B
:1029D0004078032803D0D4484078062803D1082043
:1029E000D249087070E0D048407810280AD1CE480B
:1029F00080790930CD490870CB4880790830CD49BD
:102A0000087061E0FA20C94908705DE0C1480078AB
:102A1000C6490978884257D10020C6490870052068
:102A2000BD49087050E013E0FFE7BE48807CE8BB7A
:102A300040F22551B948F8F745FD012844D1B7487F
:102A4000F8F7C0FCC4B22146BB4807F074F93BE07C
:102A500040F22771B148F8F735FD012834D1022042
:102A6000B6490870AF48807C032802D0AD48807C0E
:102A7000E0B9B34802880088401CB14B1880B148C7
:102A8000815CA648F8F79AFC07F005FAAC48008884
:102A9000AD490988884217DB00BF40219F48F8F7FD
:102AA000FBFC0028F9D040219C4800E00CE0F8F73E
:102AB00000FD002240F227719848F8F71EFC002024
:102AC0009F490880FFF726FF70BD012090490860EC
:102AD000704770B504460D4640219048F8F7E9FC70
:102AE00021468E48F8F76AFC15B1204602F0E2F85C
:102AF00070BD70B5044694480480012240F22771ED
:102B00008648F8F7FAFB9148808D642832D18548D1
:102B10008068B0F5165F05D104F10A0188B2FCF7B0
:102B200094FD25E07F488068B0F5964F08D1254692
:102B300004EBD57149100A3188B2FCF786FD17E025
:102B400078488068B0F5164F09D12546E11704EBA7
:102B5000917189100A3188B2FCF777FD08E02546AB
:102B6000E11704EB5171C9100A3188B2FCF76DFD11
:102B70007648048670BD00B5FFF7CCFE03206C4993
:102B80000870084600786B49087000BD012080F38A
:102B9000138800BF00BF6E48006800F4E0606D4914
:102BA0000843001D6A490860BFF34F8F00BF00BF94
:102BB000FEE72DE9F04782460D46BAF1000F02D03C
:102BC000BAF1040F01D1002400E00624E01C295CC6
:102BD000A01C285C01EB002086B2601C285C102839
:102BE0007ED1282E3CD14F4890F82A00012836D1BA
:102BF000A01D285C0C28FAD104F10800285C494982
:102C0000087504F10A00295C4648417504F10C007E
:102C1000295C4448817504F10E00295C4148C17566
:102C200004F11000295C3F48017604F11200295C90
:102C30003C484176002709E03A4A1432D15D07F159
:102C4000280290B2FAF726FA781C87B2062FF3DB37
:102C50000120414908700020324981F82A001BE117
:102C600040F2CB2086421DDB40F2D520864219DCA3
:102C7000A01D285C1428F2DC00270EE0E21D3A4477
:102C8000A95C07F2BA2290B2FAF704FAE01D3844C0
:102C9000285C3249C855781C87B2A01D285CB84210
:102CA000ECDCDCE742F6D04086427CDB42F6AF70DB
:102CB000864278DCA6F53050D0381721B0FBF1F20F
:102CC00001FB120098B9A6F53050D038B0FBF1F0F6
:102CD00087B2E21DA918C7EBC70202EB071200E09A
:102CE000AFE01F4B03EB42002E220DF084F903F0FE
:102CF000C7F901201B494870C7EBC70000EB07105C
:102D0000174901EB400090F82D000F2836D02BE03A
:102D1000A0012142860100208A01002000380140E4
:102D20005A00002050600020505D002087010020E4
:102D30008901002088010020ACA900205900002052
:102D400092010020505E00208C010020E0670020EE
:102D50000CED00E00000FA0582010020C0620020B6
:102D60005F6F0020E2010020C7EBC70000EB0710F7
:102D700001EB400090F82D00192892D1C7EBC70055
:102D800000EB0710F74901EB4000D0F81E0018B91E
:102D90000021F54840F837100B2F7DDAF8B2FBF729
:102DA000ECFB5CE7FFE743F29020864222DB43F234
:102DB000974086421EDC0120EC498870A6F54850F9
:102DC00090380A21B0FBF1F201FB12000028E8D193
:102DD000A6F548509038B0FBF1F087B2E21DA91873
:102DE00007EB470202EB0712E14BD01813220DF05C
:102DF00002F934E748F2A8008642D2DB48F2B0106C
:102E00008642CEDC0120D949C870A6F50040A8381A
:102E10003521B0FBF1F201FB12000028C1D1A6F56B
:102E20000040A838B0FBF1F087B2E21DA918C7EB4B
:102E30000712C2EBC202CF4BD01869220DF0DBF8AB
:102E40000DE7601C285C0628ABD1632E77DC012ED1
:102E50002BDC601D295C0020FAF71CF9201D295C81
:102E60000120FAF717F9601D285CBF494039087046
:102E7000201D285C48700846007C40F00100087462
:102E80000846017C1120FAF705F9B7484038007C64
:102E9000002886D0002000E002E2B34940394873A0
:102EA00000211020FAF7F6F8D9E6032E29DC601D80
:102EB000295C0220FAF7EEF8201D295C0320FAF7BE
:102EC000E9F8601D285CA84940398870201D285CFD
:102ED000C8700846007C40F0020008740846017C77
:102EE0001120FAF7D7F8A0484038007C0028A7D076
:102EF00000209D494039487300211020FAF7CAF894
:102F0000ADE6062E1CD1601D285C002898D0601DFF
:102F1000285CFF2894D0601D295C0620FAF7BAF8D7
:102F2000601D285C90494039087108460079924933
:102F30000870F5F7FBF9002006F0D2F88FE673E28F
:102F4000072E14D1601D295C0720FAF7A3F8601D35
:102F5000285C8549403988730846007C40F00800A9
:102F600008740846017C1120FAF794F877E6082ED9
:102F700014D1601D295C0820FAF78CF8601D285CCC
:102F800079494039C8730846007C40F00400087451
:102F90000846017C1120FAF77DF860E60F2E76D105
:102FA000601D285C7049403908730846007B06287C
:102FB0006ED2DFE800F003182D42576E4FF4165022
:102FC000694940398860FCF78BFA601D295C15203F
:102FD000FAF760F8601D295C1320FAF75BF8062009
:102FE000664908706BE04FF496405F49403988604D
:102FF000FCF776FA601D295C1520FAF74BF8601D86
:10300000295C1320FAF746F803205C49087056E063
:103010004FF41640544940398860FCF761FA601D4E
:10302000295C1520FAF736F8601D295C1320FAF7A1
:1030300031F802205149087041E04FF461404A499B
:1030400040398860FCF74CFA601D295C1520FAF7BE
:1030500021F8601D295C1320FAF71CF8012047496C
:1030600008702CE04FF4E1303F4940398860FCF7AC
:1030700037FA601D295C1520FAF70CF8601D295CF1
:103080001320FAF707F801203C49087017E01AE00E
:1030900014E04FF49630344940398860FCF720FA48
:1030A000601D295C1520F9F7F5FF601D295C1320D0
:1030B000F9F7F0FF01203149087000BF00BF00BFE1
:1030C000FFF759FDA4E3102E05D1601D285C2649A9
:1030D000403948739CE3152E1BD1601D285C0328E2
:1030E00003D0601D285C0028ECD1601D285C1E49BF
:1030F00040398874601D295C1420F9F7CBFF1A4809
:103100004038807C0028DDD106F09EFEFFF702FCEF
:103110007EE3252E0DD1601D285C0128D2DD601DC7
:10312000285C17490870601D295C1220F9F7B2FF6E
:103130006EE3272E26D1601D295C0620F9F7AAFF31
:10314000601D285C0C490870084600780649403923
:103150000871F5F7EBF8002005F0C2FF002006F03B
:1031600073FE55E35F6F002090600020E2010020B5
:103170003F7D0020526D00208E010020890100203B
:103180008F010020162E2AD1601D295C201D285C8D
:1031900001EB0020FE490968B0EB114F16D0601D0D
:1031A000285C0104201D285C01EB0060F8490988B7
:1031B00089B20844F6490860601D295C1820F9F7B7
:1031C00069FF201D295C1920F9F764FFF5F7AEF8B7
:1031D000002005F085FF002006F036FE18E3172ECC
:1031E0002DD1EB48D0F80090601D295C201D285C93
:1031F00001EB0020E6490968B0EB114F16D06FF3E0
:103200000F09601D295C201D285C01EB002040EAAD
:103210000909DF48C0F80090601D295C1620F9F705
:1032200039FF201D295C1720F9F734FFF5F77EF8E8
:10323000002005F055FF002006F006FEE8E2262EED
:103240001AD1601D295C201D285C41EA0020D1496B
:103250008887201D295C1B20F9F71CFF601D295C55
:103260001C20F9F717FFF5F761F8002005F038FF8B
:10327000002006F0E9FDCBE2282E12DB2D2E10DC1B
:10328000A6F1280000F0FF08601D295CC148143039
:1032900000F80810621DA95C08F12800F9F7FAFE91
:1032A000B6E23D2E05D1601D285CBA4981F82F0099
:1032B000AEE23E2E0CDB412E0ADCA6F13E0000F011
:1032C000FF08601D295CB3482B3000F808109FE20E
:1032D000422E0CDB452E0ADCA6F1420000F0FF086E
:1032E000601D295CAB48303000F8081090E2462E93
:1032F0000CDB492E0ADCA6F1460000F0FF08601D39
:10330000295CA448343000F8081081E24A2E05D127
:10331000601D285C9F4981F8380079E24B2E08D166
:10332000601D295C201D285C01EB0020994948871D
:103330006EE24C2E5FD1601D285C964981F83E00FC
:10334000084690F83E00012895D1084690F82F00D5
:103350008877084690F8380081F827000846408FA3
:1033600008850846817F2E20F9F794FE894890F859
:1033700027103B20F9F78EFE8648008D01123C2075
:10338000F9F788FE834890F828103D20F9F782FE6F
:10339000002726E07F482B30C15D1138C15516301B
:1033A000C15D1138C1551530C15D1138C155A0F14D
:1033B0000902D15D07F12F0290B2F9F76BFE754A51
:1033C0001F32D15D07F1330290B2F9F763FE714A03
:1033D0002332D15D07F1370290B2F9F75BFE781C1A
:1033E00087B2042FD6DB01206B49087000206949A1
:1033F00081F83E000CE25D2E05D1601D285C654918
:1034000081F82A0004E25A2E87D1601D295C201D14
:10341000285C4FF4807202FB001060490880084667
:10342000008802F0AEFDF3E1642E4EDBA32E4CDCEF
:10343000A6F1640000F0FF0808EBD8714FEA6109BB
:10344000C9EBC90000EB0910554901EB400090F8A9
:103450002D000F2809D0C9EBC90000EB091001EBC2
:10346000400090F82D0019282ED100214948403005
:1034700040F83910024612F839104FEA890202F179
:10348000BE00F9F707FE434A403202EBC902517809
:103490004FEA890202F1BF00F9F7FCFD3D4A4032D4
:1034A00002EBC90291784FEA890202F1C000F9F7F4
:1034B000F1FD384A403202EBC902D1784FEA890265
:1034C00002F1C100F9F7E6FDA2E1B6F5827F15DB56
:1034D000B6F5927F12DA301F00F0FF08601D285CFD
:1034E00040B2C8EBC80101EB08112D4A02EB4101C3
:1034F00081F8280001202B49487089E1B6F5927FB8
:1035000034DBB6F5A27F31DAA6F5927000F0FF0841
:10351000C8EBC80000EB0810214901EB400090F80F
:10352000230000F00F00C8EBC80101EB08111C4A92
:1035300002EB410181F82300C8EBC80000EB081042
:10354000114601EB400090F82310601D285C41EA11
:10355000001040B2C8EBC80101EB081102EB4101B9
:1035600081F8230001200F49487051E1A42E21DB8E
:10357000C32E1FDCA6F1A40000F0FF08601D285C2C
:10358000C8EBC80101EB0811054A02EB41010BE051
:10359000040000205060002082010020C0010020B3
:1035A0005F6F0020E201002081F822000120FD4928
:1035B00048702DE1C42E7CDBE32E7ADCA6F1C4003A
:1035C00000F0FF08601D285C98B90020C8EBC80116
:1035D00001EB0811F44A02EB410181F82D000120B2
:1035E000C8EBC80101EB081102EB410181F828008A
:1035F0002DE0601D285C1F2814DA601D285CC8EBD4
:10360000C80101EB0811E84A02EB410181F82D00E5
:103610000020C8EBC80101EB081102EB410181F861
:10362000280014E0601D285C1E38C8EBC80101EBBF
:103630000811DD4A02EB410181F82D000120C8EBA1
:10364000C80101EB081102EB410181F828000020BC
:10365000C8EBC80101EB0811D34A02EB410181F824
:103660002B00C8EBC80101EB081102EB410181F806
:103670002C000120CB494870C8EBC80000EB0810B3
:10368000114601EB400090F82D000F2809D0C8EB3F
:10369000C80000EB081001EB400090F82D0019283D
:1036A00015D1C8EBC80000EB0810BF4901EB400082
:1036B00000E00FE0D0F81E0018B90021BB4840F828
:1036C0003810B8F10B0F02DA4046FAF756FF02F055
:1036D000D7FC9DE0E42E16DBB6F5827F13DAA6F167
:1036E000E40000F0FF08601D285C40B2C8EBC80190
:1036F00001EB0811AC4A02EB410181F827000120DF
:10370000A849487084E0B6F5A27F16DBB6F5B27F13
:1037100013DAA6F5A27000F0FF08601D285C40B225
:10372000C8EBC80101EB08119F4A02EB410181F887
:10373000290001209B4948706AE0B6F5B27F2EDB74
:10374000B6F5D27F2BDAA6F5B27000F0FF0840463E
:1037500008EBD0714910A8EB410171B9611D695C9A
:1037600008EBD8725210C2EBC20303EB02128E4B6D
:1037700003EB420282F82B100DE0611D695C08EB3F
:10378000D8725210C2EBC20303EB0212864B03EB5A
:10379000420282F82C1001208249487038E0B6F5C8
:1037A000487F22D1201D285CD0B9601D285C7F494C
:1037B0004039C8740846C07C012809D1002705E0BB
:1037C000FF213846F9F766FC781C87B2FF2FF7DD3A
:1037D000F4F77EFF00211020F9F75CFCFFF7D6F923
:1037E000611D685C03F0DCFB12E0B6F5487F0FDD7D
:1037F00040F2513086420BDC601D295C201D285CA4
:1038000001EB002081B2A6F54870694A22F8101039
:1038100066484038407B7F2801D1FFF7B7F96348FD
:103820004038407B8E282ED100271AE0102F16D06A
:10383000AFB1012F13D0062F11D0152F0FD0022FAB
:103840000DD0032F0BD03D2F01DC282F07DA082FD6
:1038500005D0072F03D0FF213846F9F71BFC781C51
:1038600087B2FF2FE2DBF4F733FF00211020F9F7D6
:1038700011FC00204D494039087400211120F9F74E
:1038800009FCFFF783F9BDE8F0872DE9F34FD1B0CC
:103890008B46002700260024A146519810B151986C
:1038A000042802D14FF000090FE04FF006094FF055
:1038B000000A07E0002006A901F80A000AF1010049
:1038C00000F0FF0ABAF1060FF4DB09F101001BF862
:1038D0000000049009F103001BF80010401E1BF8C3
:1038E000000001EB002080B2039009F105001BF8F5
:1038F000000005900498062864D14C46519810B1F8
:10390000519804281BD14FF0000A0AE01BF80A2046
:103910002046611C8CB206A90A540AF1010000F08D
:10392000FF0A244800788245F0DB224606A9224897
:103930000CF0A6FB2046FFF7DCF801F05CB89BF822
:1039400000008DF818009BF801008DF81900002088
:103950008DF81A008DF81B008DF81C0006208DF8DC
:103960001D0051980128E8D14FF0000A0BE009EB47
:103970000A001BF8000009EB0A0106AA50540AF1DC
:10398000010000F0FF0ABAF1060FF0DB09F10602B0
:1039900006A90A480CF02FFB09F106000849088027
:1039A000CBE70FE0E20100205F6F00209060002075
:1039B000E067002087010020505E0020BC5A0020F4
:1039C0007E010020049810285ED1519850BB4FF022
:1039D000000A10E009EB0A001BF8000009EB0A01DD
:1039E00006AA505409EB0A01505C01F063F90AF190
:1039F000010000F0FF0ABAF1060FEBDBFE48007889
:103A000009EB0A0106AA5054FC48017809EB0A00A8
:103A1000401C1154FA48DDE9061206C00820FFF7E1
:103A200068F88AE75198042887D09BF800008DF841
:103A300018009BF801008DF8190000208DF81A007D
:103A40008DF81B008DF81C0006208DF81D004FF02E
:103A5000000A0BE009EB0A001BF8000009EB0A0161
:103A600006AA50540AF1010000F0FF0ABAF1060F4D
:103A7000F0DB09F1060206A9E2480CF0BCFA09F1F4
:103A80000600E149088058E70498032840F056876B
:103A90001BF8090006A901F8090009F101001BF84B
:103AA000001006AA115405984006010E09F1020003
:103AB000115406A911F8090001F0FCF806AA09F151
:103AC0000101505C01F0F6F806AA09F10201505C10
:103AD00001F0F0F809F103044FF0000A00F0DCBE39
:103AE0000398504485B2032D14DC0027C748465D77
:103AF0002046611C8CB206A90F542046611C8CB272
:103B000006A90E54384601F0D5F8304601F0D2F837
:103B100000F0BEBE042D12D1002748262046611CAD
:103B20008CB206A90F542046611C8CB206A90E5413
:103B3000384601F0BFF8304601F0BCF8E8E7052D43
:103B400012D1002700262046611C8CB206A90F5412
:103B50002046611C8CB206A90E54384601F0AAF822
:103B6000304601F0A7F8D3E7062D13D10027A74868
:103B700006792046611C8CB206A90F542046611CB0
:103B80008CB206A90E54384601F094F8304601F084
:103B900091F8BDE7072D13D100279C48867B20466E
:103BA000611C8CB206A90F542046611C8CB206A978
:103BB0000E54384601F07EF8304601F07BF8A7E756
:103BC000082D13D100279148C67B2046611C8CB27A
:103BD00006A90F542046611C8CB206A90E54384623
:103BE00001F068F8304601F065F891E70F2D13D128
:103BF00000278648067B2046611C8CB206A90F541C
:103C00002046611C8CB206A90E54384601F052F8C9
:103C1000304601F04FF87BE70B2D15D100270F2020
:103C2000F9F70CFA06462046611C8CB206A90F541F
:103C30002046611C8CB206A90E54384601F03AF8B1
:103C4000304601F037F863E7102D13D100276F4895
:103C5000467B2046611C8CB206A90F542046611C8D
:103C60008CB206A90E54384601F024F8304601F013
:103C700021F84DE7632D13D100276448067C2046C8
:103C8000611C8CB206A90F542046611C8CB206A997
:103C90000E54384601F00EF8304601F00BF837E7C5
:103CA000152D13D100275948867C2046611C8CB203
:103CB00006A90F542046611C8CB206A90E54384642
:103CC00000F0F8FF304600F0F5FF21E7252D13D175
:103CD00000274F4806782046611C8CB206A90F5475
:103CE0002046611C8CB206A90E54384600F0E2FF53
:103CF000304600F0DFFF0BE7272D13D100274548A2
:103D000006782046611C8CB206A90F542046611C1F
:103D10008CB206A90E54384600F0CCFF304600F0B5
:103D2000C9FFF5E6162D17D13B480068070E3A4843
:103D30000068C0F307462046611C8CB206A90F54E8
:103D40002046611C8CB206A90E54384600F0B2FF22
:103D5000304600F0AFFFDBE6172D16D12E48008865
:103D6000C0F307272C4806782046611C8CB206A9B0
:103D70000F542046611C8CB206A90E54384600F040
:103D800099FF304600F096FFC2E6262D16D11F4857
:103D9000808F070A1D4890F83C602046611C8CB259
:103DA00006A90F542046611C8CB206A90E54384651
:103DB00000F080FF304600F07DFFA9E6282D2DDBC6
:103DC0002D2D2BDCA5F128001FFA80F800270F48C5
:103DD000143010F808602046611C8CB206A90F54FC
:103DE0002046611C8CB206A90E54384600F062FFD2
:103DF000304600F05FFF8BE6960100209501002021
:103E0000505E0020BC5A00207E010020506000203F
:103E10008F0100208E010020040000202E2D13D1E0
:103E20000027F848867F2046611C8CB206A90F54F3
:103E30002046611C8CB206A90E54384600F03AFFA9
:103E4000304600F037FF63E62F2D1BDB322D19DCE7
:103E5000A5F12F001FFA80F80027EA481A3010F861
:103E600008602046611C8CB206A90F542046611CD4
:103E70008CB206A90E54384600F01CFF304600F004
:103E800019FF45E6332D1BDB362D19DCA5F1330078
:103E90001FFA80F80027DB481F3010F80860204622
:103EA000611C8CB206A90F542046611C8CB206A975
:103EB0000E54384600F0FEFE304600F0FBFE27E6CA
:103EC000372D1BDB3A2D19DCA5F137001FFA80F8DE
:103ED0000027CC48233010F808602046611C8CB2C3
:103EE00006A90F542046611C8CB206A90E54384610
:103EF00000F0E0FE304600F0DDFE09E63B2D14D177
:103F00000027C04890F827602046611C8CB206A9A3
:103F10000F542046611C8CB206A90E54384600F09E
:103F2000C9FE304600F0C6FEF2E53C2D16D1B5487C
:103F3000008D070AB34890F828602046611C8CB2B7
:103F400006A90F542046611C8CB206A90E543846AF
:103F500000F0B0FE304600F0ADFED9E53D2D14D1A5
:103F60000027A84890F82F602046611C8CB206A953
:103F70000F542046611C8CB206A90E54384600F03E
:103F800099FE304600F096FEC2E53E2D1BDB412D2A
:103F900019DCA5F13E001FFA80F8002799482B3064
:103FA00010F808602046611C8CB206A90F54204608
:103FB000611C8CB206A90E54384600F07BFE3046D8
:103FC00000F078FEA4E5422D1BDB452D19DCA5F1A0
:103FD00042001FFA80F800278A48303010F8086045
:103FE0002046611C8CB206A90F542046611C8CB27D
:103FF00006A90E54384600F05DFE304600F05AFE29
:1040000086E5462D1BDB492D19DCA5F146001FFA7C
:1040100080F800277B48343010F808602046611C87
:104020008CB206A90F542046611C8CB206A90E540E
:10403000384600F03FFE304600F03CFE68E54A2D71
:1040400014D100276F4890F838602046611C8CB26C
:1040500006A90F542046611C8CB206A90E5438469E
:1040600000F028FE304600F025FE51E54B2D16D11C
:104070006448408F070A634890F83A602046611C04
:104080008CB206A90F542046611C8CB206A90E54AE
:10409000384600F00FFE304600F00CFEF8E34C2DE1
:1040A00014D10027574890F83E602046611C8CB21E
:1040B00006A90F542046611C8CB206A90E5438463E
:1040C00000F0F8FD304600F0F5FDE1E35D2D14D180
:1040D00000274C4890F82A602046611C8CB206A943
:1040E0000F542046611C8CB206A90E54384600F0CD
:1040F000E1FD304600F0DEFDCAE35A2D15D14248FD
:1041000000880712404806782046611C8CB206A938
:104110000F542046611C8CB206A90E54384600F09C
:10412000C9FD304600F0C6FDB2E3642D70DBA32D5F
:104130006EDCA5F164001FFA80F808EBD871491015
:10414000C1EBC10202EB0111304A02EB410191F8CF
:10415000281001297ED108EBD8725210C2EBC2039D
:1041600003EB0212294B03EB420292F82D200F2A97
:104170000DD008EBD8725210C2EBC20303EB02124F
:10418000224B03EB420292F82D20192A41D14046DE
:1041900008EBD0714910A8EB410189B908EBD07147
:1041A0004A101849403151F832100F0E08EBD07107
:1041B0004A101449403151F83210C1F3074610E05B
:1041C000404608EBD0714A100E49403131F83210A8
:1041D000C1F3072708EBD0714A100A49403111F8A2
:1041E00032602046611C8CB206A90F542046611C27
:1041F0008CB206A90E54384600F05CFD304600F043
:1042000059FD45E350600020C00100205F6F002091
:10421000B1E0404608EBD0714910A8EB41010129FB
:1042200033D108EBD8714910C1EBC10202EB011187
:10423000F84A02EB4101D1F81E100A2291FBF2F17B
:10424000C1F3072708EBD8714910C1EBC10202EB9B
:10425000011100E02CE0EF4A02EB4101D1F81E1001
:104260000A2291FBF2F1CEB22046611C8CB206A963
:104270000F542046611C8CB206A90E54384600F03B
:1042800019FD304600F016FD02E300270026204607
:10429000611C8CB206A90F542046611C8CB206A981
:1042A0000E54384600F006FD304600F003FDEFE204
:1042B000404608EBD0714910A8EB4101012947D1D4
:1042C00008EBD8714910C1EBC10202EB0111D14AD0
:1042D00002EB410191F82D100B2914DC08EBD87189
:1042E0004910C1EBC10202EB0111CA4A02EB4101C4
:1042F000D1F81E10B1F57A7F02DB0027012616E007
:104300000027002613E008EBD8714910C1EBC10269
:1043100002EB0111BF4A02EB4101D1F81E10B1F5C9
:104320007A7F02DB0027002601E0002701262046D5
:10433000611C8CB206A90F542046611C8CB206A9E0
:104340000E54384600F0B6FC304600F0B3FC9FE255
:10435000002700262046611C8CB206A90F54204677
:10436000611C8CB206A90E54384600F0A3FC3046FE
:1043700000F0A0FC8CE2B5F5827F21DBB5F5927FE1
:104380001EDAA5F582701FFA80F80027C8EBC80076
:1043900000EB08109F4901EB400090F82860204690
:1043A000611C8CB206A90F542046611C8CB206A970
:1043B0000E54384600F07EFC304600F07BFC67E28D
:1043C000B5F5927F23DBB5F5A27F20DAA5F59270D3
:1043D0001FFA80F80027C8EBC80000EB08108D49D1
:1043E00001EB400090F82300C0F303162046611C47
:1043F0008CB206A90F542046611C8CB206A90E543B
:10440000384600F057FC304600F054FC40E2A42D42
:1044100020DBC32D1EDCA5F1A4001FFA80F80027C5
:10442000C8EBC80000EB08107A4901EB400090F897
:1044300022602046611C8CB206A90F542046611CE4
:104440008CB206A90E54384600F034FC304600F019
:1044500031FC1DE2C42D20DBE32D1EDCA5F1C400E0
:104460001FFA80F80027C8EBC80000EB0810694964
:1044700001EB400090F82D602046611C8CB206A92B
:104480000F542046611C8CB206A90E54384600F029
:1044900011FC304600F00EFCFAE1E42D21DBB5F50D
:1044A000827F1EDAA5F1E4001FFA80F80027C8EB2E
:1044B000C80000EB0810574901EB400090F8276056
:1044C0002046611C8CB206A90F542046611C8CB298
:1044D00006A90E54384600F0EDFB304600F0EAFB2A
:1044E000D6E1B5F5A27F21DBB5F5B27F1EDAA5F5E1
:1044F000A2701FFA80F80027C8EBC80000EB081074
:10450000444901EB400090F829602046611C8CB2C0
:1045100006A90F542046611C8CB206A90E543846D9
:1045200000F0C8FB304600F0C5FBB1E1B5F5B27F45
:1045300032DBB5F5D27F2FDAA5F5B2701FFA80F81D
:104540000027404608EBD0714910A8EB410149B95A
:10455000C8EBC80000EB08102E4901EB400090F8B2
:104560002B6008E0C8EBC80000EB0810294901EBFC
:10457000400090F82C602046611C8CB206A90F54B4
:104580002046611C8CB206A90E54384600F092FBFE
:10459000304600F08FFB7BE1B5F5D27F23DBB5F52C
:1045A000E27F20DAA5F5D2701FFA80F80027C8EB69
:1045B000C80000EB0810174901EB400090F82300F9
:1045C00000F00F062046611C8CB206A90F5420464D
:1045D000611C8CB206A90E54384600F06BFB3046C5
:1045E00000F068FB54E140F2CA20854214D1002754
:1045F00056262046611C8CB206A90F542046611C29
:104600008CB206A90E54384600F054FB304600F038
:1046100051FB3DE15F6F002040F2CB20854222DB61
:1046200040F2D52085421EDCA5F2CB2080B202905C
:10463000FB49029811F810700121029801EB40002B
:10464000F7490E5C2046611C8CB206A90F54204627
:10465000611C8CB206A90E54384600F02BFB304684
:1046600000F028FB14E1B5F5487F13D10027ED4891
:10467000C67C2046611C8CB206A90F542046611CE2
:104680008CB206A90E54384600F014FB304600F0F8
:1046900011FBFDE0B5F5487F1EDD40F2513085424B
:1046A0001ADCA5F54870E04931F810000712A5F5AD
:1046B000487011F810602046611C8CB206A90F5496
:1046C0002046611C8CB206A90E54384600F0F2FA5E
:1046D000304600F0EFFADBE04FF6F250854213D19E
:1046E0000027D24806782046611C8CB206A90F54D8
:1046F0002046611C8CB206A90E54384600F0DAFA46
:10470000304600F0D7FAC3E042F6D040854237DBAE
:1047100042F6AF70854233DCA5F53050D038172112
:10472000B0FBF1F0C0B202900298C0EBC00101EB07
:104730000010BF4901EB40000090A5F53050D03883
:104740001721B0FBF1F201FB12000190DDE900013D
:1047500030F81100070ADDE9000110F81160204669
:10476000611C8CB206A90F542046611C8CB206A9AC
:104770000E54384600F09EFA304600F09BFA87E06F
:1047800043F29020854236DB43F29740854232DC8B
:10479000A5F5485090380A21B0FBF1F0C0B2029064
:1047A000029800EB400101EB0010A2490844009080
:1047B000A5F5485090380A21B0FBF1F201FB120038
:1047C0000190DDE9000130F81100070ADDE9000180
:1047D00010F811602046611C8CB206A90F542046C7
:1047E000611C8CB206A90E54384600F063FA3046BC
:1047F00000F060FA4CE048F2A800854236DB48F24F
:10480000B010854232DCA5F50040A8383521B0FB58
:10481000F1F0C0B202900298C0EB0010C0EBC000F3
:10482000854908440090A5F50040A8383521B0FB23
:10483000F1F201FB12000190DDE9000130F81100F6
:10484000070ADDE9000110F811602046611C8CB2F6
:1048500006A90F542046611C8CB206A90E54384696
:1048600000F028FA304600F025FA11E00027002673
:104870002046611C8CB206A90F542046611C8CB2E4
:1048800006A90E54384600F015FA304600F012FA28
:104890000AF1010000F0FF0A05988245FFF620A901
:1048A00066480778664806782046611C8CB206A9DF
:1048B0000F542046611C8CB206A90E54519804284E
:1048C00006D105984200C91C5E480BF094FB34E009
:1048D000519840B9224606A95B480BF0D1FB20460F
:1048E000FEF707F929E09BF800008DF818009BF807
:1048F00001008DF8190000208DF81A008DF81B00BA
:104900000321059801EB4000000A8DF81C00059872
:1049100001EB4000C0B28DF81D00059801EB40008E
:1049200000EB090206A949480BF065FB0321059835
:1049300001EB40004844464908805CE04548407827
:10494000192858D11BF809602046611C8CB23E49D9
:104950000E54304600F0AEF909F101001BF800607A
:104960002046611C8CB238490E54304600F0A2F942
:104970002C4806792046611C8CB233490E543046CF
:1049800000F098F9274806782046611C8CB22E4921
:104990000E54304600F08EF9224846782046611CBD
:1049A0008CB229490E54304600F084F91D488678AF
:1049B0002046611C8CB224490E54304600F07AF92E
:1049C0001848C6782046611C8CB21F490E543046E8
:1049D00000F070F9194806782046611C8CB21A491B
:1049E0000E54174806782046611C8CB216490E54A6
:1049F0002046FEF77EF853B0BDE8F08F2DE9F04772
:104A0000074615480078401C134908701348007881
:104A100013490978884225D00020BDE8F0870000BE
:104A2000C062002050600020E067002009000020E4
:104A30005F6F00203F7D0020526D00209601002016
:104A40009501002090610020505E0020BC5A00209B
:104A50007E010020505D002094010020860100208E
:104A6000870100208B480078FF280BD08948007808
:104A700089490979884205D08648007810B100201C
:104A8000BDE8F08783484078192847D10421814840
:104A900000F020F905467F4840797E49097900EB0E
:104AA0000120A84201D00020EAE77A4880787949BD
:104AB000C978884202DB7748C07801E07548807881
:104AC0008046744880787349C978884202DB71480F
:104AD000807801E06F48C07881466F480079404592
:104AE00003DB6D480079484501DD0020C8E76B48CD
:104AF00000780BF0F3F9F3F7F5FB142190FBF1F2DA
:104B000001FB1200C6B2002404E06420FAF772FD33
:104B1000601CC4B2B442F8DB0120B1E75D484078C4
:104B2000032809D05B484078062805D059484078CA
:104B3000102801D00020A3E75648C178807801EB07
:104B40000020092847D15348407806281FD15148F2
:104B5000807951490978884201D0002090E74D487A
:104B6000C0794D494978884201D0002088E74948FA
:104B7000007A49498978884201D0002080E7454879
:104B8000407A4549C978884201D0002078E74148F9
:104B90004078032808D1F3F7A5FB052190FBF1F23B
:104BA00001FB12003E4908703D480078012801D001
:104BB000002065E7F3F796FB142190FBF1F201FB6F
:104BC0001200C6B2002404E06420FAF713FD601C52
:104BD000C4B2B442F8DB2F484078062822D1082F0F
:104BE00020DC2C48C078022806DA2B48007C00F034
:104BF0000100B8B1002043E72648C078042806DA4F
:104C00002548007C00F0020060B1002038E7214810
:104C1000C078082806D12048007C00F0040008B1C4
:104C200000202DE71F480078801EC1B2194800F00F
:104C300051F805461B480078401E1649095C194882
:104C40000078801E134A105C01EB0020A84201D1BD
:104C5000012015E7002013E710B50E48C0780D4974
:104C6000897800EB012084B22046FFF7C7FE60B1CF
:104C7000FDF72BFF00F018F806490020FEF705FEAF
:104C800004490020FDF795FF01E0FDF743FE10BD4C
:104C900070470000505D002050600020940100200B
:104CA0008401002087010020FF201849087018495E
:104CB00008707047164A127882EA0001154A525C61
:104CC000124B1B785A40124B1A70134A525C0F4B0E
:104CD0001A707047F0B502460B46FF24FF250026E8
:104CE0000BE03046771CFEB2105C80EA04010948F4
:104CF000405C80EA05040848455C181EA3F10107E2
:104D0000FBB2EED145EA0420F0BD00009501002081
:104D1000960100204A2802084A2902087047704775
:104D200010B5FDF733FF10BD10B50446142221461F
:104D3000FE480BF060F91422FC4940F2BA20F8F763
:104D40002EFA10BD10B50446F9480078F8494978A4
:104D500000EB0120F649897800EB0140F449C9785D
:104D600000EB0160D4F8B410884212D1142204F18F
:104D70003401EE480BF0D0F858B10021472001551E
:104D8000142204F13401E9480BF07AF9E748FFF7FF
:104D9000CBFFE748007994F8C81088421CD094F8FB
:104DA000C800002818DD94F8C800FF2814DA94F829
:104DB000C800DF490871084601790620F8F76AF94A
:104DC000DB480079DB49087008460078DA4981F849
:104DD000F800002004F084F994F8F800D549097827
:104DE00088421BD094F8F800C0B194F8F800FF286E
:104DF00014D094F8F800CF49087008460078CE49DE
:104E000081F8F800CB480078C94908710846017953
:104E10000620F8F73FF9002004F062F9C448007951
:104E200094F84910884215D094F84900002811DD03
:104E300094F84900FF280DDA94F84900BC4908713C
:104E4000084601790620F8F725F9B9480079BA49EA
:104E500081F84900D4F8CC0001F070FCB74909682A
:104E600088420CD0D4F8CC0048B1D4F8CC0001F082
:104E700065FCB24908600846006803F09EFC10BD5E
:104E800010B5AB480078AA49497800EB0120A84941
:104E9000897800EB0140A649C97800EB0160A6497A
:104EA000C1F8B400A248007981F8C800A048007990
:104EB00081F84900A1480068C1F8CC00012081F8C0
:104EC0004800142299499C4834300BF0D9F810BDA1
:104ED0007047704770477047704710B594488068B6
:104EE000B0F5964F04D14FF49640FAF7F9FA30E056
:104EF0008F488068B0F5165F04D14FF41650FAF76A
:104F0000EFFA26E08A488068B0F5164F04D14FF4D6
:104F10001640FAF7E5FA1CE085488068B0F5614F65
:104F200004D14FF46140FAF7DBFA12E08048806860
:104F3000B0F5E13F04D14FF4E130FAF7D1FA08E0DF
:104F40007B488068B0F5963F03D14FF49630FAF76E
:104F5000C7FA10BD76488068B0F5165F01D105200C
:104F6000704773488068B0F5964F01D10620F7E787
:104F70006F488068B0F5164F01D10720F0E76C4804
:104F80008068B0F5614F01D10820E9E76848806882
:104F9000B0F5E13F01D10920E2E765488068B0F54E
:104FA000963F01D10A20DBE70620D9E77047024689
:104FB00000207047704730B504460B46002214B1FC
:104FC000032C2FD117E0002112E0C1EBC10000EB50
:104FD00001105B4D05EB400090F82800012805D139
:104FE0009A4201D1084630BD501CC2B2481CC1B221
:104FF0002029EADB16E0002111E0C1EBC10000EB43
:1050000001104F4D05EB400090F8280028B99A4256
:1050100001D10846E7E7501CC2B2481CC1B22029A2
:10502000EBDB00BF00BF4FF0FF30DCE770B504469C
:105030000D4621460020FFF7BEFFC6B2701C10B11E
:105040002E70012070BD0020FCE770B504460D46AF
:1050500021460320FFF7AFFFC6B2701C10B12E70BF
:10506000012070BD0020FCE7F8B505460E46144649
:1050700035B1012D66D0022D65D0032D72D1B4E07B
:1050800024B92C4800780DF081F9F8BD012C04D129
:10509000274988680DF07AF9F7E7022C04D12449F2
:1050A000887C0DF073F9F0E7032C04D123480068E5
:1050B0000DF06CF9E9E7042C08DB072C06DC211F56
:1050C0001B4A1A32505C0DF061F9DEE7082C09DB4F
:1050D0000B2C07DCA4F10801154A1F32505C0DF0BF
:1050E00055F9D2E70C2C09DB0F2C07DCA4F10C01DD
:1050F0000F4A2332505C0DF049F9C6E7102C04D159
:105100000B49088D0DF042F9BFE7112C56DB302C0E
:1051100054DCA4F11100C0EBC00101EB0010084900
:1051200001EB400090F82800E8B90DE0C0620020D3
:10513000506000208E010020D46200200400002076
:105140005F6F0020C9E0EDE0A4F11101C1EBC102E5
:1051500002EB0111FC4A02EB410191F82D000DF028
:1051600015F992E7DDE0A4F11100C0EBC00101EBFD
:105170000010F54901EB400090F82D0000280FDDEC
:10518000A4F11101C1EBC10202EB0111EE4A02EBE5
:10519000410191F82D1001F11E000DF0DFF874E7C8
:1051A000A4F11101C1EBC10202EB0111E64A02EBCD
:1051B000410191F82D000DF0E9F866E7312C04D19A
:1051C000E249888F0DF0E2F85FE7322C04D1DF4925
:1051D000887F0DF0DBF858E7332C05D1DB4991F8D7
:1051E0003E000DF0D3F850E79DE069462046FFF7FA
:1051F0002CFF9DF80000C0EBC00101EB0010D2496C
:1052000001EB400090F82D00002865DD9DF80000BE
:10521000C0EBC00101EB0010CB4901EB400090F85E
:105220002800E8BB9DF80000C0EBC00101EB0010B6
:10523000C54901EB400090F82D000C280CDB9DF8CF
:105240000000C0EBC00101EB0010BF4901EB4000C2
:1052500090F82D00162819DD9DF80000C0EBC00164
:1052600001EB0010B84901EB400090F82D00172821
:1052700020DB9DF80000C0EBC00101EB0010B2493B
:1052800001EB400090F82D001E2813DC9DF8000073
:10529000C0EBC00101EB0010AB4901EB400000E0A6
:1052A0001AE090F82600012801D10020EDE64FF029
:1052B0007E50EAE69DF80000C0EBC00101EB001053
:1052C000A14901EB400090F82600012802D14FF0DF
:1052D0007E50DAE60020D8E600BF69462046FFF798
:1052E000A5FE9DF80000C0EBC00101EB001096493F
:1052F00001EB400090F82D00002811DD9DF8001012
:10530000C1EBC10202EB01118F4A02EB4101D1F85E
:105310001E000DF023F807468D490CF0EDFEB4E6B3
:1053200000BF00BF00BF00BF00BFAEE62DE9F843DD
:105330000546884614461E4625B1012D7ED0032D14
:105340007DD142E2D4B930460CF0E8FF7F490871C4
:1053500030460CF0E3FF7F49087030460CF0DEFF6A
:10536000C7B239460620F7F795FEF2F7DFFF0020B7
:1053700003F0B6FE002004F067FDE4E1012C7DD1CE
:1053800030460CF0CBFF7149886008468068B0F564
:10539000165F13D1002008730846017B1520F7F72C
:1053A00079FE6A48017B1320F7F774FE4FF416501C
:1053B000FAF796F8062068490870C4E163488068E7
:1053C000B0F5964F14D10120604908730846017B5F
:1053D0001520F7F75FFE5D48017B1320F7F75AFEB3
:1053E0004FF49640FAF77CF803205B490870AAE175
:1053F00056488068B0F5164F0FD102205349087304
:105400000846017B1520F7F745FE4FF41640FAF7E2
:1054100067F802205049087095E14C488068B0F563
:10542000614F17D10320494908730846017B1520B5
:10543000F7F730FE4548017B132001E084E19DE24F
:10544000F7F728FE0120444908704FF46140FAF74D
:1054500047F878E13D488068B0F5E13F16D1042077
:105460003A4908730846017B1520F7F713FE3748C1
:10547000017B1320F7F70EFE012000E020E0364903
:1054800008704FF4E130FAF72BF85CE12F488068A0
:10549000B0F5963F91D105202C4908730846017B51
:1054A0001520F7F7F7FD2948017B1320F7F7F2FDE8
:1054B0000120294908704FF49630FAF711F842E1BB
:1054C000022C0AD130460CF029FF20498874084686
:1054D000817C1420F7F7DEFD35E1032C20D1304626
:1054E0000CF01CFF1D49086008460068010E1620DC
:1054F000F7F7D0FD19480068C0F307411720F7F708
:10550000C9FD16480088C0F307211820F7F7C2FD2F
:10551000124801781920F7F7BDFDF2F707FF12E1F5
:10552000042C1DDB072C1BDC30460CF0F7FEC2B24E
:10553000201F06491A310A54221F0B46995C2F324C
:1055400090B2F7F7A7FDFEE05F6F002050600020EB
:1055500000007A448E010020890100200400002010
:10556000082C11DB0B2C0FDC30460CF0D7FEC2B23E
:10557000A4F10800FA490A5402460B46995C3332FA
:1055800090B2F7F787FDDEE00C2C12DB0F2C10DC5D
:1055900030460CF0C3FEC2B2A4F10C00F049091D64
:1055A0000A5402460B46995C373290B2F7F772FD07
:1055B000C9E0102C13D130460CF0B0FEE8491F3979
:1055C00008850846008D010A3C20F7F763FDE44892
:1055D0001F3890F828103D20F7F75CFDB3E0112C40
:1055E00066DB302C64DC002130460CF047FE1BD11A
:1055F00030460CF093FEC1B2A4F11100C0EBC00222
:1056000002EB0010D74A02EB400080F82D10012178
:10561000A4F11100C0EBC00202EB0010D14A02EB72
:10562000400080F828103FE0CF4930460CF0C2FE21
:105630001BD230460CF072FEC1B2A4F11100C0EBD7
:10564000C00202EB0010C74A02EB400080F82D10A8
:105650000021A4F11100C0EBC00202EB0010C14A0E
:1056600002EB400080F828101EE0C04930460CF0E4
:10567000A1FF07460CF052FEC1B2A4F11100C0EB2D
:10568000C00202EB0010B74A02EB400080F82D1078
:105690000121A4F11100C0EBC00202EB0010B14ADD
:1056A00002EB400080F828100120B14948704AE020
:1056B000312C15D130460CF031FEA9491F398887AD
:1056C0000846808F010A1B20F7F7E4FCA4481F3826
:1056D00090F83C101C20F7F7DDFCFBF731FE32E0C0
:1056E000322C06D130460CF019FE9D491F398877BF
:1056F00029E0332C27D130460CF010FE98491F3991
:1057000081F83E00084690F83E0001281BD108466B
:10571000817F2E20F7F7BEFC914A521F115D04F1E4
:105720002F00F7F7B7FC8E4A115D04F13300F7F74D
:10573000B1FC8B4A121D115D04F13700F7F7AAFC8A
:1057400001208C4908701AE169462046FFF76EFC7B
:105750009DF80000202800DB11E19DF80000C0EB5F
:10576000C00101EB00107F4901EB400090F82800D8
:10577000012829D19DF80000C0EBC00101EB001009
:10578000784901EB400090F82D0058B903209DF8AE
:105790000010C1EBC10202EB0111724A02EB4101A0
:1057A00081F82D00744930460CF038FE07460CF0A5
:1057B00099FD9DF80010C1EBC10202EB0111694A8D
:1057C00002EB4101C1F81E00D9E069462046FFF70F
:1057D0003CFC9DF80000202800DBD0E0012064495B
:1057E00048709DF80000C0EBC00101EB00105D495E
:1057F00001EB400090F82800F0BB9DF80000C0EBE2
:10580000C00101EB0010574901EB400090F82D005A
:1058100058B901209DF80010C1EBC10202EB011143
:10582000504A02EB410181F82D00534930460CF0FB
:10583000F5FD07460CF056FD9DF80010C1EBC102C6
:1058400002EB0111474A02EB4101C1F81E009DF82D
:105850000000C0EBC00101EB0010114601EB40005D
:1058600090F82D000C280EDB9DF80000C0EBC00165
:1058700001EB0010114600E047E001EB400090F81A
:105880002D00162819DD9DF80000C0EBC00101EBCA
:105890000010344901EB400090F82D00172820DB60
:1058A0009DF80000C0EBC00101EB00102D4901EB99
:1058B000400090F82D001E2813DC002130460CF02B
:1058C000DDFC01D1012000E000209DF80010C1EBBB
:1058D000C10202EB0111234A02EB410181F82600CB
:1058E0003DE0002130460CF0C9FC01D0012000E071
:1058F00000209DF80010C1EBC10202EB0111194A12
:1059000002EB410181F8260029E09DF80000C0EB80
:10591000C00101EB0010134901EB400090F82D008D
:1059200058B903209DF80010C1EBC10202EB011130
:105930000C4A02EB410181F82D000F4930460CF072
:105940006DFD07460CF0CEFC9DF80010C1EBC102C6
:1059500002EB0111034A02EB4101C1F81E000EE007
:105960006F6000205F6F00200000F8410000F041F0
:10597000E20100208201002000007A4400BF00BF45
:10598000BDE8F883F8B504460F4615461E46052CBB
:105990004BD2DFE804F03903381D3700694628464A
:1059A000FFF744FB9DF80000202800DB3EE00120CB
:1059B000FE4948709DF80010C1EBC10202EB0111D5
:1059C000FB4A02EB4100152231460AF014FB2DE0A0
:1059D00069462846FFF739FB9DF80000202800DBC8
:1059E00024E00120F14948709DF80010C1EBC1028C
:1059F00002EB0111EE4A02EB4100152231460AF09A
:105A0000FAFA13E012E011E005EB450000EB051097
:105A1000E8490844316840F8061F71684160317AEE
:105A200001720120E149887000BF00BF00BFF8BDCE
:105A3000F0B50446012C7CD1202A00DB82E05F2BEC
:105A400009D10025C2EBC20606EB0216D84F07EBC0
:105A5000460686F82D503E2B09D10325C2EBC2061F
:105A600006EB0216D24F07EB460686F82D50402B68
:105A700009D10425C2EBC20606EB0216CC4F07EB98
:105A8000460686F82D50032B1ED10D25C2EBC2060B
:105A900006EB0216C64F07EB460686F82D50C2EB02
:105AA000C20505EB02153E4606EB450595F82300B9
:105AB00000F00F0040F01000C2EBC20505EB02152C
:105AC00006EB450585F82300052B1ED11325C2EBF7
:105AD000C20606EB0216B64F07EB460686F82D50B7
:105AE000C2EBC20505EB02153E4606EB450595F8EF
:105AF000230000F00F0040F03000C2EBC20505EBC0
:105B0000021506EB450585F82300052B18D0032B5D
:105B100016D0C2EBC20505EB0215A54E06EB4505F6
:105B200095F8230000F00F0040F04000C2EBC205E2
:105B300000E006E005EB021506EB450585F82300BD
:105B400000E000BF00BFF0BD0246012A04D0022AD7
:105B50000FD0042A0FD10DE0202909DAC1EBC100D2
:105B600000EB0110924B03EB400090F827007047C8
:105B700002E001E000E000BF00BF00BFF7E730B582
:105B8000012804D0022811D0042810D10DE053B20E
:105B9000C1EBC10404EB0114854D05EB440484F80A
:105BA00027300123814C637002E001E000E000BF78
:105BB00000BF30BD704738B505460C4625B1012DF4
:105BC0000DD0032D33D11EE0342C07DA04EB440052
:105BD00000EB041077490844801D38BD28E0694671
:105BE0002046FFF723FA9DF80000202801DB002063
:105BF000F3E79DF80000C0EBC00101EB00106C4919
:105C000001EB4000E9E769462046FFF71EFA9DF8E0
:105C10000000202801DB0020DFE79DF80000C0EB3A
:105C2000C00101EB0010624901EB4000D5E700BF65
:105C300000BF61A0D1E738B505460C4625B1012D5E
:105C40000CD0032D34D11EE0342C06DA04EB4400D2
:105C500000EB04105749084438BD2AE06946204645
:105C6000FFF7E4F99DF80000202801DB0020F3E7AE
:105C70009DF80000C0EBC00101EB00104C4901EBA6
:105C800040001530E8E769462046FFF7DEF99DF849
:105C90000000202801DB0020DEE79DF80000C0EBBB
:105CA000C00101EB0010424901EB40001530D3E781
:105CB00000BF00BF40A0CFE738B504460D460CB981
:105CC0005F2038BD012C70D169462846FFF7AEF938
:105CD0009DF80000202801DB0020F2E79DF800007D
:105CE000C0EBC00101EB0010314901EB400090F81E
:105CF000280008B95F20E4E79DF80000C0EBC00170
:105D000001EB00102A4901EB400090F82D00032818
:105D10000CD09DF80000C0EBC00101EB001024493D
:105D200001EB400090F82D00072801D13E20C8E784
:105D30009DF80000C0EBC00101EB00101C4901EB15
:105D4000400090F82D0004280CD09DF80000C0EB16
:105D5000C00101EB0010164901EB400090F82D0046
:105D6000082801D14020ACE79DF80000C0EBC0013D
:105D700001EB00100E4901EB400090F82D000D28BA
:105D800001D102209DE79DF80000C0EBC00101EBAE
:105D90000010074901EB400090F82D00132818D09F
:105DA0009DF80000C0EBC0010AE016E0E20100200F
:105DB0005F6F00203F7D00206E756C6C000000005E
:105DC00001EB0010E24901EB400090F82D000B2898
:105DD00001D1052075E75F2073E7032C05D1052D60
:105DE00001DB00206DE75F206BE75F2069E7F8B516
:105DF00006460F4615461C46052E4AD2DFE806F039
:105E00003B033A1E390069462846FFF70FF99DF813
:105E10000000202800DB3DE00120CE4948709DF8BD
:105E20000000C0EBC00101EB0010C94901EB4000CC
:105E3000216840F8151F616841602BE069462846DB
:105E4000FFF703F99DF80000202800DB22E0012085
:105E5000C04948709DF80000C0EBC00101EB001084
:105E6000BB4901EB4000216840F8151F61684160A3
:105E700010E00FE00EE005EB450000EB0510B64921
:105E8000084421680160A18881800120B14988709F
:105E900000E000BF00BFF8BDB048704710B5B04883
:105EA0000088FF2835D008DC002834D0012813D022
:105EB00002281FD0942847D12AE0A0F2E530D0B1C3
:105EC0000A280AD0A0F2E510002830D0A0F57A40C8
:105ED0003538002838D11DE000BF1422A1A1A54803
:105EE0000AF0CEF81422A4A1A5480AF0C9F840F29D
:105EF000EF3010BD00BF1422A2A19E480AF0C0F8E6
:105F00001422A3A19E480AF0BBF840F2E530F0E766
:105F100000BF00BF00BF1422A0A196480AF0B0F84D
:105F20001422A2A196480AF0ABF89420E1E71422CB
:105F3000A2A190480AF0A4F81422A3A190480AF064
:105F40009FF840F2CA50D4E785480088D1E78948D5
:105F500070478B48704710B5044601207D49087191
:105F60001422214683480AF046F810BD10B50446B5
:105F70000120784908711422214681480AF03BF833
:105F800010BD10B50446E1B21D20F7F783F82112C9
:105F90002020F7F77FF84CB1FF2C07D04FF6FF70A9
:105FA000844203D0012C01D0022C00D110BD6C48DA
:105FB000048000BFFAE770B505460C461646224637
:105FC000294686480AF017F82046FCF792FD70BD76
:105FD0000120704718B10121814A116002E00021BF
:105FE0007F4A116070477F480079704710B50446BA
:105FF000210E1620F7F74EF8C4F307411720F7F7E4
:1060000049F8C4F307211820F7F744F8E1B2192042
:10601000F7F740F810BD10B5044621461220F7F7F7
:1060200039F810BD002070476F48007860B16F48A4
:106030000088002805DD6D480088401E6B490880F7
:1060400002E000206849087070470246002070474F
:106050007047014600207047024600207047014605
:10606000002070470146002070470146002070471D
:106070000146002070470146002070477047704776
:1060800010B500220021002019E0C0EBC00303EB93
:1060900000132F4C04EB430393F82830012B06D157
:1060A000534B9854534B1A54531CDAB205E0524BDD
:1060B0005854524B19544B1CD9B2431CD8B2202807
:1060C000E3DB4F4B1A704F4B197010BD30B50446CF
:1060D0000A46002314B1032C2FD117E0002112E04F
:1060E000C1EBC10000EB0110194D05EB400090F829
:1060F0002800012805D1914201D1184630BD581C15
:10610000C3B2481CC1B22029EADB17E0002111E02C
:10611000C1EBC10000EB01100D4D05EB400090F804
:10612000280028B9914201D11846E7E7581CC3B2AC
:10613000481CC1B22029EBDB00E000BF00BF4FF0DC
:10614000FF30DBE701460020704702460020704721
:106150005F6F0020E20100203F7D0020C062002030
:10616000C00100204E4554495820436F6E74726F31
:106170006C730000980100204E4343420000000071
:10618000AC0100204A6574436F6E74726F6C7300CB
:106190004A65742050726F647563740054656D6352
:1061A0006F436F6E74726F6C7300000054656D63A3
:1061B0006F2050726F647563740000004D696372E4
:1061C0006F67726F000000004D6963726F67726FD6
:1061D0002050726F6475637400000000505E0020F0
:1061E000A0012142506000200A0000200C00002085
:1061F00060670020A067002080670020C067002043
:10620000E9010020EB010020F04908807047F049C7
:1062100008607047EF490860704710B50020FFF72D
:10622000F9FF0020FFF7F3FFEB49888FFFF7ECFF42
:10623000E94991F83C100902E74A928F41EA22218C
:1062400088B2F9F762FCE44890F83C000002E249A9
:10625000898F40EA212081B2E048A0F8441010BDA7
:1062600030B587B00025DE48007800F00200A0B30A
:10627000DC48DD490860DD480288DD480168DA480D
:10628000006809F0B8FED9480088DA49088000BFE4
:10629000D94800680088ADF81800D74800684088E1
:1062A000ADF81A0000BFD4480068C18806A8F9F705
:1062B0009AFB0446012000234FF41672C94900904E
:1062C00001A802F046FA05462DB101232A46C54928
:1062D00001A803F07CFD0020A08007B030BDBD48C0
:1062E00000687047BB480068401C08B10120704737
:1062F0000020FCE7B64800687047C0490860704756
:10630000BE4800687047B1480088704710B5034622
:10631000002033B1D3F801400C60B3F8054014807D
:10632000062010BD2DE9F04786B004468A46174680
:106330001E46DDF838800025A94600200090B048B0
:10634000007850B9B8F1010F07D1A24800680028C1
:1063500003DA002006B0BDE8F0878120A949087063
:106360000220ADF8080020894FF6FF71884206D060
:106370002089002801DDA07A08B1207848B99F481B
:10638000006801909148008800900B209D4948705A
:106390000EE02078062808D16A4601A92046FFF7BA
:1063A000B5FF0A209749487002E04FF0FF30D1E76F
:1063B00001980390BDF80000ADF80A000020049099
:1063C00005900225321D91B28E4A501902F0F2F862
:1063D00005448C4948193246394609F00CFE3544CB
:1063E000B8F1010F06D18648007818B929468548CA
:1063F000FAF777FDA94640F27621824809F07AFE45
:1064000000254846A6E72DE9F0478EB081460C46A8
:1064100016461F464FF0000800200D9009900A9084
:106420000B900C90059006900790089001900290B8
:1064300003900490002582467148007848B9012FE6
:1064400007D164480068002803DA00200EB0BDE8D8
:10645000F0876848B0F8008063480460012F0CD1D1
:106460006748007848B9B8F1000F01DA0020EDE77D
:10647000B8F1000F01D10020E8E74FF000082078C4
:10648000812804D05E48007808B90020DEE794F83F
:1064900001A00DA9A01C02F092F800200A90ADF80E
:1064A00026000690ADF816000290ADF8060054489C
:1064B000007840B950480068C088ADF826004E48C2
:1064C000006800680A90BDF83400001F80B20D908B
:1064D000BAF10A0F03D0BAF10B0F3CD124E0FFF759
:1064E00009FF0A99884208D1FFF70DFFBDF8261071
:1064F000884202D100200D9015E009A9484602F01B
:1065000003F9BDF83400B0420BDA002504E0281D81
:10651000205C6055681C85B2BDF834008542F6DB0E
:1065200001E000200D9017E009A9484602F0ECF8C0
:10653000BDF83400B0420BDA002504E0281D205CD1
:106540006055681C85B2BDF834008542F6DB01E079
:1065500000200D9000E000BF00BFBDF8340075E7DB
:106560000021B0B106220270194A1268C0F8012059
:10657000421C164B1B88A0F8053000220281827253
:1065800000BF04E0002300F10B025354491C07290B
:10659000F8DB70470021C0B106220270174A12686A
:1065A000C0F80120421C094B1B88A0F805304FF6AB
:1065B000FF7202810022827200BF04E0002300F11A
:1065C0000B025354491C0729F8DB7047D001002007
:1065D000D4010020CC010020506000208055002014
:1065E0004001002044680020DC0100203C01002024
:1065F00034010020E001002048010020D8010020E3
:10660000E80100209C6A00200146474830F811004C
:1066100070477047014641F288304843800A70470E
:10662000014642F210704843800A704702463F48D4
:10663000805C022804D141F288304843800A7047C8
:106640003A48805C012804D144F620604843800A1F
:10665000F5E73648805C032804D142F210704843C5
:10666000800AECE73148805C042802D02F48805C27
:1066700020B940F6B8304843800AE0E700BFDEE7C3
:106680002020704701462A4850F831007047002208
:10669000274941F830207047F0B502460C460023E8
:1066A00000200021002511462546224E36F81160B3
:1066B000AE1B33B2642B02DA13F1640F08DC1D4EFB
:1066C00036F8116006EB63061A4F27F8116026E0D2
:1066D000184E36F81160C1EBC10707EB0117DFF860
:1066E00058C00CEB470797F822707E43114F27F8EC
:1066F00011603E4636F811602E4427F811603E4680
:1067000036F81160C1EBC10707EB01170CEB470727
:1067100097F8227096FBF7F6064F27F81160054EA2
:1067200036F81100F0BD0000D41600201F750020BF
:1067300090600020126D00205F6F0020704770474E
:106740002DE9F04F81460B4608254FF0000AA9F1CC
:10675000010000F0FF094C464FEA690900BFF94803
:106760000078012874D1B9F1030F5EDC642700BF03
:1067700009EB0910F44E06EB4001088C984205DB4A
:10678000F24800EBC4004068BDE8F08F08889842EA
:1067900003DCEE4850F83400F6E7082241E031F817
:1067A0001200984222DC501E31F8100098421DDB86
:1067B000521E31F81260501C31F81000351A9DB18C
:1067C00031F81200C01A00FB07F898FBF5F802FB3D
:1067D0000788DF4850F824C00CFB08FC9CFBF7FC42
:1067E000DA4850F8340084446046CDE70DB94FF0E4
:1067F000010A284605EBD076751031F81200984250
:1068000001DD2A4400E0521B002A03DCCF4850F887
:106810003400B9E7102A04DBCC4800EBC400406820
:10682000B2E7BAF1000FBAD0D5E064271925C949FB
:106830000888984203DBC54850F83400A4E7B1F853
:106840006400984205DCC14800EBC40040689BE747
:1068500064E019225EE0488E98422DDA192628E07D
:1068600031F81600984222DC701C31F81000984272
:106870001DDB701C31F8100031F816B0A0EB0B05D1
:106880009DB131F81600181A00FB07F898FBF5F8CF
:1068900006FB0788AE4850F824C00CFB08FC9CFBA4
:1068A000F7FCAA4850F83400844460466CE7701C3A
:1068B000C6B2322ED4DB2CE0002628E031F81600D8
:1068C000984222DC701C31F8100098421DDB701CCD
:1068D00031F8100031F816B0A0EB0B059DB131F87E
:1068E0001600181A00FB07F898FBF5F806FB078856
:1068F000974850F824C00CFB08FC9CFBF7FC93481D
:1069000050F83400844460463EE7701CC6B2192E2D
:10691000D4DB00BFBAF1000F9DD05CE0642709EB27
:106920000910894E06EB40010825088C984204DBCB
:10693000864800EBC400406826E70888984203DCDC
:10694000824850F834001FE7082241E031F8120075
:10695000984222DC501E31F8100098421DDB521E76
:1069600031F81260501C31F81000351A9DB131F821
:106970001200C01A00FB07F898FBF5F802FB078825
:10698000734850F824C00CFB08FC9CFBF7FC6F48D4
:1069900050F8340084446046F6E60DB94FF0010A21
:1069A000284605EBD076751031F81200984201DDCB
:1069B0002A4400E0521B002A03DC644850F83400EB
:1069C000E2E6102A04DB614800EBC4004068DBE625
:1069D000BAF1000FBAD00020D6E62DE9F05F0746E5
:1069E0000E460125A7F1140007B200BFC7EB071040
:1069F000C0EBC00058490844093005EB450100EBE5
:106A00004104B4F90000FFF79AFEB04205D1D4F872
:106A10000200FFF793FEBDE8F09FB4F90000FFF716
:106A20008EFEB04208DD34F9060CFFF788FEB04256
:106A300002DA681E05B203E0681C05B20E2DD5DD32
:106A400000BF0F2D21DBC7EB0710C0EBC000424990
:106A5000084400F10F04B4F9000034F9061C884220
:106A600009DD34F9060CB04202DB54F8040CD2E71D
:106A7000D4F80200CFE734F9060CB04202DC54F837
:106A8000040CC8E7D4F80200C5E7C7EB0710C0EB59
:106A9000C00031490844093005EB450100EB4104D1
:106AA000B4F90600FFF74BFE0146B4F90000FFF70A
:106AB00046FE081A05B2BDB1B4F90000FFF73FFE6B
:106AC000A6EB000A50460BF049FC81462349484694
:106AD0000BF0A4FC814628460BF040FC8246514650
:106AE00048460BF009FB8146A068FFF727FE0146E8
:106AF000D4F80200FFF722FEA1EB000A50460BF08B
:106B00002DFC8046002140460BF0B8FB15D04146D5
:106B100048460BF083FC8146104948460BF0ECFADE
:106B20008146D4F80200FFF709FE83460BF016FCFD
:106B3000824649460BF072FA814648460BF0D2FB7A
:106B400069E7000074000020FE2C0208482C0208AF
:106B5000202C0208982C0208526D002000007A4474
:106B60002DE9F0410027AD4C52E1FFF789FDB84215
:106B70007EDD94F92300C0F30710A949C85594F8A5
:106B80002700002875D194F82D00002872D03846CF
:106B9000FFF73AFD064694F82800A8BB14F8235FD7
:106BA00005F0F00500BF68B22070A07A233C0C28E5
:106BB0000CDB94F82D00162808DCB6F5006F01D91F
:106BC000012000E0002084F8260007E0B6F5006F01
:106BD00001D3012000E0002084F8260094F82D0065
:106BE00017280BDB94F82D001E2807DCB6F5006F84
:106BF00001D3012000E0002084F8260094F826004C
:106C000018B14FF47A7001E002E000200646D9E0A6
:106C100094F828000128FAD114F8235F05F0F00554
:106C200000BF68B22070A07A233C1A286FD2DFE838
:106C300000F0B00D0E11120F1013143D3E646F736F
:106C400078A77D7E82699293949596A800BF00BF35
:106C500000BF00BF00BF00BF00BF3846FFF7D4FC35
:106C6000B0F57A6F0DDD94F8235005F0F00502E0E1
:106C7000C3E0CAE0ACE045F0010568B284F8230047
:106C80000DE03846FFF7C0FC502808DA94F823508E
:106C900005F0F00545F0020568B284F82300B1B2B2
:106CA00094F82D00FFF74CFD064673E000BF384610
:106CB000FFF7AAFC40F6B831884209DD94F823506A
:106CC00005F0F00545F0010568B284F823000DE0F9
:106CD0003846FFF799FC502808DA94F8235005F05D
:106CE000F00545F0020568B284F82300B1B294F8CB
:106CF0002D00FFF725FD06464CE0B008FFF78AFCA3
:106D0000064647E0B008FFF78BFC064642E040E04D
:106D100044487043060B3DE044F620607043060B88
:106D200038E044F620607043060B33E000BF3D4876
:106D30007043060B2EE0CC20B0EB960F01D9002655
:106D400008E0CC20C0EB9600364948434FF44C7124
:106D5000B0FBF1F61EE000BF00BF00BF00BFB108EE
:106D60003846FFF763FC6421B0FBF1F694F82D0080
:106D700031B2FFF732FE06464FF47A70464309E01F
:106D800000BF3846FFF77EFC4FF47A7100FB01F636
:106D900000E000BF00BF94F8290048B994F82C1017
:106DA00094F82B0001EB0020642101FB006609E050
:106DB00094F82C1094F82B0001EB00206FF0630185
:106DC00001FB00663046FFF7B9FCC4F81E001CE06A
:106DD0001E34657905F0F00500BF68B26071384671
:106DE000FFF712FC800840F6B831484340F2FF310B
:106DF000B0FBF1F044F81E0907E094F8235005F0C9
:106E0000F00500BF68B284F82300781CC7B22E34A6
:106E1000202FFFF6AAAEBDE8F08100005F6F0020D2
:106E20001F750020A086010070B50025FE4840783F
:106E300001282CD172B60020FB494870F6F7D8FA29
:106E4000FA48F6F70AFB00240FE0C4EBC40202EB99
:106E50000412F74B03EB4201F64A2E2303FB0420F6
:106E60001A4609F0C8F8601C84B2202CEDDB4FF400
:106E7000B8652A46EF49ED48F6F7ECFB4FF47A7116
:106E8000EA48801EF6F70DFBF6F7B8FA62B6E64858
:106E90008078012832D172B60020E3498870F6F775
:106EA000A7FAE548F6F7D9FA00240EE004EB44020D
:106EB00002EB0412E14BD118DE4A132303FB04203A
:106EC0001A4609F098F8601C84B2DD4800888442B4
:106ED000ECDBDB48008800EB400101EB001085B2E1
:106EE0002A46D449D448F6F7B5FB4FF47A71D24814
:106EF000801EF6F7D6FAF6F781FA62B6CA48C0786D
:106F000001282BD10020C849C87072B6F6F770FA74
:106F1000CC48F6F7A2FA00240EE0C4EB0412C2EB50
:106F2000C202C94BD118C34A692303FB04201A4685
:106F300009F061F8601C84B2052CEEDB40F20D25EF
:106F40002A46BC49BF48F6F785FB4FF47A71BD4825
:106F5000801EF6F7A6FAF6F751FA62B6B248007943
:106F600001281CD172B6F6F743FAB848F6F775FA5D
:106F70001422B749B548801CF6F76CFB1422B549BA
:106F8000B2483430F6F766FB42F21071AF48F6F7BC
:106F900088FAF6F733FA62B60020A349087170BD8B
:106FA00010B5044672B6F6F723FA04F0010010B1EA
:106FB000A948F6F752FA04F0020018B19B48801E67
:106FC000F6F74BFA04F0040018B19B48801EF6F760
:106FD00044FA04F0080018B19A48801EF6F73DFA0A
:106FE00004F0100010B19948F6F737FA04F02000C9
:106FF00010B19A48F6F731FAF6F700FA62B6FBF7E5
:10700000C5FD10BD70B586B0002500268748801EDE
:10701000F6F764FA05464FF6FF7085427ED172B6E8
:10702000F6F7E6F98148801EF6F717FA00248EE09D
:1070300022468BA1684608F043FDC4EBC40101EB76
:1070400004117B4A02EB41001522694608F0D3FF88
:10705000C4EBC40000EB0410754901EB400000993B
:1070600040F8151F019941609DF808100172002039
:10707000C4EBC40101EB04116D4A02EB4101C1F8FC
:107080001E000120C4EBC40101EB041102EB41011D
:1070900081F822000020C4EBC40101EB041102EBD3
:1070A000410181F82300C4EBC40101EB041102EBA0
:1070B000410181F82400C4EBC40101EB041102EB8F
:1070C000410181F82500C4EBC40101EB041102EB7E
:1070D000410181F82600C4EBC40101EB041102EB6D
:1070E000410181F82700C4EBC40101EB041102EB5C
:1070F000410181F82800C4EBC40101EB041102EB4B
:10710000410181F82900C4EBC40101EB041102EB39
:10711000410181F82A00C4EBC40100E030E001EB3A
:10712000041102EB410181F82B00C4EBC40101EB17
:10713000041102EB410181F82C00C4EBC40101EB06
:10714000041102EB410181F82D00601C84B2202C57
:10715000FFF66EAF4FF4B86632463549354808F051
:107160004AFF324633493148F6F774FA4FF47A71E0
:107170002E48801EF6F795F9F6F740F962B624E03E
:107180004FF4B86632462A492848F6F74BFA0024ED
:1071900019E0C4EBC40000EB0410254901EB4000EA
:1071A00090F82D000F2809D0C4EBC40000EB0410A8
:1071B00001EB400090F82D00192802D1E0B2F7F75A
:1071C000DCF9601C84B20B2CE3DB1B48801EF6F755
:1071D00085F905464FF6FF70854271D172B6F6F714
:1071E00007F91548801EF6F738F900244FE004EB44
:1071F000440000EB04101149014404EBC4001A4A96
:10720000104402680A6042684A60007A087204EB1F
:10721000440000EB04100949084404EBC401124A7D
:1072200011440A6822E00000E201002002F0030895
:107230005F6F00203F75002002F803083F7D0020AB
:10724000EA01002002E00308526D0020000004085B
:1072500098010020AC01002000E8030800080408A1
:1072600054332D41492575004A2A020840F8062F5B
:107270004A684260097A0172002004EB440101EB84
:107280000411484A1144C1F80F00601C84B2342C28
:10729000ADDB4FF4777632464249434808F0ABFE07
:1072A000324641494148F6F7D5F94FF47A713F48E3
:1072B000801EF6F7F6F8F6F7A1F862B607E0FFE7EA
:1072C0004FF47776324637493848F6F7ABF9384805
:1072D000F6F704F905464FF6FF70854220D172B6E5
:1072E000F6F786F83248F6F7B8F840F20D21314843
:1072F00008F000FF40F20D2632462E492A4808F0D9
:107300007AFE324628492A48801CF6F7A3F94FF442
:107310007A712748F6F7C5F8F6F770F862B607E015
:1073200040F20D26324623492148801CF6F77AF9AF
:107330002148F6F7D3F8054642F21070854208D08E
:1073400014211E4808F0D6FE14211D4808F0D2FE74
:107350000BE0142219491848801CF6F763F914222F
:10736000174915483430F6F75DF9002415E0C4EBF1
:10737000C40000EB0410134901EB400090F82D000D
:1073800048B90120C4EBC40101EB04110D4A02EB22
:10739000410181F82800601C84B2202CE7DB06B094
:1073A00070BD00003F7D00203F75002002F80308FB
:1073B00000E00308526D002000000408980100203E
:1073C000AC0100205F6F002010B545F25550F2F778
:1073D00033FC0420F2F733FC4FF47A60F2F732FC0E
:1073E000F2F738FCF2F731FC10BD0000002801D0A4
:1073F000D14B036011B1D04808380860002A02D090
:10740000CD48001F10607047412801D2012070470D
:1074100000207047C94800787047C949085C401C83
:107420007047C849084410F8010C70472DE9F04135
:1074300006460C463046FFF7F4FF00256F1E7CB170
:1074400055212180676025720421A172C2B20021FA
:107450000120FDF709FE206184F87052D4F87442CF
:10746000DCB16F202080676025720820A07204F1D3
:107470001000074604F0D4FF00221146384604F0FD
:10748000D8FF00220121384604F0D3FF0022022158
:10749000384604F0CEFF84F870523046BDE8F04123
:1074A000FEF7DDBD10B503460C4600221846FFF777
:1074B000B8FF402B08D2C1B20120FEF77CFB014689
:1074C000204605F076F80246104610BD2DE9F0433F
:1074D000ADF51B7D814608469846A39DA29CFFF70B
:1074E000A0FF0227FE1E4F2A42D008DC1C2A32D001
:1074F000242A68D04B2A1BD04D2A08D11EE0512ADD
:1075000066D0552A39D06F2A41D0752A6CD02770A1
:10751000202028703046002806DBB8F1FF3F03D05A
:1075200027703220287030460DF51B7DBDE8F083B2
:1075300002460021484604F0D7FBECE7C1B2012027
:10754000FEF739FB014601A805F033F801A94846CA
:1075500004F087FCDFE7C1B20120FEF76CFB0146B7
:1075600001A805F026F801A9484604F07AFCD2E704
:107570000021484604F07BFDCDE7C2B20021012086
:10758000FDF772FD0146484604F01EFEC3E797A8CA
:1075900004F046FF0022114697A804F04AFF00229B
:1075A000012197A804F045FF0022022197A804F0CA
:1075B00040FF0022032197A804F03BFF97A948460B
:1075C00004F01EFBA7E70021484604F050FDA2E7A7
:1075D000C1B20120FDF7EBFC08B1012100E0002160
:1075E000484604F03CFA96E7C1B20120FEF764FB7E
:1075F0000146484604F03BFD8DE770B5ADF51A7DB8
:10760000044600256A4604F11000D4F8681203F01D
:10761000F4FC0222002808DA84F86D22252084F880
:107620006E0200200DF51A7D70BD2089822809D0D8
:10763000E068401C06D084F86D22322084F86E0287
:107640000020EFE76068FFF7ECFE0146208909267D
:1076500051285FD008DC0DF10D031C2849D02428E7
:107660000AD04D2808D133E055280CD0672803D024
:107670006F2801D0752818D084F86D22202084F856
:107680006E022846CEE79DF80200042804D084F854
:107690006D2284F86E62F4E7CAB294F86C1201208D
:1076A000029BFDF743FE0125EBE79DF80200092848
:1076B00004D084F86D2284F86E62E2E70298CAB2C0
:1076C000C3B294F86C120120FEF7B2F90125D8E795
:1076D0009DF80200072804D084F86D2284F86E62B9
:1076E000CFE7CAB294F86C120120FEF74BF90125DE
:1076F000C7E79DF80200072804D084F86D2284F8BB
:107700006E62BEE7CAB294F86C120120FEF76FFBFE
:107710000125B6E79DF80200012804D084F86D2207
:1077200084F86E62ADE79DF80820C9B20120FDF72C
:1077300041FC0125A5E70000B02D0208E901002069
:1077400060670020A0670020002801D0F84B03608C
:1077500011B1F74808380860002A02D0F448001F29
:1077600010607047401E704710B502460C4600215D
:107770001046FFF7F7FF802A08D2C1B20020FEF7BB
:107780001AFA0146204604F014FF0146084610BDCF
:10779000812801D20120704700207047E548007819
:1077A0007047401C70472DE9F04105460027002432
:1077B000802D11D2E04EEAB2E1B20020FDF754FC78
:1077C000B04206D0EAB2E1B20020FDF74DFC074618
:1077D00002E0641C102CEED33846BDE8F0812DE9A0
:1077E000F041054600240026802D0CD2D24FEAB28B
:1077F000E1B20020FDF738FCB84201D0661C02E07F
:10780000641C102CF3D33046E7E710B50B46114645
:107810000022802809D241B1102906D8062904D0B7
:10782000C2B20020FDF782FD0122104610BD10B546
:10783000002280280BD251B1102908D8062906D081
:10784000C2B2C9B2BC4B0020FDF770FD0122104648
:1078500010BD2DE9F04FADF51B7D8246DDF8949209
:10786000DDF8908208461F4600240026FFF77AFFC5
:1078700005464FF0FF3B512A7ED00CDC4B2A2DD021
:1078800004DC1C2A3FD0242A11D17AE04D2A2CD0C6
:107890004F2A0CD145E0682A6FD004DC552A46D027
:1078A000572A04D18AE06F2A4AD0752A7CD0022058
:1078B00088F80000202089F800005C46002C08DBD6
:1078C0007F1C06D0022088F80000322089F80000D2
:1078D0005C460DF51B7D2046BDE8F08F2A4602214F
:1078E000504604F001FA0446E8E7E9B20020FEF74A
:1078F00062F9014601A804F05CFE01A9504604F0BB
:10790000B0FA0446DAE7E9B20020FEF794F901463E
:1079100001A804F04EFE01A9504604F0A2FA044664
:10792000CCE70221504604F0A2FB0446C6E72846F5
:10793000FFF739FF0146504604F046FC0446BDE718
:1079400097A804F06DFD0022114697A804F071FD80
:107950000022012197A804F06CFD0022022197A8C3
:1079600004F067FD0022032197A804F062FD97A9A7
:10797000504604F045F902E009E071E014E00446E5
:107980009CE70021504604F072FB044696E7E9B2FA
:107990000020FDF70CFB08B1012100E0002150465A
:1079A00004F05DF8044689E7E9B20020FEF784F9A7
:1079B0000146504604F05BFB04467FE787B1781C24
:1079C00014D0102F44D80021EAB20846FDF74CFB32
:1079D0005949884231D1504604F07AF804466DE79F
:1079E0001021504604F011FB044667E7EAB2F1B2F9
:1079F0000020FDF739FB5049884204D10AEB04000E
:107A000004F066F809E0EAB2F1B20020FDF72CFBC1
:107A100001460AEB040004F0D7FB0444B4F5167FDA
:107A200003DA761C102EE1D348E7052088F8000021
:107A3000122089F800005C4640E70021EAB20846BF
:107A4000FDF712FB0146504604F0BEFB044635E745
:107A5000022088F800002A2089F800005C462DE703
:107A60000021504604F0B0FB044627E72DE9F04121
:107A7000ADF51A7D04460D46164600276068FFF7EF
:107A800071FE80464046FFF783FE80B16A4604F1EE
:107A90001000D4F8681203F0B0FA022100280CDAC2
:107AA00029702520307000200DF51A7D95E6012003
:107AB00028701F2030700020F6E72089572807D053
:107AC000E268521C04D02970322030700020EBE7AD
:107AD000092251286AD00EDC0DF10D034B2877D016
:107AE00004DC1C283CD024280DD171E04D2825D081
:107AF0004F2808D16CE055280AD0572868D06F2845
:107B000066D075283ED02970202030703846CBE7EB
:107B10009DF80200042802D029703270F6E794F82C
:107B20006C2240460299FFF770FE0127EEE7000045
:107B3000DC2D0208EA01002000007F439DF80200CE
:107B4000072804D084F86D1284F86E22DEE708F06E
:107B5000FF0294F86C120020FDF714FF0127D5E70F
:107B60009DF80200072804D084F86D1284F86E2274
:107B7000CCE708F0FF0294F86C120020FEF737F90A
:107B80000127C3E79DF80200092804D084F86D128C
:107B900084F86E22BAE7029808F0FF02C3B294F8A4
:107BA0006C120020FDF744FF0127AFE79DF80200AB
:107BB000092804D084F86D1284F86E22A6E79DF897
:107BC000082008F0FF010020FDF7F4F901279DE7E8
:107BD00029702820307099E72DE9F04106460C46BF
:107BE0003046FFF7BFFD00256F1E7CB15521218077
:107BF000676025720421A172C2B200210846FDF718
:107C000033FA206184F87052D4F87442DCB16F20EA
:107C10002080676025720820A07204F110000746DA
:107C200004F0FEFB00221146384604F002FC00225C
:107C30000121384604F0FDFB00220221384604F001
:107C4000F8FB84F870523046BDE8F041FEF70ABAFE
:107C500030B5002203780C78A34201D0002030BD5B
:107C6000072B0BD9072309E084188D1864786D78E9
:107C7000AC4201D0002030BD521CD2B29A42F3D3A4
:107C800002890B899A4201D0002030BD2AB1837A43
:107C90008A7A934203D0002030BD012030BD072BEB
:107CA00000D90723002209E084188D18E47AED7AC0
:107CB000AC4201D0002030BD521CD2B29A42F3D364
:107CC000012030BDFD49FE4A09E00B78DB0705D0F5
:107CD0004B68834202D100200870704724319142E2
:107CE000F3D9704770B50020821EF449F44C0AE0C5
:107CF0000B7803F00703012B04D10B6A934201D8E0
:107D00001A4608462431A142F2D980254FF4616613
:107D100010B10570066270BDE8490AE00B7803F007
:107D20000703032B04D10B6A934201D81A46084675
:107D30002431A142F2D90028EDD00570066270BD51
:107D400042F2DC31DD4808F0F7B910B5DB4800221B
:107D5000DB4B0CE00178CC0704D0890701D4016A21
:107D600001B902700178090600D5027024309842EA
:107D7000F0D910BD30B5D14BD14C18E01D78ED07CE
:107D800014D05D68854211D1187884070CD432B1C3
:107D900040F0040018704FF0FF30186230BD20F042
:107DA00004001870196230BD196230BD2433A3423B
:107DB000E4D930BD70B50D4616460022BF4CC0490F
:107DC00013E02378DB070FD0636883420CD120785F
:107DD00080070CD4122204F10C01304608F00BF994
:107DE000A0682860012202E024348C42E9D91046C0
:107DF00070BD2DE9F04180460E460027AF4CB04DD6
:107E000010E0207800F0030001280AD1414604F177
:107E10000C0002F0EDFF20B10EB160683060012768
:107E200002E02434AC42ECD93846BDE8F0812DE9BB
:107E3000F04706460F4691460020A04C4FF461687B
:107E40009F4D24E02178C90720D06168B1421DD13F
:107E50001222494604F10C0008F0CDF8A760207802
:107E60009849820701D521620BE0420703D54FF004
:107E7000FF31216205E0020702D5C4F8208000E04E
:107E8000216220F002002070012002E02434AC4284
:107E9000D8D94FF0010A38B9884C03E02178C907D6
:107EA00017D02434AC42F9D9002810D1FFF71AFFBB
:107EB0000446002C0BD084F800A06660A760122254
:107EC000494604F10C0008F096F8C4F82080BDE89B
:107ED000F08784F800A06660A7601222494604F18A
:107EE0000C0008F088F8C4F820800120DCE72DE9B8
:107EF000F04105460F4610460026704C70491BE0C5
:107F00002278D20717D06268AA4214D12178890753
:107F10000FD40126122204F10C0108F06CF8A068BD
:107F200038602078010704D520F0080020706548EB
:107F30002062304679E724348C42E1D95F4803243B
:107F40004FF4616604E0027812F0810F0AD0243009
:107F50008842F8D9FFF7C6FE10B10470456006628A
:107F6000002062E704704560066200205DE770B59E
:107F70000D461646514C524916E02378DA0712D0C6
:107F8000636883420FD11222314604F10C0008F0DD
:107F900032F8A560207820F002002070400701D45C
:107FA0004848206270BD24348C42E6D970BD70B55B
:107FB00004460D4616460020FF2C14D23F4A04EB1F
:107FC000C40102EB8104217801F0030101290AD1E7
:107FD000122204F10C01184608F00DF860682860C0
:107FE000A0683060012070BD00203449344A06E0AA
:107FF0000B7803F00303012B00D1401C2431914284
:10800000F6D97047F0B5ADF5177D064600252B4C27
:108010002B4F28E0207800F00300012822D17019AE
:108020000821626803F060FE0544A18A701903F01C
:10803000ECFF0544A27D52B104F1170101A804F040
:1080400016FC701901A903F074FE05440AE0227BB6
:1080500004F10D0101A804F00AFC701901A903F054
:1080600068FE05442434BC42D4D90DF5177D28465A
:10807000F0BD2DE9F04FADF5197D81460D46002785
:10808000B84605F11800989004F0CAF9002211468C
:10809000989804F0CEF900220121989804F0C9F9CB
:1080A00000220221989804F0C4F9E86AC0F5167B12
:1080B00000202863FFF798FF824605E01C8100201E
:1080C000D4A40020805101005FEA0A0004D0A86A0D
:1080D0000123082805D007E000200DF5197DBDE833
:1080E000F08FC5F844A0AB63686C00280ADAAA6B6D
:1080F000511C0144012902DA6A64AB6302E0A963FE
:1081000040426864A86B504501D90020E5E7696CDE
:108110000144491E00910099514501D9CDF800A0B4
:10812000414C012600E02434217801F003010129AB
:10813000F9D105E0217801F00301012904D02434AC
:10814000B042F7D1019645E02434761CF8E7BBF144
:10815000110F05D201220221989804F06AF93CE03F
:1081600009EB07000821626803F0BEFD804607EBBB
:108170000800A18A484403F048FF8044A27D62B110
:1081800004F1170102A804F072FB07EB0800484451
:1081900002A903F0CEFD40440CE0227B04F10D0166
:1081A00002A804F064FB07EB0800484402A903F0AE
:1081B000C0FD4044ABEB000B0744B046761C2434B2
:1081C000286B401C286300E02434207800F0030072
:1081D0000128F9D100988642B9D90198012804D123
:1081E00001220021989804F024F9D04504D10122FD
:1081F0001146989804F01DF938466EE730B50A49E3
:1082000000230A4C0DE00A7812F0810F08D05207C3
:1082100006D40A6A824202D3121A0A6200E00B7084
:108220002431A142EFD930BD1C810020D4A400200C
:10823000002801D0DA4B036011B1D9480838086032
:10824000002A02D0D6480C3810607047412801D26D
:108250000120704700207047D24800787047D2490B
:10826000085C401C70477047D049084410F8010C66
:108270007047002070470020704700B50022FFF7CC
:10828000F3FF402801D2CA490A5C104600BD00B580
:10829000FFF7EAFF402802D2C54A0021115400BD71
:1082A0002DE9F04106460C463046FFF7DDFF4FF062
:1082B000FF3700258CB15521218067602572092187
:1082C000A172C2B200210320FCF7CEFE0AF026F80C
:1082D000206184F87052D4F8744254B36F20208027
:1082E000676025720820A07204F11000074604F0B0
:1082F00097F800221146384604F09BF8002201212D
:10830000384604F096F800220221384604F091F82D
:108310003046FFF7B0FF28B101220321384604F0B0
:1083200088F804E000220321384604F082F884F83B
:1083300070523046BDE8F0419FE70020704793E758
:1083400010B503460C4600221846FFF78DFF402B60
:1083500008D2C1B20320FDF72EFC0146204604F0EE
:1083600028F90246104610BD2DE9F047ADF51A7DFB
:10837000824608469946A39EA29DFFF775FF0446D4
:108380004FF002084FF0FF374F2A42D008DC1C2A7A
:1083900032D0242A76D04B2A1BD04D2A06D11EE09B
:1083A000542A74D0552A39D06F2A43D085F80080DA
:1083B000202030703846002807DBB9F1FF3F04D099
:1083C00085F800803220307038460DF51A7DBDE802
:1083D000F08722460321504603F086FCEBE7E1B22A
:1083E0000320FDF7E8FB0146684604F0E2F8694621
:1083F000504603F036FDDEE7E1B20320FDF71BFC3B
:108400000146684604F0D5F86946504603F029FD58
:10841000D1E70321504603F02AFECCE7E2B2002167
:108420000320FCF721FE09F079FF0146504603F0D6
:108430001EFEC0E796A803F0F3FF0022114696A89F
:1084400003F0F7FF0022012196A803F0F2FF0022BB
:10845000022196A803F0EDFF2046FFF70CFF28B19C
:108460000122032196A803F0E4FF04E00022032187
:1084700096A803F0DEFF96A9504603F0C1FB9AE7E9
:1084800000E004E00021504603F0F1FD93E72046B0
:10849000FDF758FE0146504603F0E9FD8BE7F0B5C5
:1084A000ADF51B7D044600256A4604F11000D4F8A2
:1084B000681202F0A2FD02262527002807DA84F8B8
:1084C0006D6284F86E7200200DF51B7DF0BDE068D2
:1084D000401C06D084F86D62322084F86E020020C1
:1084E000F2E720894F2854D008DC1C2851D02428DA
:1084F0004FD04B284DD04D280BD14AE004F26E23CB
:108500005A1E512822D054282DD0552808D06F2823
:108510003FD084F86D62202084F86E022846D3E7AD
:108520000921684604F0ABFB05462800F6D0029806
:10853000012805D80298C1B26068FFF7FEFEEDE79A
:10854000002584F86D6284F86E72E7E701216846C1
:1085500004F095FB05462800E0D09DF808106068FF
:10856000FFF7EDFEDAE70921684604F088FB0546CF
:108570002800D3D00298022805D20298C1B26068C0
:10858000FDF7E3FDCAE7002584F86D6284F86E729A
:10859000C4E784F86D62282084F86E02BEE700000C
:1085A000002E0208EB01002080670020C067002039
:1085B000F8A400200A0A02704170022070470029C6
:1085C00005D0027812020A80407802430A80022015
:1085D00070470A0C02700A0A4270817003207047CB
:1085E000002909D0027812040A60437842EA032283
:1085F0000A60807802430A60032070470A0E027006
:108600000A0C42700A0A8270C17004207047002967
:108610000DD0027812060A60437842EA03420A60EB
:10862000837842EA03220A60C07802430A60042089
:10863000704701700120704700290CD002781206A3
:1086400003D56FF0FF020A6001E000220A600078A3
:108650000A6802430A60012070470A0A02704170EA
:108660000220704700290FD00278120602D5254A51
:108670000A6001E000220A6003780A6842EA0322E5
:108680000A60407802430A60022070470A0C0270B8
:108690000A0A4270817003207047002914D00278C2
:1086A000120603D54FF07F420A6001E000220A6003
:1086B00003780A6842EA03420A60437842EA0322E6
:1086C0000A60807802430A60032070470A0E027035
:1086D0000A0C42700A0A8270C17004207047002997
:1086E0000DD0027812060A60437842EA03420A601B
:1086F000837842EA03220A60C07802430A600420B9
:10870000704700000000FFFF00280CD000290AD0AD
:108710004A68C0F801204988A0F8051006210170B8
:10872000002101818172704738B50546049C002004
:10873000002C07D0012C04D128460094FDF7F2FD4F
:1087400080B238BD00200090284601F0E6F980B2E2
:1087500038BD30B40446029B0020002B05D0012B0D
:1087600008D1204630BCFDF74EBE204630BC002369
:1087700001F0F3B930BC7047002907D0012903D0BC
:10878000022901D0042903D1FDF704BF01F04ABA40
:108790007047002907D0012903D0022901D00429FC
:1087A00003D1FDF7DDBE01F02DBA7047F649002078
:1087B00008707047F4484068704701460120B1F5E1
:1087C000800F04D2F04A5160F04A116070470020D7
:1087D0007047ED494968814201D10120704700206E
:1087E0007047FDF75BBB10B5FEF7D8FF441CFEF7E2
:1087F00011FE044401F090FB044402F029F8044403
:10880000FFF72AFD044404F0A4FC204410BD2DE928
:10881000F0410F4690460025012806D10821396015
:10882000D9494968C8F800100125441E01266DB9D0
:10883000641EFEF7B3FF0646B44207D2022038603A
:108840002046FEF7AEFFC8F8000001256DB9A41B55
:10885000FEF7E0FD0646B44207D20020386020460D
:10886000FEF7DBFDC8F8000001256DB9A41B01F07F
:1088700053FB0646B44207D201203860204601F07F
:108880004EFBC8F8000001256DB9A41B01F0E0FF04
:108890000646B44207D204203860204601F0DBFFD0
:1088A000C8F8000001256DB9A41BFFF7D5FC0646EA
:1088B000B44207D2032038602046FFF7D0FCC8F846
:1088C0000000012565B9A41B04F043FC844207D2D3
:1088D00080203860204604F03FFCC8F800000125E5
:1088E0002846BDE8F0812DE9FF4FADF51D7D064618
:1088F000DDF8A892AB9F9846002400250020029046
:1089000001909F98A0494FF0FF3A4F2878D020DC83
:108910003F2870D00EDC1E286ED006DC0B286CD0F1
:108920000C286BD01C2839D162E12C2867D03E2856
:1089300034D13CE14B284AD006DC402878D0462888
:1089400077D049282AD146E14C2820D04D2825D17E
:1089500044E0792860D00EDC6B286BD006DC602800
:1089600069D0612868D0622818D193E070284DD072
:10897000782813D161E0DFF818B2B0F57A7F70D0B3
:1089800006DC8B286ED09B286DD0D12806D1C4E0A0
:10899000A0F54070E93867D0012870D0022089F82E
:1089A0000000202038705446002C0BDB9F984C2888
:1089B00008D0B8F1FF3F05D0022089F8000032202E
:1089C000387054460DF5217D2046BDE8F08F4A6889
:1089D0000821304603F088F90446E5E7FDF75CFA24
:1089E000014603A803F0E5FD03A9304603F039FA78
:1089F0000446D9E704E00BE1F3E0E5E040E034E0D1
:108A00000821304603F033FB0446CDE709783046B1
:108A100003F02DFB0446C7E7FDF799FA014603A8CA
:108A200003F0C7FD03A9304603F01BFA0446BBE779
:108A3000F6E00AE0C2E04DE038E0FFF7D2FE014682
:108A4000304603F0E2FA0446AEE7FDF782FA01464B
:108A500003A803F0AEFD03A9304603F002FA044672
:108A6000A2E7E5E01CE0CDE0F6E04AA103A803F0B0
:108A7000A0FD03A9304603F0F4F9044694E7F2E0C0
:108A800046A103A803F095FD03A9304603F0E9F9D8
:108A9000044689E70121304603F0B7FA044683E72C
:108AA0000C21304603F0B1FA04467DE799A803F0A3
:108AB000B7FCE8B201F0B6FC0246E9B299A803F0AF
:108AC000B8FC6D1C282DF4D399A9304603F098F812
:108AD000044669E799A803F0A3FCE9B2002299A82B
:108AE00003F0A7FC6D1C332DF7D3274C08344FF44B
:108AF000806509E0A06830B1804720B1217801226B
:108B000099A803F096FC38342088A842F2D399A99A
:108B1000304603F075F8044646E7FFF764FE8346E7
:108B2000B8F1000F0FD0B8F1FF3F12D001AA02A98F
:108B30004046FFF76CFE30B3DDE90121304603F01B
:108B4000D3F8044630E75946304603F05EFA04464F
:108B50002AE7012514E001AA02A92846FFF757FEDB
:108B6000DDE90121301903F0BFF804442044B0F5D9
:108B7000167F04DB362038706FF0010414E76D1C9B
:108B80005D45E8D910E70BE0EC010020040000206F
:108B9000E0670020302E382E30000000312E3000EB
:108BA000022089F800002A2038705446FCE64FF471
:108BB0001671304603F029FA0446F5E603213046E3
:108BC00003F055FA0446EFE64EF66021304603F016
:108BD0001CFA0446E8E60021304603F016FA044683
:108BE000E2E64FF416713046FFF70CFA0446DBE676
:108BF000FEA103A803F0DDFC03A9304603F031F920
:108C00000446D1E60021304603F0FFF90446CBE6E6
:108C100000F0F0FF0146304603F0F7F90446C3E6E2
:108C200000F0ECFF0146304603F0EFF90446BBE6E6
:108C3000BBF800103019694303F0E7F904442044FD
:108C4000B0F5167F04DB362038706FF00104ABE618
:108C50006D1C052DECD9A7E6BBF80210304603F0D9
:108C6000D4F90446A0E6BBF82610304603F0CDF94F
:108C7000044699E670B5ADF51A7D044600256A46AE
:108C800004F11000D4F8681202F0B7F90223252687
:108C9000002807DA84F86D3284F86E6200200DF542
:108CA0001A7D70BD20894C2809D0E168491C06D086
:108CB00084F86D32322084F86E020020EFE70DF167
:108CC0000D0178285ED00ADC4FF00902402834D02C
:108CD000462861D04B2814D04D280BD165E0792867
:108CE00047D0B0F57A7F0AD0A0F54070E9386AD055
:108CF00001286FD084F86D32202084F86E02284657
:108D0000CDE79DF802000C2804D084F86D3284F879
:108D10006E22F4E7BDF80800082809D10398FFF790
:108D20004CFD28B10398C0B2FDF775F90125E6E7BF
:108D300084F86D3284F86E62E1E79DF80200022843
:108D400004D084F86D3284F86E22D8E70298401E71
:108D5000FD2809D80298C4B2204600F031FF204611
:108D6000FDF759F90125CAE784F86D3284F86E627F
:108D7000C5E79DF802000728C1D10846FDF7EBF8CA
:108D80000125BCE79DF802000228B8D1029880B204
:108D9000FDF7F7F80125B2E79DF802000728AED1EC
:108DA0000846FDF7E3F80125A9E79DF8020007282A
:108DB00004D084F86D3284F86E22A0E70846FBF7F1
:108DC000B3FF01259BE79DF80200022897D10125FA
:108DD00095E7FFE79DF80200022890D101258EE774
:108DE0002DE9F04704468846914600252088022652
:108DF000282709283DD2DFE800F0052B0E19223C78
:108E00003C3C34006068FEF7FFFA00B384F86D6202
:108E100084F86E722DE06068FEF7BAFCB8B14A467D
:108E200041462046FEF722FE054622E06068FFF735
:108E30000DFA60B184F86D6284F86E7219E06068B2
:108E400001F000FD18B1204601F088FE054610E053
:108E5000606801F05BF860B1204601F0EAF9054670
:108E600007E06068FFF7B5FC18B12046FFF702FF86
:108E700005462846BDE8F087012070475F484068F6
:108E8000704710B502460C4600205C4949688A428A
:108E900007D1FDF701F801462046BDE8104003F078
:108EA00088BB10BD002801D0554B036011B1544858
:108EB0005C300860002A02D0514870301060704762
:108EC0000021002802D104E0491C001D0268521C48
:108ED000FAD1084670470246484808304FF480638C
:108EE00002E0914204D0383001889942F9D3002041
:108EF00070472DE9FC4106464FF0FF300C69002C0D
:108F000019D04A69BAB10A89022332254B2A14D0F2
:108F10004F2A26D0B769002F0BD00B764D7601F182
:108F20001900431ECDE90030CB68B5694968204679
:108F3000A847BDE8FC810020FBE7CA68521C02D0AC
:108F40000B764D76F5E70888082802D12B4A52683F
:108F50004A604A68014602B02046BDE8F04102F08E
:108F6000C3BECA68521C02D00B764D76E1E7098871
:108F70002046BDE8FC4103F07AB82DE9F0410446F3
:108F80004FF0FF372088FFF7A6FF054601264FF078
:108F90001F0875B1296941B16068884728B1214629
:108FA0002846FFF7A6FF074606E0267684F81980D4
:108FB00002E0267684F81980384692E410B502461D
:108FC0000C4600202060A06020611046FFF783FF60
:108FD00038B1036A2BB104F1100204F108012046F4
:108FE00098472068D0B1FFF76BFF0BE04261636EDA
:108FF00065742050726F647563740000EC0100208A
:10900000202E02086060A06850B1FFF759FFE060B1
:10901000206938B1FFF754FF606110BD0020E4E71C
:109020000020F4E70020F7E710B5FFF754FF08B180
:10903000406A10BD002010BD70B50D4616460024D4
:10904000FFF749FF28B143691BB1314628469847CD
:109050000446204670BD2DE9F043ADF5197D8146EB
:109060000E4617464FF0000800209890FFF7BBFB14
:10907000054601241FE097AA98A92046FFF7C7FBE1
:10908000C0B1989880B2FFF726FF98B143698BB1C1
:1090900001A99798984768B101A9484603F0DAFA00
:1090A00040B14FF001080EB1989830602FB19798F9
:1090B000386002E0641CAC42DDD90DF5197D4046F4
:1090C000BDE8F08370B50D46002480B2FFF703FFC2
:1090D00020B102692846904700B10124204670BDA6
:1090E00010B5FF4800210171417181710172417217
:1090F000816200F124031A6822F0080222F02002A3
:1091000022F0010222F002021A60F64A12788272FC
:10911000F54A127802730122C2728182C17100F095
:10912000BAFE012010BD70470022FF2911D0012393
:1091300003704170012143185A70491C0729FADB5A
:109140000281827200214318DA72491C0729FADB76
:10915000704702704270EDE710B588B004460020F9
:10916000E24A00211378002B0BD0117000236A46CD
:1091700003A9DF4803F0F4FE80B20121217008B09A
:1091800010BDDC4A1378002BF9D011700022501E5C
:10919000014603F0D0FF082002212170EFE72DE9FE
:1091A000F043ADF5197D8946A09D90461E464FF6C9
:1091B000FF77002455218DF85C12FF218DF85D1298
:1091C0008DF85E0203F014FC014648468DF85F926C
:1091D00003F00EFC014640468DF8608203F008FC67
:1091E0000146280A8DF8610203F002FC0146E8B24C
:1091F0008DF8620203F0FCFBC0438DF863023DB9B9
:109200000EE0305D394603F008FC0746641CA4B24A
:10921000AC42F6D3F8438DF85802000A8DF8590293
:1092200000F024FE012000F016FEB5B19899979841
:10923000CDE900012A46314602A806F0DCFE0DEB1E
:109240000500BDF8581201810A35A9B2684600F040
:1092500026FE0DF5197DBDE8F083082197A800F0E2
:109260001EFEF6E72DE9F843002400949C4D4FF0D4
:10927000010805F12C07287900280CD04FF00209CD
:1092800001282AD005F12406022865D003286FD0D2
:109290002C71BDE8F88300F013FE38B100F0FBFD3F
:1092A000E879FF28F5D2401CE871F2E7514668469C
:1092B00000F008FE0028ECD000F0EDFDE879FF2872
:1092C00001D2401CE8719DF80000552801D185F8B5
:1092D000048085F804803870DBE700F0C4FD5A286C
:1092E00003D9FBF7F8FD2C71D3E700F0E9FD40B19D
:1092F00000F0D1FDE879FF2801D2401CE8712C7103
:10930000C7E75146684600F0DDFD0028C1D000F0F7
:10931000C2FDE879FF2801D2401CE8719DF80000E9
:10932000FF21FF2809D055280DD003280ED0192879
:109330000CD0FBF7CFFD2C71ABE76C8229707970F4
:1093400085F80490A5E785F80480A2E76C8229706F
:10935000787085F804909CE700F085FD5A2808D9BC
:10936000306840F001003060FBF7B5FD2C7190E7EC
:10937000E6E000F0A5FD60B100F08DFDE879FF2882
:1093800001D2401CE871306840F0010030602C715F
:109390007FE75146684600F095FD002885D000F033
:1093A0007AFDE879FF2801D2401CE871688A98B1FB
:1093B000012839D04FF00308022842D003284DD0AD
:1093C000042859D0052866D0306840F0010030608C
:1093D000FBF780FD2C715CE729789DF8000003F015
:1093E00007FB28709DF800002872397855290CD1A8
:1093F0007978FF2909D1072807D900F04CFDE879D1
:10940000FF2801D2401CE8712C719DF80000B87053
:109410003878FF2802D17878192802D0A5F8128070
:1094200037E7FBF75AFD34E729789DF8000003F091
:10943000DFFA28709DF80000A871F870A5F8129066
:1094400027E729789DF8000003F0D2FA28709DF8EC
:10945000000068723871A5F812801AE729789DF823
:10946000000003F0C5FA28709DF800000102A982EF
:109470007871042068820CE729789DF8000003F0D9
:10948000B7FA2870A98A9DF800000144A982B87132
:1094900005206882FDE69DF80000F871104806215D
:1094A0002C30FBF717FCF979BA7901EB02218142E4
:1094B00002D1FBF712FDECE629789DF8000003F0DD
:1094C00097FA287055281BD0FBF704FD306840F050
:1094D0000100306000F0DFFCE879FF280ED20BE0DD
:1094E000B40300208E0100208F01002034040020EE
:1094F00038A5002035040020401CE8712C71C8E616
:10950000A88A48B1E98A884206D86C824FF6FF7073
:10951000288285F80480BCE638B1306840F001004C
:109520003060FBF7D7FC2C71B3E6A879A97A8842A2
:1095300001D0FF28F7D1306840F002003060F2E738
:1095400000F091FC5A2807D9306840F001003060E3
:10955000FBF7C1FC2C719CE600F0B2FC60B100F09E
:109560009AFCE879FF2801D2401CE871306840F08D
:10957000010030602C718CE65146684600F0A2FC78
:10958000002887D000F087FCE879FF2801D2401C32
:10959000E871688AA98A88420DD2298A9DF800005C
:1095A00003F03BFA2882688AAA6A9DF800101154D9
:1095B000401C68826DE609D1298A9DF8000003F0FD
:1095C0002CFA2882688A401C688262E6491C88421C
:1095D00095D1298A9DF8000003F01FFA2882A0F592
:1095E0007041B83907D0306840F001003060FBF7B7
:1095F00071FC2C714DE6A879A97A884201D0FF2828
:10960000F7D1306840F002003060F2E72DE9FF5FEB
:109610000024FE4EF178307B491C401CB1FBF0F277
:1096200000FB121101F0FF08B27A511CB1FBF0F3FC
:1096300000FB131101F0FF0BB1784B1CB3FBF0F5ED
:1096400000FB1530C0B2029006F1240A96F805C05E
:10965000DAF80030002523F004000390304601279B
:10966000407A4FF00409BCF1090F79D2DFE80CF021
:10967000051579DCF9F8F7F6F500B270F2703220D2
:10968000306203987771012420F0020020F001007D
:10969000CAF8000000F0FFFB3BE200F0E4FBB0F58D
:1096A000FA7F0ED3FBF717FCF57106207071DAF81C
:1096B000000020F0020020F00100CAF800000124A0
:1096C00027E2DAF80000C10708D0FBF703FCDAF85C
:1096D000000020F00100CAF800001AE28107DBD583
:1096E000317A072932D2DFE801F004123129311F23
:1096F0001A00B179FF2929D020F00200757020F0FE
:109700000400CAF800000220707101241EE00095D8
:109710000023B27A717A0220FFF741FD16E040F093
:109720002000CAF8000011E040F02000CAF8000054
:10973000B079FF280AD00820707107E0B08A009045
:10974000B27A717A0420B36AFFF729FD707908288C
:10975000A2D0DAF8000020F00200CAF80000D8E138
:10976000D6E1019501A8FFF7F7FC30839DF80410BE
:1097700081B3022908D10090A54BB27AFF210620BF
:10978000FFF70DFD86F805909DF8040007280BD023
:10979000012814D0032503281DD0042827D005282C
:1097A0002FD006282DD035E0308B0090984BB27A20
:1097B000FF210620FFF7F3FC86F805902AE0308BA6
:1097C0000090934BB27AFF210620FFF7E8FC86F861
:1097D00005901FE022E0FBF77BFB0146308B0090F9
:1097E0008C4BB27A0520FFF7DAFC757112E0308BF2
:1097F0000090874BB27AB17B0520FFF7D0FC7571E2
:1098000008E0308B0090824BB27AB17B0520FFF7E5
:10981000C6FC75717078401C70707AE1F07A7070D7
:10982000012486F8059074E100F01DFBB0F5937FEC
:1098300007D9FBF750FBF07A707086F80590012489
:1098400067E1DAF80000C1070CD020F00100CAF887
:10985000000086F8059001245BE13AE1DCE0AAE033
:1098600084E024E08107D8D5B179B27A914215D14C
:10987000317A042908D0062909D0072901D0777147
:109880000DE086F805900AE086F8059007E040F0C4
:109890002000CAF8000086F8059000E07771DAF839
:1098A000000020F00200CAF80000012431E17078C5
:1098B00096F80BC0604503D202207071012428E1A4
:1098C00058070DD491420BD186F803B000235946B6
:1098D00001200095FFF763FCF5610720707118E126
:1098E000306A312818D249485B07006A00F101004C
:1098F00007D5594505D0757030620220707101247A
:1099000007E13062002318460095FFF748FCF56137
:10991000F57105207071FCE088451BD158070DD505
:109920000299F170002301200095FFF738FCB07A0E
:10993000B070F561376207207071EAE0F2700023C1
:1099400018460095FFF72BFCF5613762F57105208D
:109950007071DEE086F80380002341460120009507
:10996000FFF71DFCF56107207071D2E000F07BFA73
:109970005F2805D8F079042801D977710124C8E05F
:10998000F06970B10299F17000950023B27A01205C
:10999000FFF705FCB07AB070F56135620720707191
:1099A000B7E0F76100950023B27AB1781846FFF767
:1099B000F6FBF571ADE002EB82004FF4FA7808EBAC
:1099C000400900F050FA484505D2F079042801D941
:1099D000777101249DE0B07A401C00EB800008EB19
:1099E000400700F040FAB8420ED286F803B0009566
:1099F0000023B27A59460120FFF7D1FBB07AB0704C
:109A0000F56135620720707183E00000B403002027
:109A100038A50020C0AD0020990720D5B17991422A
:109A200002D1317A022908D077710124DAF80000D6
:109A300020F00200CAF800006BE00399CAF8001099
:109A4000B070F5710023014618460095FFF7A7FB9B
:109A5000B07AF0703562F56105207071E6E700F0CC
:109A600002FA5F2803D89AF80000C00751D0DAF84C
:109A70000000410704D5757002207071012421E0B7
:109A8000B178B27A914209D0F57100231846009559
:109A9000FFF785FBF5610520707113E0904509D053
:109AA00086F803800023414601200095FFF777FBED
:109AB000F56107E040F00400CAF80000757002206C
:109AC00070710124DAF8000020F00100CAF80000EB
:109AD0001FE019070ED5308B00905B4B717B062081
:109AE000FFF75DFBDAF8000020F00800CAF800007C
:109AF000777106E00146002307200095FFF74FFB32
:109B00007771DAF8000020F00200CAF8000000E0E7
:109B1000777104B02046BDE8F09F2DE9F04117466B
:109B2000069A06461C460020484D002A0FD1497867
:109B3000286861F30410286022463946424806F03E
:109B40005AFAA5F1240004837178417320462968EC
:109B500041F008012960BDE8F0812DE9F041064699
:109B600000273A4D243DA86A002801D1A962EA8263
:109B7000364C206881070BD4C00709D1FFF772FB70
:109B80002168880704D4C80702D128790028F5D1B4
:109B9000287940B92E49A87A0978884203D8FFF776
:109BA00035FD0028FBD12068810607D520F0200074
:109BB0002060AF8A01203070687A70703846CAE73A
:109BC000224924390873704721490978884206D808
:109BD0001E4924398872097B884200D9F0E7704712
:109BE0001A482438807A7047002802D0174924394F
:109BF000C872704715482438C07A70471348243813
